:100000000040002081630000C1630000C363000062
:1000100000000000000000000000000000000000E0
:10002000000000000000000000000000C5630000A8
:100030000000000000000000C7630000C96300006A
:10004000CB630000454A0000FD670000CB63000061
:10005000CB63000000000000CB630000CB63000016
:10006000CB630000CD6A0000A52C0000CB6300002C
:10007000CB630000CB630000CB630000CB630000C8
:10008000CB630000656C0000CB630000CB63000015
:10009000CB630000CB630000CB630000CB630000A8
:1000A000CB630000CB6300000000000000000000F4
:1000B0000000000000000000000000000000000040
:1000C00010B5064C2378002B07D1054B002B02D02E
:1000D000044800E000BF0123237010BD640200202B
:1000E0000000000050D40000044B10B5002B03D0DA
:1000F0000349044800E000BF10BDC04600000000F6
:100100006802002050D40000164B002B00D1144B85
:100110009D46402292029A1A924600218B460F4633
:100120001348144A121A0AF045FB0F4B002B00D05B
:1001300098470E4B002B00D0984700200021040068
:100140000D000D48002802D00C4800E000BF0AF066
:10015000F1FA2000290006F06FFB0AF0C5FAC0464C
:100160000000080000400020000000000000000027
:10017000640200209C2F002000000000000000000E
:100180000123034010D104280CD90268120909D0B8
:10019000531E9B001A1DC1180979002902D0013392
:1001A0009342F8D1180070470023FBE70378002B37
:1001B00003D05AB2002A01DB013070473F2293433B
:1001C000C03B59424B41C01803789343802BF4D174
:1001D0000130F9E710B500240378002B01D120008D
:1001E00010BDFFF7E3FF0134F6E770B5002204000D
:1001F0000D00411C092003F065F8002806D00123FA
:100200006200134343600023A34200DB70BD9A00E9
:10021000A958821891600133F6E770B5012803DC14
:100220001C2000F091FE70BD01230D6811201D42BD
:10023000F7D04868184206D1042804D90F23026871
:100240001340042B01D00E20EBE702F0A5FE6D1049
:100250000400002D03DDFFF7BDFFA84206DA1220DF
:10026000DFE72000FFF7A2FF0400013D012DF8D1D8
:1002700020787F2809DDDF280BDCF8233F22DB0014
:10028000800118406378134018430123400018434D
:10029000C9E7EF280BDCFC22637812019B011340B5
:1002A0003F220007000C0343A0781040ECE7F7283A
:1002B00012DCFC22637892021B031340E0228004CC
:1002C000520310403F221843E3781340FC220343BB
:1002D000A07812018001E8E701204042D5E7F0B59F
:1002E000070085B00D001C20012F06DD4C6801239E
:1002F00022001A40019203D10D2000F025FE54E0A7
:10030000022F02D08A681A42F6D001232E681E42BC
:1003100000D07EE0042E00D87BE01C41002C00DCE5
:100320001C000F2332681340092B29D173685B101E
:100330000193022F05D0AB68019A5B109A4200DD51
:100340000193019B01221F1B0137FB43DB171F4059
:10035000791C092002F0B6FF061E09D001237F0098
:100360001F4303002A68083347600199A14202DA5B
:10037000300005B0F0BD0134A100515802C3F4E7CC
:10038000042B46D1300002F007FEFFF723FF029056
:10039000022F04D0AB685B10984200DD0293029BF1
:1003A0009C4204DD002002F0F9FF0600E0E7300087
:1003B00002F0F2FD0700019B9C4222DC3000019715
:1003C00002F0EAFD03903800FFF7F0FE029B0134D3
:1003D0000700A342F7DA019BC71A380002F0DEFFDC
:1003E000061EC5D002F0D8FD0400286802F0D4FD36
:1003F000039A019B991A41183A0020000AF0BEF9AD
:10040000B6E73800FFF7D2FE019B070001330193E6
:10041000D1E7212071E7F8B54D680F00EB0706D44E
:10042000042D04D90F232E683340092B03D00B2051
:1004300000F08AFDF8BD6B6836095C10731EA3429C
:100440000FD80321200008F071F86421642803DC30
:100450000100032800DA03212800891902F062FF55
:1004600005002B6800201B09013B9C42E2D23A6840
:10047000A31C9B005A510123013464001C436C608F
:10048000D8E7F0B585B0012803DC1C2000F05CFD46
:100490002AE001244D682200022806D08B682342FE
:1004A00003D05C10002C00DC140001231D4200D09E
:1004B00073E0042D00D870E00F272B680E683B40D6
:1004C000042B27D1033B1E4205D1042E03D93368E8
:1004D0001F40042F01D00E20D8E72800FFF750FE60
:1004E000A04203DA0120404205B0F0BD280002F02E
:1004F00053FD0700300002F04FFD013C01003819A8
:100500000AF0EFFC0028EDD00123C01B01304000B1
:100510001843E9E7092B40D16B685B1000939C42BC
:10052000E0DC01231E4230D1042E2ED933683B403B
:10053000042B2AD1300002F02FFD012302900193F9
:100540000397671CBB00E858864203D101986400FA
:100550002043C9E7019B18420ED104280CD9036837
:10056000039A1340042B07D102F016FD01000298F4
:100570000AF092FC0028E9D0009B3C009F42E0DD9D
:10058000B0E71C00009B9C42ACDC631C9A00AA589C
:10059000B242F6D164000120DAE7212076E710B5F7
:1005A00002F0DEFC43000120184310BD10B57F2986
:1005B00002DC0170013010BD1A4B99420CDC402363
:1005C0008A115B42134303703F230B408021494251
:1005D000194341700230EEE7134B994210DC20239F
:1005E0000A135B4213433F24802203708B11524253
:1005F0002340214013430A43437082700330DAE7FB
:100600000A4B9942D7DCF0230370603B4370113BE7
:100610008A11FF3B1A4382703F2211401943C17077
:100620000430C8E7FF070000FFFF0000FF0F0100D4
:10063000F0B50D0085B0002803DC1C2000F084FC20
:100640000DE009680122080010400AD002AC1141F7
:100650002000FFF7ABFF011B200002F0ABFE0400FF
:100660001AE004293FD90F230C682340092B3AD103
:100670004B685B10019303239C46019B9A420EDD5D
:1006800002F08CFE041E07D02E68012502F084FCC7
:100690002F00019B9D421DDD200005B0F0BD013201
:1006A0009300CC580123234001D10D20C6E76410EC
:1006B0007F2C0DDD0D4E0223B44209DD0C4E634646
:1006C000B44205DD00270B4EE30FA6427B419B00A1
:1006D000C018D2E70135AB00F1583942E5D04910D6
:1006E000FFF764FFD5E72120A8E7C046FF07000019
:1006F000FFFF0000FF0F010010B5040001200840BB
:1007000010D104290DD90F230A681340042B08D1F6
:10071000080002F041FC010020000AF0BDFB43424A
:10072000584110BD0020FCE7F7B50F00012803DC9D
:100730001C2000F009FCFEBD01264D682E4006D1AC
:10074000042D04D90F222B681A40092A01D00B204E
:10075000EFE76A681B095410A34200D85C1E396891
:100760001E48FFF7C9FF01230190002813D1396803
:100770001B48FFF7C1FF002811D0002C0DD001232A
:10078000621C013C9C409200535123436B6004E087
:100790000136B200AB50B442FADA0020CBE73B6836
:1007A0000D20DA07C5D55B10002B11DD9C420FDB55
:1007B0009B00A200291DEB1889180433994209D126
:1007C0000123013C9C40AA181C4353606C60E4E781
:1007D0001220AEE758681860EFE7C046FFBD000082
:1007E00003BE0000002310B50C000B70C30705D535
:1007F0000D49421020000AF021FB08E00B490028B7
:1008000002D0042804D10A4920000AF037FB10BDA9
:100810000428FCD90F2302681340042BF7D102F0FF
:10082000BBFB04490200E5E75CC6000008BE00000F
:100830000EBE000013BE0000F0B593B0039003009D
:1008400002911C20012B1DDD029B01251B681C0051
:100850002C4000D0A8E0042B00D8A5E01A680F2394
:100860001A40092A48D10194019A029992008A58A3
:1008700016002E4005D1042A03D910681840092813
:1008800004D0222000F060FB07002CE052685210D8
:10089000A418019A013201920199039A8A42E3D184
:1008A000611C012202F00EFD071E01D100271AE093
:1008B00064002543456005000835029AB300D1580D
:1008C0004B680A685B1012099A4200D8531E002236
:1008D00093420BDCDA43D21713409B00ED18019BC7
:1008E00001369E42E9DB380013B0F0BD90000C18D1
:1008F000A46801322C50EBE7042A55D12F002600C2
:100900001D00029AB300D058384237D1042835D997
:1009100003682B40042BB4D1FFF732FC039B013654
:100920002418B342EDD1200002F038FD071EBDD0DF
:10093000039B029D9B00EB18041D029301232E686C
:100940001E4222D1042E20D90F2233681340042BDB
:100950000DD13000FFF714FC0190300002F01CFBB9
:10096000019A0100200009F009FF019BE418029B95
:100970000435AB42E2D100232370B4E705A9FFF7A9
:1009800031FF05A80AF092FAC8E705A93000FFF781
:1009900029FF05A80AF08AFA0600020005A920002E
:1009A00009F0ECFEA419E2E7212000F0CDFA7DE782
:1009B000F0B50D0095B0002806DC1C2000F0C4FA4C
:1009C0000400200015B0F0BD0C68012123000B408D
:1009D000009306D1042C04D922680F331A40092A47
:1009E00001D00B20EAE7626852100392002A03DC70
:1009F000009802F0D3FCE3E73F4A019201280BD0B4
:100A00006868084208D1042806D902681340042BFC
:100A100002D102F0C1FA019001980AF047FA0600EB
:100A20000F27039B0834013B04935E43039B029012
:100A30009B001B19059301232068184251D10428FB
:100A40004FD903683B40042B52D1FFF799FB059B1C
:100A500004343618A342EED1300002F09FFC041E8D
:100A6000AFD02B680593029B002B03D0686802F07F
:100A700093FA0190200002F08FFA0500009B059A7E
:100A80009B00D3189F68380002F086FA0123060005
:100A90001F4201D1042F04D807A93800FFF7A2FE96
:100AA00007AE30000AF002FA070002003100280009
:100AB00009F064FE029BED19002B0AD0049B009AFA
:100AC000934206DD2800029A019909F057FE029B25
:100AD000ED18009B01330093009A039B9342CDD104
:100AE0006FE707A9FFF77EFE07A80AF0DFF9AEE778
:100AF00002F052FAF9E7C04663C1000010B50024C5
:100B0000A04207DD0B6801341C4003D05C10E343B6
:100B1000DB171C40611C0122092002F0D3FB0028D6
:100B200003D0012364001C43446010BD0B6870B502
:100B300018000125284032D1042B30D90F241A681F
:100B400049681440092C16D15C6812092C41A24254
:100B500000D8541E844205DC02200132904206DB9C
:100B600000200FE085005D19A9600130F2E78400E4
:100B700019510130F2E7032C11D1294203D113207E
:100B800000F0E2F970BD4910FF29F8D812090433CA
:100B900092009A189A42E3D919700133FAE70B20B0
:100BA00000F0D2F9DCE700000123F7B500264D681C
:100BB0000F002B400093B3420DD11E00042D0AD923
:100BC0000F222B681A40092A0FD16A681B09561098
:100BD000B34200D85E1E3968CB0713D54C10002CE9
:100BE00001DDA64219DA12202EE0042A04D12800E1
:100BF000FFF7C6FA0600EEE7009E032AEBD11E09B6
:100C0000B600E8E72E48FFF777FD002814D00AF079
:100C1000B1F8310007F070FD4C1C009B002B4CD14B
:100C2000042D4AD92A680F331340092B10D10134FF
:100C3000A40064592000FEBD39682248FFF75CFD1E
:100C400034000028E9D1113000F07EF90400F1E70A
:100C5000042B2AD1280002F09FF90600FFF7BAFA08
:100C6000A042C0DB012C1ADC280002F095F90090AC
:100C70003000FFF79BFA851B280002F08FFB041E53
:100C8000D8D002F089F90190786802F085F9009BCC
:100C90002A00F11A4118019809F070FDCAE73000E6
:100CA000FFF784FA013C0600DCE7032B05D12C1981
:100CB000E478023B64001C43BCE70B20C4E7C04659
:100CC000F8BD000003BE0000F7B54C680F0001201E
:100CD000210001402AD1042C28D90F222368BE68A4
:100CE0001A40092A13D162681B0955100191AB42C1
:100CF00000D85D1E39682848FFF7FEFC002829D07F
:100D00000F2322681340092B19D1012313E0032A72
:100D10000CD1064203D1132000F016F9FEBD72106B
:100D20000192FF2AF7D81D09AD00E3E70B20F3E796
:100D300001339A00A6509D42FADA0020EEE7032B19
:100D4000FBD1230001331A1BAA42F6DC6A46127952
:100D5000DA70F7E73968CB0706D54910002901DDBD
:100D60008D4209DA1220D7E70C48FFF7C5FC2900AD
:100D7000002801D11130CFE70F2322681340092B3F
:100D800003D1013189000E51D7E7032BD5D16B4632
:100D90001B796418E370D0E7FFBD000003BE0000BC
:100DA00010B501240868204216D1042814D90F2256
:100DB00003681A40092A01D1406810BD032A03D1F3
:100DC0001809C0002043F8E7042A05D102F0E4F82E
:100DD000FFF700FA4000F5E70B2000F0B5F8ECE76C
:100DE00010B5034A0A21034803F036FF10BDC04680
:100DF000A8BD0000A0BD000002000120104001D0ED
:100E0000501070470D22014B1A70FAE7A40200201F
:100E1000F0B585B00393019002912C4E2C4B002A23
:100E200002D002223270013A00251A601B68F55484
:100E3000019B9D4201DB05B0F0BD029AAB00D0588A
:100E4000234B1C68C8239B0037191C1B0123184225
:100E500006D0204A43102100380009F0BDFF09E008
:100E60001D4A002802D004281BD11C4A210038004A
:100E700009F0B2FF30000AF019F8154A039B106020
:100E8000002B0CD0019B013BAB4208DD144B984278
:100E900005D8431C1360202232540022F25401353D
:100EA000C6E704280FD90F2302681340042B04D18E
:100EB00002F072F80B4A0300CDE7092B04D1436816
:100EC000094A5B10C7E70123084AC4E7A5020020CE
:100ED000C80500205CC6000008BE00000EBE000071
:100EE0001F0300007BCC000078C0000087C000001A
:100EF0000123020010B51A4015D1042801D9026857
:100F000012090B4011D1042901D90B681B090024D7
:100F1000934206D104309B000431C318984206D393
:100F20000124200010BD0022EBE70023EFE7047846
:100F30000A78002C01D1002AF2D00130013194420C
:100F4000ECD00024EDE70000014B18700020704742
:100F5000A402002070B501F093FD094C0100251D8D
:100F60001F22280009F0A9FF280009F09FFF042391
:100F700004308008000118432060200070BDC04686
:100F800080020020C368F0B59D00836889B05D19B8
:100F90000300183306930369069A9F00069B02908C
:100FA000DF19436901939B00D3180393CD4B1B7842
:100FB000002B26D17F222B68CB491C1213409B00AB
:100FC0005B58043501929F46029B587804F020FA42
:100FD0000023029A137027E0C24B1B78002B10D11C
:100FE0002B68019A1C121340BF4A9B009B58043582
:100FF000E9E7069B3A1DD11ABA4BD82928DD1A22F7
:101000001A70029BB74C9B6821780193EA1A029BE5
:1010100092109B7812021A43029B587804F000FA4F
:101020000023029A23701370029B069A9B68019317
:10103000ED1A029BAD10DD60069BFE1A029BB610F6
:101040001E61039B9B1A029A9B10536109B0F0BD6D
:101050001B783C60002B01D01700D2E72B68019968
:101060001C120B40A0499B005B5817000435AAE7EF
:10107000069B3A1DD11A9B4BD82902DD1A221A7001
:10108000BFE728681B78291D3860002B02D01700A5
:101090000D00B6E76B6801991C120B4092499B004A
:1010A0005B58170008358EE7069B3A1DD11A8D4B09
:1010B000D82902DD1A221A70A3E7A4001B782C1984
:1010C0003C60002B01D017009BE72B6801991C1294
:1010D0000B4085499B005B581700043573E7069B5E
:1010E0003A1DD11A7F4BD82902DD1A221A7088E7DF
:1010F0007E49A40061581B783960002B01D017008D
:101100007FE72B6801991C120B4077499B005B58C5
:101110001700043557E7043F744B3A68A400E250C7
:10112000704B1B78002B00D06BE72B68019A1C12C8
:1011300013406D4A9B009B58043544E76B4BA40059
:10114000E058FFF759FE043F06003868FFF754FEE9
:1011500036180120654B76000643E650614B1B783C
:10116000002B00D04DE72B68019A1C1213405E4AF9
:101170009B009B58043526E7069B3A1DD11A594B14
:10118000D82902DD1A221A703BE70698039C012138
:10119000A04202D221000C3909681B783960002B6B
:1011A00001D017002DE72B6801991C120B404E4906
:1011B0009B005B581700043505E7069B3A1DD11AC2
:1011C000484BD82902DD1A221A701AE706990398AB
:1011D00081420FD203000C3B1B6845495B10641829
:1011E000E41AA40023583B603E4B1B78002B05D02B
:1011F000170006E7182119700023F4E72B680199FE
:101200001C120B4038499B005B5817000435DAE686
:10121000069B039A934219D213000C3B1B68344A75
:10122000043FA4185B10E31A039A39689B00995095
:101230002C4B1B78002B00D0E3E62B68019A1C1284
:101240001340294A9B009B580435BCE61822254BC5
:101250001A70EDE7069B039A93422DD2244B3E1F52
:10126000E31814000C3C04932368049A5B10D31A0F
:10127000039A9B009858FFF7BFFD07903068FFF76F
:10128000BBFD2468049B64101C1B079BA4001F1853
:1012900001207F00039B0743E7503700114B1B7869
:1012A000002B00D0ADE62B68019A1C1213400E4AA9
:1012B0009B009B58043586E618220A4B1A70EDE70E
:1012C000069B3A1DD11A074BD82902DD1A221A7043
:1012D00097E60399A40061581B783960002B09D068
:1012E00017008EE6A402002078BE0000802D0020AA
:1012F000FDFFFF3F2B6801991C120B40D7499B0053
:101300005B58170004355EE6043F039B3A68A4006F
:10131000E250D34B1B78002B00D072E62B68019A69
:101320001C121340CD4A9B009B5804354BE6039B8F
:10133000A4001C192368043F38685E10FFF75CFDA9
:1013400036180120C64B76001B7806432660002B1A
:1013500000D056E62B68019A1C121340BF4A9B002E
:101360009B5804352FE6069BA4003F1BBC4CBB4298
:101370000CD82378002B00D043E62B68019A1C126E
:101380001340B64A9B009B5804351CE6B54801F053
:10139000F3FD2378002B00D033E62B68019A1C1252
:1013A0001340AE4A9B009B5804350CE6A300ED1891
:1013B000002C00DA38E6AA4B1B78002B00D020E680
:1013C0002B68019A1C121340A44A9B009B580435B9
:1013D000F9E5043F3B68042B04D1A300ED18002C71
:1013E00000DA21E69E4B1B78002B00D009E62B6823
:1013F000019A1C121340994A9B009B580435E2E560
:10140000043F3B68042B06D0A200AD18002C02DA82
:10141000002B00D108E6924B1B78002B00D0F0E5A2
:101420002B68019A1C1213408C4A9B009B58043570
:10143000C9E53A1F13685B10013B002B06DD012153
:101440005B00A4000B432D191360EDE5844B1700DE
:101450001B78002B00D0D4E52B68019A1C12134096
:101460007E4A9B009B580435ADE53A00069B0C3242
:10147000D31AD82B03DD1A22794B1A70C1E5FF234A
:1014800061005B001940FE3BFF3B19433960029944
:1014900006988968241204916D1A0299AD10897812
:1014A0002D020D4303999D40091A891099401D434F
:1014B0000B43BB60029B7D609C70E4B26A4BE4000E
:1014C0000392E358029A9360654A1278002A03D087
:1014D00008331D00039F94E51D00019A9B680C359D
:1014E0001C1213405D4A9B009B58039F6BE53B1FFA
:1014F0001C68039A069B93422DD10A20E3070CD463
:10150000042C13D90F2322681340042B11D120007F
:1015100001F042FD09F0CAFC0630643003F02CFCF7
:1015200000280FD1043D069B03937DE50720042C82
:10153000F3D02000431E9841FA234042FF33184065
:101540000730EAE7029B2100587803F07BFF002375
:10155000029A1370E7E7039B039A0C3B1B680299FE
:101560005B109B00D31A0C3B1C601F1D1300083B33
:101570001B685A108A70D2B23B49D2005B005558A2
:101580009B0A029A9B009560ED18039B069A043B08
:101590001B685B109B00D3180393314B1B78002B07
:1015A00000D02EE52B68019A1C1213402B4A9B0099
:1015B0009B58043507E53B1F1868FFF71DFCA40086
:1015C00006003F1B1E2827DC00280DDC244B1B785F
:1015D000002B00D015E52B68019A1C1213401F4AFE
:1015E0009B009B580435EEE401F038FA033E3618B0
:1015F00001F034FA1D4B801B9842F9D8184B1B7828
:10160000002B00D0FDE42B68019A1C121340134AF2
:101610009B009B580435D6E40123029A137001F015
:101620001DFA029B0A3886195E60FDE43B1F1868AC
:10163000FFF7E2FBA40006003F1B002818DC084B64
:101640001B78002B00D0DCE42B68019A1C1213409D
:10165000024A9B009B580435B5E4C04678BE0000A2
:10166000A402002099C00000882500203F420F00FE
:10167000CA4B984203DD1D22C94B1A70C1E40123F5
:10168000029A137001F0EAF9FA239B005E43029B71
:101690000A3E30185860C7E4A300FF1A0023200058
:1016A0001A003900FFF7B4FBBE4EBF4C3168200072
:1016B00001F080FEBD4B31681860200003F076FD1C
:1016C0003168200003F0C5FE3168200001F00EFFF4
:1016D000B34B1B78002B00D093E42B68019A1C12AB
:1016E0001340B34A9B009B5804356CE4AC4BA400F8
:1016F0001B783F1B002B00D083E42B68019A1C123F
:101700001340AB4A9B009B5804355CE4029803F0FD
:1017100097FBA34B1B78002B00D072E42B68019A37
:101720001C121340A24A9B009B5804354BE43B1FFC
:101730001B68002B3ED13B000C3B1B68DA072CD505
:10174000390001225B105800083902430A60002B5F
:1017500044DD012259001143381F01603900083966
:1017600009681141CB1A39000C390968114224D09B
:101770009B189340A4001343039AA350884B1B78F3
:10178000002B00D03DE42B68019A1C121340884ABC
:101790009B009B580435FFF716FC042B06D90F223B
:1017A00019680A40092A01D15B68C9E719227C4BF4
:1017B0001A7026E45B10013BC9E7042909D90F22FE
:1017C00008680240092A04D102339B005B58A40038
:1017D000D2E71922724B1A70FFF713FC0435CDE7DC
:1017E000A300069AFB189B1AD82B13DC0122631E58
:1017F000002C14DC6A4B1B78002B01D0FFF701FC96
:101800002B68019A1C121340694A9B009B580435AF
:10181000FFF7D9FB1A22624B1A70FFF7F2FB3A600E
:101820001C000437E3E7069A3B1D9B1A5C4ED82B3D
:1018300003DD1A233370FFF7E4FB069B039AA40031
:1018400093422AD23B1F1868FFF7D6FA011E21DD0A
:10185000039B0C3B1A68521082421BDB9007801AD4
:10186000544B4018C018039B8000C2583B1B1A60A1
:101870004B4B3F1B1B780437002B01D0FFF7C1FBFC
:101880002B68019A1C121340494A9B009B5804354F
:10189000FFF799FB20233370EAE71823FBE7434B5C
:1018A000A4001A683B1B1F001A603D4B04371B78CD
:1018B000002B01D0FFF7A5FB2B68019A1C121340E7
:1018C0003B4A9B009B580435FFF77DFBA3009C46D9
:1018D000FE1A002C17DC1C22314B1A7000233360D7
:1018E0006346FF1A2E4B04371B78002B01D0FFF7FD
:1018F00088FB2B68019A1C1213402D4A9B009B58B1
:101900000435FFF760FB002033685A108300F1585C
:1019100001230B4003D10D21214A1170DFE749104B
:101920008A4200DD0A0001308442EFDC01235200CC
:101930001343D4E7A3009C46FE1A002C17DC1C229C
:10194000174B1A70002333606346FF1A144B043799
:101950001B78002B01D0FFF754FB2B68019A1C1257
:101960001340134A9B009B580435FFF72CFB0020C3
:1019700033685A108300F15801230B4003D10D2125
:10198000074A1170DFE749108A4200DA0A00013085
:101990008442EFDC012352001343D4E780EE36008B
:1019A000A4020020C8050020A50200200800002095
:1019B00078BE0000FCFFFF3F3B00083B1868FFF7C4
:1019C0001BFA3B1F06001868FFF716FA0023864231
:1019D00000DA0433A4003A1B17001360E34B04370A
:1019E0001B78002B01D0FFF70CFB2B68019A1C120F
:1019F0001340DF4A9B009B580435FFF7E4FA3B0095
:101A0000083B1868FFF7F8F93B1F06001868FFF756
:101A1000F3F9F30FC217B0425341A4003A1B170069
:101A20009B001360D14B04371B78002B01D0FFF7CC
:101A3000E8FA2B68019A1C121340CD4A9B009B5870
:101A40000435FFF7C0FA3B00083B18683B1F1968D4
:101A5000A600BE1B0423814202D0042802D8002322
:101A6000336016E001231842F9D10F2302681A40AF
:101A7000042AF4D1033A1142F1D10429EFD90A68BA
:101A80001340042BEBD1FFF733FA431E984180003B
:101A90003060B64BA4001B783F1B0437002B01D0ED
:101AA000FFF7AFFA2B68019A1C121340B04A9B0053
:101AB0009B580435FFF787FA3B00083B18683B1F2B
:101AC0001968A600BE1B0023814202D0042802D858
:101AD0000423336016E001231842F9D10F23026872
:101AE0001A40042AF4D1033A1142F1D10429EFD962
:101AF0000A681340042BEBD1FFF7FAF9434258412F
:101B000080003060994BA4001B783F1B0437002BEA
:101B100001D0FFF776FA2B68019A1C121340944A01
:101B20009B009B580435FFF74EFA3B00083B1868B2
:101B3000FFF762F93B1F06001868FFF75DF9F3171E
:101B4000C20F86425341A4003A1B17009B0013604A
:101B5000864B04371B78002B01D0FFF752FA2B6815
:101B6000019A1C121340824A9B009B580435FFF7D0
:101B70002AFA3B00083B1868FFF73EF93B1F0600B6
:101B80001868FFF739F90023864200DD0433A4000A
:101B90003A1B17001360754B04371B78002B01D0DC
:101BA000FFF72FFA2B68019A1C121340704A9B0012
:101BB0009B580435FFF707FA3B1F1B68A400043B42
:101BC0005A1E93413A1B17009B001360674B043762
:101BD0001B78002B01D0FFF714FA2B68019A1C1216
:101BE0001340634A9B009B580435FFF7ECF93B0018
:101BF000083B1868FFF700F93B1F06001868FFF75D
:101C0000FBF832180120A4003B1B1F0052000243C6
:101C10001A60564B04371B78002B01D0FFF7F1F9FF
:101C20002B68019A1C121340514A9B009B580435A3
:101C3000FFF7C9F93B00083B1868FFF7DDF83B1FC9
:101C400006001868FFF7D8F8321A0120A4003B1BE1
:101C50001F00520002431A60444B04371B78002BCC
:101C600001D0FFF7CEF92B68019A1C121340404AAD
:101C70009B009B580435FFF7A6F93B00083B18680A
:101C8000FFF7BAF83B1F06001868FFF7B5F8020027
:101C90000120A4003B1B1F007243520002431A6044
:101CA000324B04371B78002B01D0FFF7AAF92B68C1
:101CB000019A1C1213402E4A9B009B580435FFF7D3
:101CC00082F93B1F1868FFF797F8061E17D11F22ED
:101CD000264B1A70A4003B1B1F001E60234B0437C9
:101CE0001B78002B01D0FFF78CF92B68019A1C128E
:101CF00013401F4A9B009B580435FFF764F93B00D3
:101D0000083B1868FFF778F8310006F00FFC012651
:101D100040000643DEE73B1F1868FFF76DF8061E1C
:101D200017D11F22114B1A70A4003B1B1F001E600D
:101D30000E4B04371B78002B01D0FFF762F92B689C
:101D4000019A1C1213400A4A9B009B580435FFF766
:101D50003AF93B00083B1868FFF74EF8310006F0EF
:101D6000CBFC012649000E43DEE7C046A40200205A
:101D700078BE00003B1F1868FFF73EF8C2178018B6
:101D800050400122A4003B1B1F004000104318607C
:101D9000F64B04371B78002B01D0FFF732F92B6884
:101DA000019A1C121340F24A9B009B580435FFF71E
:101DB0000AF9A300FE1A3068012C24D1FFF71CF8A1
:101DC0000494079008F0D6FF0799002900DC012150
:101DD00006F092FC049BA400C91801234900194392
:101DE000E24B3F1B1B7831600437002B01D0FFF71B
:101DF00008F92B68019A1C121340DD4A9B009B587E
:101E00000435FFF7E0F8FEF7F7FF04907068FEF77F
:101E1000F3FF049B0130C31A0793D3E7A300FE1A14
:101E200031002000049301F001FB049B3060FF1A95
:101E3000CE4B04371B78002B01D0FFF7E2F82B685C
:101E4000019A1C121340CA4A9B009B580435FFF7A5
:101E5000BAF83B00083B1868FEF7CEFF3B1F0600B0
:101E60001868FEF7C9FF02000120A4003B1B1F00F9
:101E70003240520002431A60BC4B04371B78002BDF
:101E800001D0FFF7BEF82B68019A1C121340B84A24
:101E90009B009B580435FFF796F83B00083B1868F9
:101EA000FEF7AAFF06003B1F1868FEF7A5FF3200E9
:101EB00002430120A4003B1B1F00520002431A6092
:101EC000AA4B04371B78002B01D0FFF79AF82B6838
:101ED000019A1C121340A64A9B009B580435FFF739
:101EE00072F83B00083B1868FEF786FF06003B1FB0
:101EF0001868FEF781FF320042400120A4003B1B1E
:101F00001F00520002431A60984B04371B78002BC5
:101F100001D0FFF776F82B68019A1C121340944AFF
:101F20009B009B580435FFF74EF83B1F1868FEF7DF
:101F300063FFC0430122A4003B1B1F00400010436D
:101F400018608A4B04371B78002B01D0FFF759F833
:101F50002B68019A1C121340854A9B009B5804353C
:101F6000FFF731F83B00083B1868FEF745FF060015
:101F70003B1F1868FEF740FF3200824051000122EB
:101F8000A4003B1B1F000A431A60784B04371B78E0
:101F9000002B01D0FFF735F82B68019A1C12134073
:101FA000734A9B009B580435FFF70DF83B00083B34
:101FB0001868FEF721FF06003B1F1868FEF71CFF9C
:101FC0003200024151000122A4003B1B1F000A43C2
:101FD0001A60664B04371B78002B01D0FFF711F80D
:101FE0002B68019A1C121340614A9B009B580435D0
:101FF000FEF7E9FF3B000C3B1868FEF7FDFE3B00D7
:10200000083B06001868FEF7F7FEF1170200C31739
:10201000300006F0C3FB3B1F049005911868FEF7E3
:10202000EBFE02000498059906F06CFB43000120CA
:10203000A4003E1B370018434C4B30601B7804371C
:10204000002B01D0FEF7DDFF2B68019A1C12134014
:10205000474A9B009B580435FEF7B5FFA300FE1AC4
:10206000310020000493FEF749FD049B3060FF1A05
:102070003E4B04371B78002B01D0FEF7C2FF2B68C4
:10208000019A1C1213403A4A9B009B580435FEF7F4
:102090009AFFA300FF1A39002000FEF747FD334BDB
:1020A0001B78002B01D0FEF7ACFF2B68019A1C12A5
:1020B00013402F4A9B009B580435FEF784FFA30072
:1020C000FE1A310020000493FEF76EFD049B306081
:1020D000FF1A264B04371B78002B01D0FEF791FF27
:1020E0002B68019A1C121340214A9B009B5804350F
:1020F000FEF769FFA300FF1A39002000FEF7E4FD98
:102100001A4B1B78002B01D0FEF77BFF2B68019A3E
:102110001C121340164A9B009B580435FEF753FFD0
:10212000A300FE1A310020000493FEF739FE049B41
:102130003060FF1A0D4B04371B78002B01D0FEF7DF
:1021400060FF2B68019A1C121340094A9B009B58A0
:102150000435FEF738FF069B3E1DF31A034CD82BBF
:1021600008DD1A232370FEF74CFFC046A4020020AE
:1021700078BE000000F07CFC430001201843237867
:102180003860002B02D03700FEF73BFF2B68019A26
:102190001C121340F44A9B009B5837000435FEF78D
:1021A00012FF069B3E1DF31AF04CD82B03DD1A23B9
:1021B0002370FEF726FF00F051FCED4B4000184065
:1021C0000123184323783860002B02D03700FEF734
:1021D00018FF2B68019A1C121340E34A9B009B587E
:1021E00037000435FEF7EFFE0123A600BE1B2000DA
:1021F0001A003100FEF70CFEDE4C2068643002F05D
:10220000BBFD002802D1043DFEF70EFF029B2168B2
:102210005A78D94803F02BF90123029A370013703A
:1022200000F01CFCD54B22681B680632534318187B
:10223000029B5860FEF7F8FEA600BE1B200001239B
:1022400000223100FEF7E4FDCA4C2068643002F041
:1022500093FD0028D7D0C84802F000FFDCE7A400B7
:102260003E1BFEF777FE3700C04B30601B7804370B
:10227000002B01D0FEF7C5FE2B68019A1C121340FB
:10228000B94A9B009B580435FEF79DFEA4003E1BF7
:10229000300000F01CFC3700B44B30601B78043772
:1022A000002B01D0FEF7ADFE2B68019A1C121340E3
:1022B000AD4A9B009B580435FEF785FEA4003E1BEB
:1022C000300000F006FC3700A84B30601B78043764
:1022D000002B01D0FEF795FE2B68019A1C121340CB
:1022E000A14A9B009B580435FEF76DFEA300FE1A21
:1022F00031002000049300F0EFFB049B3060FF1AD4
:102300009A4B04371B78002B01D0FEF77AFE2B681E
:10231000019A1C121340944A9B009B580435FEF707
:1023200052FEA4003F1B380000F008FC8F4B1B78C6
:10233000002B01D0FEF765FE2B68019A1C1213409A
:10234000894A9B009B580435FEF73DFEA300FE1A08
:1023500031002000049300F019FC049B3060FF1A48
:10236000824B04371B78002B01D0FEF74AFE2B6806
:10237000019A1C1213407C4A9B009B580435FEF7BF
:1023800022FEA4003F1B380000F042FC774B1B7874
:10239000002B01D0FEF735FE2B68019A1C1213406A
:1023A000714A9B009B580435FEF70DFE0121200069
:1023B00000F016FC6D4B1B78002B01D0FEF721FEC0
:1023C0002B68019A1C121340674A9B009B580435E6
:1023D000FEF7F9FD0021200000F002FC634B1B78A2
:1023E000002B01D0FEF70DFE2B68019A1C12134042
:1023F0005D4A9B009B580435FEF7E5FDA4003E1B9B
:10240000300000F027FC3700584B30601B78043751
:10241000002B01D0FEF7F5FD2B68019A1C1213402A
:10242000514A9B009B580435FEF7CDFDA4003E1B8E
:10243000300000F023FC37004C4B30601B78043731
:10244000002B01D0FEF7DDFD2B68019A1C12134012
:10245000454A9B009B580435FEF7B5FDA4003F1B81
:10246000380000F0E5FB414B1B78002B01D0FEF754
:10247000C8FD2B68019A1C1213403B4A9B009B58D5
:102480000435FEF7A0FDA4003F1B380003F00AFB53
:10249000364B1B78002B01D0FEF7B3FD2B68019A59
:1024A0001C121340304A9B009B580435FEF78BFDED
:1024B000A4003E1B300003F08DFB37002B4B306037
:1024C0001B780437002B01D0FEF79BFD2B68019A87
:1024D0001C121340244A9B009B580435FEF773FDE1
:1024E000A4003F1B380003F08DFA204B1B78002B13
:1024F00001D0FEF786FD2B68019A1C1213401A4A80
:102500009B009B580435FEF75EFDA4003E1B300087
:1025100003F08EFA3700154B30601B780437002B20
:1025200001D0FEF76EFD2B68019A1C1213400E4A73
:102530009B009B580435FEF746FDA300FF1A3900A7
:10254000200001F075FA094B1B78002B01D0FEF733
:1025500058FD2B68019A1C121340034A9B009B589C
:102560000435FEF730FDC04678BE0000A40200200E
:10257000FEFFFF7FC8050020A50200200400002008
:10258000A300FF1A3900200001F0DAF89F4B1B78F6
:10259000002B01D0FEF735FD2B68019A1C12134069
:1025A0009B4A9B009B580435FEF70DFDA300FF1AC4
:1025B0003900200001F0D4F8944B1B78002B01D097
:1025C000FEF71FFD2B68019A1C121340904A9B00D6
:1025D0009B580435FEF7F7FCA300FF1A39002000D2
:1025E00001F0E6F8894B1B78002B01D0FEF709FDBE
:1025F0002B68019A1C121340854A9B009B58043596
:10260000FEF7E1FCA300FE1A31002000049303F062
:1026100086FB049B3060FF1A7C4B04371B78002B31
:1026200001D0FEF7EEFC2B68019A1C121340784A89
:102630009B009B580435FEF7C6FCA300FE1A310030
:102640002000049303F073FB049B3060FF1A6F4B70
:1026500004371B78002B01D0FEF7D3FC2B68019ABE
:102660001C1213406A4A9B009B580435FEF7ABFCD2
:10267000A300FE1A31002000049303F060FB049BCA
:102680003060FF1A614B04371B78002B01D0FEF736
:10269000B8FC2B68019A1C1213405D4A9B009B58A2
:1026A0000435FEF790FCA300FE1A310020000493CD
:1026B00003F060F9049B3060FF1A544B04371B7819
:1026C000002B01D0FEF79DFC2B68019A1C121340D1
:1026D0004F4A9B009B580435FEF775FCA300FF1A78
:1026E0003900200001F02CF9484B1B78002B01D059
:1026F000FEF787FC2B68019A1C121340444A9B008A
:102700009B580435FEF75FFCA300FF1A3900200038
:1027100001F076F83D4B1B78002B01D0FEF771FCE1
:102720002B68019A1C121340394A9B009B580435B0
:10273000FEF749FCA300FE1A31002000049300F0CC
:10274000CDFF049B3060FF1A304B04371B78002B01
:1027500001D0FEF756FC2B68019A1C1213402C4A3C
:102760009B009B580435FEF72EFCA300FF1A39008E
:10277000200001F043F9254B1B78002B01D0FEF718
:1027800040FC2B68019A1C121340214A9B009B5865
:102790000435FEF718FC069B029AFB1A9B10136186
:1027A000A300FF1A3900200002F06AFA174B1B78C9
:1027B000002B01D0FEF725FC2B68019A1C12134058
:1027C000134A9B009B580435FEF7FDFB069B029ABB
:1027D000FB1A9B101361A300FE1A31002000049322
:1027E00002F04EFA049B3060FF1A084B04371B7846
:1027F000002B01D0FEF705FC2B68019A1C12134038
:10280000034A9B009B580435FEF7DDFBA402002021
:1028100078BE00000023F7B55A1E0192002B07DA9C
:1028200001F01CF902F020FD02F080FE1923019353
:1028300000263000194B1968B14212DD184B1A6896
:1028400001328A420FDAF0241A601D68154F6C437A
:10285000E35D002B1FD0E419022B06D12000FEF708
:1028600091FB019BD8E70022EDE7012B0DD1002859
:1028700001D100F0F3F8F0226A43BB185B680A4903
:10288000C31A8B4201D80223BB54F0235D43054B8E
:10289000EB5C022BE2D00136CCE7C046CC05002031
:1028A00000000020281C00203F420F0001220021D0
:1028B0000A4B0B481A61195004301950A221042008
:1028C000C9005850C121C0208900800258501A60A8
:1028D000044BFC311960044B1A70704700A0004093
:1028E0000405000000E100E0F3050020042070472B
:1028F000F8B550C9012322001A40101E2DD03340D4
:10290000181E2AD0641000201C2C26D81D4B7610CF
:1029100035009E4200DD1D001B4F3B5D012B05D0A5
:102920000121200004F01EF901233B55174B1B78B1
:10293000002B01D1FFF7BAFF0023154A9E420DDCA0
:10294000FF2514491448D65CB44202D15E0070528F
:10295000D5540133042BF6D10420F8BDD15C8C4250
:1029600003D10C4A5B009D52F6E70133042BF5D1ED
:102970000023D15CFF2901D1D454F2E70133042BA9
:10298000F7D1E9E788130000D4050020F305002003
:102990001C0000200E000020DC050000F8B530C946
:1029A000012623003340181E1BD02B003340181E75
:1029B00017D0344100201C2C13D8174F3B5DB34275
:1029C00004D03100200004F0CDF83E556910080015
:1029D000124A1038124B904204D9012252421A6016
:1029E0000420F8BD1C600F4805F0A0FD0E4B1880B8
:1029F0000E4B1B78002B02D1FFF758FFF0E70122A6
:102A00000B4B9A64A922D2009A588018A82280B24F
:102A1000D2009850E4E7C046D4050020908601001B
:102A20001800002020A107000C000020F305002062
:102A300000A000400420704701220020054B0649F9
:102A40001A615850043103305850083180185850DA
:102A50001A60704700800040040500000122034B0B
:102A60001A64A822D20098587047C04600800040DF
:102A700010B5FFF7F3FFFA21890005F0CDFC10BD7A
:102A800000487047ECC000001D20704770B5054E2F
:102A90000400335C0D008B4202D004F063F835551E
:102AA00070BDC046D405002070B50024064D635D9E
:102AB000012B05D10021200004F054F800236355B8
:102AC00001341D2CF2D170BDD405002070470D20BB
:102AD00070473B2070470000F8B501240B680600E2
:102AE0000D00234204D10D20FEF72EFA2000F8BD80
:102AF0005B102000052BFAD80E4A9B009C580E4F05
:102B00003B5D002B05D00021200004F02BF80023B2
:102B10003B55012E06DD6B68042B03D102212000FA
:102B200004F020F8200003F0CBFE012440002043F5
:102B3000DDE7C046D4C00000D4050020F8B501266A
:102B40000568354202D04468344203D10D20FEF7B7
:102B5000FBF9F8BD6D101C2DFBD80A4F7B5D012BD6
:102B600004D03100280003F0FDFF7E5506496410B3
:102B70008C4202DCE143C9172140280003F026FF04
:102B8000E7E7C046D4050020FF03000070B501242C
:102B90000D68254204D10D20FEF7D6F9200070BD46
:102BA0006D101C2D17D80024012804DD4C68043C4E
:102BB00063425C416400094E735DA34204D021006E
:102BC000280003F0CFFF7455280003F0FFFF030037
:102BD0000420012BE3D00020E1E7C046D40500200B
:102BE00070B504000D001C280ED8084E335C012B74
:102BF00004D0012103F0B6FF012333552900200042
:102C00004D1EA94103F0CCFF70BDC046D405002085
:102C1000036810B5DA0703D40D20FEF795F910BD4F
:102C20004168581004394A425141FFF7D9FFF6E78D
:102C300037B569460A00064B30CB30C20368022024
:102C4000042B02D100F08CFD37BD00F0B1FDFBE795
:102C5000ACC0000010B5084C6379002B05D00021F2
:102C6000052003F07FFF00236371052003F0AEFF12
:102C700043425841800010BDD405002010B5084CD7
:102C8000E37A002B05D000210B2003F06BFF00231B
:102C9000E3720B2003F09AFF43425841800010BDBD
:102CA000D4050020F7B5304D304E6B6C002B15D09D
:102CB000A8240023E40037596B642D4B18680028C2
:102CC0000CDB2C4B19784A425141C9B2197003F000
:102CD00067FF294B1B88DF19BFB23751AB6C002B44
:102CE00039D00021254B264FF458A9643A780C348A
:102CF0000193244D8A4206D02B68032B03D8224A25
:102D0000D05C03F04DFF2B68204A0133134004D5FB
:102D10000422013B5242134301331B4900228C46DB
:102D20002B60042B18D06046C05C591CFF2802D1D0
:102D30000B000122F5E7002A00D02B60012103F0EF
:102D40002FFF01233B702B68114A5B009B5AE4184C
:102D5000019BA4B2F450F7BD01235B422B6000231A
:102D60003B700C4BF3E7C046FCA0004000A00040C5
:102D700018000020F20500200C000020440500008F
:102D8000F1050020D00500201C0000200300008079
:102D90000E00002050460000084B094AFF201A8010
:102DA0005A809A80DA800023064A07491370074A3E
:102DB000087048708870C870136070470E0000205B
:102DC000DC050000F10500201C000020D0050020DB
:102DD0000122024B52421A607047C0461800002080
:102DE00010B5034A0421034801F036FF10BDC04668
:102DF000B4C000009CC70000E12170B5490214482E
:102E000003F056FBFFF718FE0A2003F053FD0023E2
:102E1000FF21104A995401331D2BFBD101220020C0
:102E20000D4B01001A6004230C4A0D4D1468002C50
:102E3000FCD02C680002013B20431160002BF5D12F
:102E40000122084B1A6003F0EFFC00F053FF70BD45
:102E5000B01B0020D405002000D0004000D100406D
:102E600008D5004004D00040F8B50B4E07003000F4
:102E70000D0003F065FB0400A84200DD2C003D00BE
:102E8000EB1B9C4205DD300003F064FB287001352C
:102E9000F6E72000F8BDC046B01B002010B50100C9
:102EA000014803F00DFB10BDB01B002010B5054C10
:102EB000200003F013FBE1212000490203F0F8FA9F
:102EC00010BDC046B01B0020C3070CD4064B1B68C6
:102ED000834208D8054B1B68984204D8031F1B681F
:102EE000002B00D018007047FC050020F8050020DA
:102EF0000023012210B50A48990001334250642B87
:102F0000FAD1084C084B00211A602000074A07F04C
:102F100051FC074B074A6360074B1A6010BDC0465F
:102F2000802D00200006002008000020D4090000A9
:102F30003027000004060020F405002010B5044BE3
:102F4000044A1A60044B054A1A60FFF7D1FF10BD0E
:102F5000FC05002000060020F8050020D40F00200A
:102F6000044B1B68186800090238C343DB1718407C
:102F70007047C046F405002000B59BB0020005492B
:102F800001A807F05BFF01A802F084F802F0CEFA76
:102F9000FCE7C04653C100000A4BC20704D4042812
:102FA00004D8094B00D0094B180070470F22036862
:102FB0001A40031D042AF7D0054B092AF4D0054B0B
:102FC000F2E7C04639C100000EBE000008BE000096
:102FD0004CC1000043C100000020064A0649131FEF
:102FE000186013681B0902339B00D2188A42F6D37B
:102FF0007047C04604060020D40F0020F7B50F2408
:103000000126304B304A1968304B314D186813682F
:103010001F002740072F25D813681B0902339B0088
:10302000D218AA42F3D300242A4EA500AD1928686D
:10303000FFF74AFF01342860642CF6D1264C206843
:10304000FFF742FF2060254C2068002802D0FFF7E0
:103050003BFF20600025224B1B680093009B9D4294
:1030600013DBF7BD1B099B00D3189A42D4D01F680D
:10307000374208D1B94206D2B84204D3043F3F6870
:10308000002F00D01F60043BEFE7F0236B43154A8D
:103090009B181A78002A01D10135DFE71F693C230C
:1030A00000266B43DB199B0001930136BB1BF3D455
:1030B000019BB4001C1B0B4B1C19A069FFF704FFFC
:1030C000A061F2E7FC05002004060020F8050020BE
:1030D000D40F0020802D002008000020D40F0020F5
:1030E000CC050020281C0020F7B50124204244D143
:1030F000224B1B689C4698423FD3214B1B6801938F
:1031000098423AD8031F1B68002B36D1020003688F
:1031100000941B09002B0FD10099131F19609042D6
:103120002BD015682B1F1B68990069180C68013B90
:1031300014600A602A00EDE79D0055192968009C7B
:10314000214218D18C4516D8019C8C4213D30E1FF6
:103150003468002C0FD10F680F343C40072C07D97E
:103160002F60151F2B600B680A601B090A00D1E74E
:1031700000993160CEE7013BCCE7F7BDFC050020AC
:10318000F80500200D49F0B50B000F260C4D18680E
:103190001C1F276802090232002F0BD000208B422F
:1031A00000D0080020609000091892009B18AB42E4
:1031B000EDD3F0BDB0431860F7E7C0460406002029
:1031C000D40F0020F8B5114C26000F2233681F09D8
:1031D00013420DD07D1CAD00A64204D02A00310060
:1031E000200007F0D4FA00226319043564191A602C
:1031F0000237BF00064BF6199E42E6D31B1B9B10FD
:10320000013B1B012360034B1C60F8BD040600203A
:10321000D40F0020F4050020F0B59BB0FFF71EFC92
:1032200000240700204AA300D0580134FFF75CFFB8
:10323000642CF7D11D4B1868FFF756FF1C4B18681C
:10324000002801D0FFF750FF00261A4B1B689E4252
:1032500016DBFFF797FFFFF7D1FEFFF7B3FFFFF78E
:10326000FDFB154BC21B1B6814491B6801A81B09F9
:10327000023B07F0E3FD01A801F00CFF1BB0F0BD1D
:10328000F02575430E4BED182B78002B01D101363C
:10329000DBE72B695C1E002CF9DBA300EB189869B7
:1032A000FFF722FF013CF6E7802D002008000020F8
:1032B000D40F0020CC050020F405002019C1000027
:1032C000281C0020F7B5164D4F1C2B6806001B6804
:1032D0000C0001921B099F420ADBFFF79DFF2B6840
:1032E0001B681B099F4203DB0A20FDF72DFEFEBD74
:1032F0002868A71CBA00DB1B81181B010B60296022
:103300000021031F19600F231E40030024012643E0
:1033100040C3083A9A189A42E9D9019902C3FAE7D8
:10332000F4050020F7B503000122134004000D004E
:103330000193002B2AD1164B1B68834226D8154BCC
:103340001B68834222D90F23134F3860006818404E
:10335000FFF7B8FF019B3C68061E3B6016D0236850
:1033600004301B099D4200DD1D00AA00211D251F00
:1033700007F004FAFFF730FE2E60FFF73FFE002350
:103380002B6022680F339A43226034002000FEBD78
:10339000FC050020F8050020D40F00200323043092
:1033A00010B5C11719400918891000220420FFF731
:1033B00089FF10BD70B5050008000C00FFF7EEFF97
:1033C0000023002804D170BDE95CC21811710133DB
:1033D000A342F9DBE343DB171C40002304192371EC
:1033E000F1E7000010B501240B681C4016D05C10FA
:1033F000200005F02FFB0B4905F0FAF907F0E0F883
:1034000003F028FD0022084B06F094FA03F0CAFCF2
:1034100007F066F843000120184310BD0D20FDF7AA
:1034200093FDE5E7D30237390000D040086870B556
:1034300001240500254006D1042804D90F23026881
:103440001340042B03D00E20FDF77EFD70BDFFF767
:10345000A3FD03782900233B5A4253411022C01890
:1034600007F0DAFD80239B05C218044B9A4201D96C
:103470001420E9E740002043E8E7C046FFFFFF3F94
:1034800010B5034A0221034801F0E6FB10BDC04617
:103490006CC1000064C100000020704710B51E2000
:1034A000FDF752FD10BD10B51E20FDF74DFD10BDFE
:1034B00010B51E20FDF748FD10BD10B51E20FDF70C
:1034C00043FD10BD10B51E20FDF73EFD10BD10B52B
:1034D0001E20FDF739FD10BD10B51E20FDF734FD8F
:1034E00010BD10B51E20FDF72FFD10BD7047000068
:1034F00010B5034A0921034801F0AEFB10BDC046D8
:103500008CC10000D4C100000120034B1860034BA4
:103510001B68834018437047F80F0020D80F002025
:10352000F0B5EFF310810123194083F31088134C99
:10353000134AA4461268134E013A9340124F134A9D
:10354000002B17D0146803420FD03D682C60C04692
:10355000C046C046C046C046C046C046C0460C4CE9
:103560001568246825605B08EAE765462C601468E6
:103570003460F8E781F31088F0BDC04608050050BC
:10358000200000200C050050E40F0020EC0F00206C
:10359000E00F002030B585B001AD0C2206492800AF
:1035A00007F0ECF80024285D01210134FFF76EFAE2
:1035B0000C2CF8D105B030BD60C20000F7B56A46EA
:1035C000394B01AD13801C239370384B2B800A2399
:1035D000AB70FFF743FA364B364CC018236898425D
:1035E00001D2002323602668002E3DD16B469F5DEB
:1035F00001213800FFF74AFA01360021380003F0B4
:10360000CFFA032EF2D10026AF5D01213800FFF77B
:103610003DFA01360121380003F0C2FA032EF3D13E
:10362000C8200138C046C046C046C046C046C04655
:10363000C046C046C046C046C046C046F1D1002183
:103640002878FFF723FA68780021FFF71FFAA87897
:103650000021FFF71BFAFFF701FAFA2300251B01EF
:10366000C01820602800FEBDFFF7F8F92368002588
:103670009842F7D3032003F023F90600042003F057
:103680001FF936180A2003F01BF90B4B9B1B181A65
:103690000A4BA84206DB18600023094A2360136026
:1036A0000125DFE71D60F7E71A1B00000304000097
:1036B00010270000F00F0020E3030000D80F0020C7
:1036C000F80F002010B50124044002D0441020005F
:1036D00010BD0D20FDF738FCF9E700000868F8B5CB
:1036E000C3071AD5FFF7EEFF0300203B5E2B23D85C
:1036F0000520012258430023104E451DA84217D033
:1037000005211024375C3C4200D09B18013952003F
:1037100064100029F7D10130F0E704280CD90F22FA
:1037200003681A40042A07D11B0905D00079DBE79A
:1037300001205B001843F8BD0120FCE76CC20000CB
:103740000022054B10B51A60044B1B68934201D050
:1037500002F05EFB002010BDF40F0020D41A002000
:1037600070B508680D00FFF7ADFF04006868FFF74B
:10377000A9FF621E0100042A14D8451E042D11D889
:1037800005236B439B18012215009D402B00064822
:1037900005682B430360054B1B68002B02D02000FB
:1037A00002F037FB002070BDF40F0020D41A002077
:1037B00070B508680D00FFF785FF04006868FFF723
:1037C00081FF621E0100042A13D8451E042D10D863
:1037D00005236B439B1801229A40074803689343D3
:1037E0000360064B1B68002B03D00022200002F070
:1037F00010FB002070BDC046F40F0020D41A00203A
:10380000F0B5050089B008680C00FFF75BFF069073
:10381000022D36DD6068FFF755FF0190A068FFF7C5
:1038200051FF04000127231D661E0793731C02939A
:10383000079B9E4235D0052373430593019B019D51
:1038400005330493049BAB421ED0042E16D86B1E86
:10385000042B13D80122059B2349013B5B199A4095
:103860009446224A0B681068069A3A4003920DD09B
:1038700062461A430A60012200280DD17F000135FB
:10388000E0E701240194CDE7029ECFE7624693432F
:103890000B600028F2D0039A0299280002F0B9FACE
:1038A000ECE7019B1E1D042E1AD8012C18D100250F
:1038B00005273B0021006B439B1999400B000A4AE6
:1038C000013511689943094B11601B68002B05D025
:1038D000019B0022581D290002F09BFA052DE8D11A
:1038E000002009B0F0BDC046F40F0020D41A00201B
:1038F00010B5041E10DA00240A4BA400E25801237C
:103900009340094A09491360094A1160094A0A4962
:1039100011600A4A136010BDFFF7B6F8A042EADD55
:10392000EAE7C0460CCF0000EC0F0020080500506D
:10393000E40F0020E00F00200C0500501805005097
:103940002B4BF7B51B680C00002B03D10120404224
:10395000FFF7CEFF24680126250035401AD0FF224C
:103960006310120260121040DAB21043FF221B02F1
:103970001204134018431F4B1B68202B06D1B44080
:103980001D4BA40EA400E35800021843FFF7C8FD26
:103990000020FEBD042CFBD90F2322681340092B05
:1039A000F6D1FF2763683F025B100193019B9D42A4
:1039B000EEDAAB00E3189B68334216D05A10581267
:1039C000D1B238400843FF21120209040A401043D3
:1039D000084A1268202A06D15B009B0E06499B000C
:1039E000020258581043FFF79BFD0135DEE7C04641
:1039F000EC0F00202000002048C4000002000868EE
:103A000010B5C3070FD540101823012A03DD4A68FB
:103A1000042A00D10833054A1360FFF757F8FFF76F
:103A200067FF002010BD01204042EDE7200000208C
:103A3000086810B5C30703D5FFF744FE054B1860AF
:103A4000054B1B68002B03D0024B186802F0E2F90B
:103A5000002010BDF40F0020D41A00207FB5A04C28
:103A60002368002B0AD19F4A1268002A06D19E4B78
:103A70001B68002B01D0FFF7A1FD7FBD9B4D2A687D
:103A8000002A26D1984A1268002A1BD0FFF796FD1B
:103A90000028F2D0FFF77EFD924B24681A681C6064
:103AA000002A16D0002C14D101AD0C229049280018
:103AB00006F064FE285D00210134FEF7E7FF0C2CC0
:103AC000F8D1DAE7874A1268002AE5D1002BE3D063
:103AD000E0E700211A2003F063F800211B2003F027
:103AE0005FF800211C2003F05BF82E68012E5CD0EB
:103AF000022E00D1A2E0002E50D101363100794CC7
:103B000003202368994303F04BF804202168014007
:103B10004B42594103F044F8102123680A20194010
:103B20004B42594103F03CF88021236809011940B8
:103B30004B425941062003F033F8802123680902E3
:103B400019404B425941072003F02AF8802123688D
:103B5000490219404B425941092003F021F88021C4
:103B60002368890219404B425941192003F018F883
:103B700080212368C90219404B425941182003F0A3
:103B80000FF8802321681B0319404B42594117202D
:103B900003F006F831001A2003F002F82B68032125
:103BA000581C04F0A9FD296067E702214D4C17203D
:103BB000236819404B42594102F0F2FF0821236863
:103BC000182019404B42594102F0EAFF8021236836
:103BD000C90019404B425941042002F0E1FF802105
:103BE0002368490119404B4259410A2002F0D8FF8D
:103BF00080212368C90119404B425941032002F03A
:103C0000CFFF80212368890319404B425941092085
:103C100002F0C6FF802321681B0419404B42594122
:103C2000192002F0BDFF3100062002F0B9FF31007B
:103C3000072002F0B5FF31001B20ADE72021294C01
:103C40001720236819404B42594102F0A9FF402137
:103C50002368182019404B42594102F0A1FF8021EE
:103C60002368192019404B42594102F099FF8021E5
:103C70002368490019404B425941092002F090FF46
:103C800080212368890019404B425941072002F0E6
:103C900087FF80212368890119404B425941062042
:103CA00002F07EFF80212368490319404B425941AD
:103CB0000A2002F075FF80212368C90319404B4296
:103CC0005941032002F06CFF802321685B041940F6
:103CD0004B425941042002F063FF01211C205BE7A5
:103CE000F40F0020E80F0020F80F0020DC0F002068
:103CF00060C20000012010B54042FFF7F9FD10BD81
:103D000010B5034A0921034800F0A6FF10BDC046C4
:103D100048C5000090C5000030B502248025094B3D
:103D2000094AED009C505C59002CFCD0A124E40011
:103D3000884202D30021995030BD8025ED001851F2
:103D40004019F5E700E001400405000010B5002827
:103D500006D1C020B02140028902FFF7DDFF10BD6F
:103D6000B02080218002C902F7E700004342584199
:103D7000064B40421840B0239B02C0180368002045
:103D80001A0E532A01D11B02180A704700C0FEFF09
:103D900030B501248025054B054AED009C505C5947
:103DA000002CFCD001600021995030BD00E00140A2
:103DB0000405000043425841074B40421840B023DD
:103DC0009B02C018A62310B50902DB05090A194396
:103DD000FFF7DEFF10BDC04600C0FEFF70B5012436
:103DE00080250D4B0D4EED009C515C59002CFCD0F4
:103DF000002902DC00229A5170BD557814782D02FA
:103E000025439478013924042543D47804322406C8
:103E10002C4310C0ECE7C04600E001400405000060
:103E200070B505004B680A009C1C2100A400FFF738
:103E3000D5FF281970BD0000134B1B68002B0CD058
:103E40008022B023D2029B0200280BD11A1D5B688E
:103E50001B0E522B00D110007047B022C0239202DB
:103E60005B02F1E782420DD903681B0E522B09D188
:103E7000436802339B00C018824203D903681B0EBB
:103E8000522BE9D00020E7E7FC10002070B500209D
:103E9000FFF7D2FFFF260500002801D1280070BDE2
:103EA00003681C143440FFF7C7FFDA2CF4D1050077
:103EB000F2E700008022F0B55200A1B0002167486F
:103EC00006F078FC802200215200654806F072FC62
:103ED000644BFF271B681A00049353425A41100099
:103EE0000592FFF733FF049C0020631E9C415E4B4C
:103EF00064421C405D4BE418FFF7C8FF0600002E2B
:103F00002DD10498FFF732FF411C0598FFF752FFAF
:103F1000059A574D534B2C601A60FEF7C7FF514B63
:103F200064201B68A0215A4253414F4A5B42134010
:103F3000B0222C6892029B18E41A6043490204F0F4
:103F4000F5FAA0225202030000924A49220007A873
:103F500006F074FF07A801F09DF821B0F0BD3268AB
:103F6000131412123A403B4003921A000A3A092AEB
:103F700049D83A4B039A995C002931D110223E4826
:103F800006F018FC35002B6803991A123A4091424A
:103F900009D11A143A400B2A27D0132A2DD00A2A05
:103FA00001D1354B1D602800FFF746FF051EEAD101
:103FB000314B196800290FD02000FFF731FF0400B2
:103FC0002D4B5B195968002903D02000FFF728FF0B
:103FD000040004350C2DF3D1204B0121039A995490
:103FE0003000FFF729FF060089E73B40022BDADCAF
:103FF000214A9B00D3185D60D5E7102200211E489E
:1040000006F0D8FBCFE71A00153A082AE8D8144A78
:104010000399525C002AE3D13500152B00D015001E
:10402000300003681A143A40152A0FD01D2A00D117
:104030000025FFF701FF0028F3D1002D04D0200058
:104040002900FFF7EDFE0400054BC6E7039A1B129B
:104050003B409A42EDD10500EBE7C046FC0F002043
:1040600004110020FC10002000C0FEFF04C002006C
:104070000011002029C60000102F0020F0B50020FC
:10408000B7B00024FFF7D8FE270005002600002D5A
:104090002ED1284D2868FFF769FE32003B000190C1
:1040A0000094254904A806F0C9FE04A800F0F2FF18
:1040B000224B64201C682B68A0215A425341204A9D
:1040C0005B421340B02292029B18E41A60434902FB
:1040D00004F02CFAA0225202030000921949220097
:1040E00004A806F0ABFE04A800F0D4FF37B0F0BD82
:1040F000FF226B6829689C460233FF180B120136B9
:1041000013409C4200DA1C00FF200A140240039274
:104110006246014001920091039A0B4904A806F0FF
:104120008DFE04A800F0B6FF2800FFF785FE05000D
:10413000ADE7C046FC1000209AC600000011002028
:1041400000C0FEFF44C6000086C6000070B5002017
:10415000FFF70CFE04000120FFF708FE844200DA9E
:1041600004000A4B1D686A42554128001D60FFF794
:10417000EDFDA0226B4252021340054A28009B1815
:10418000044A611C1360FFF715FE70BDFC1000208F
:104190000480010000110020F8B50020FFF7E6FDC3
:1041A00007000120FFF7E2FD3E00204D0643204CB2
:1041B0000DD18021C020C9024002FFF7ADFD0121D1
:1041C0003000FFF7F7FD1B4B2E6023601DE0874298
:1041D00009DD0023B0212B60164B89022360236880
:1041E0000020012517E0012380212B60124BC9021A
:1041F0002360F4E7120E522A08D0002800D0236072
:104200000E4800F047FFFFF7A1FFF8BD28005A68ED
:10421000023292009B188B4205D21A68561CE9D1D3
:104220000028F2D0D1E72160EFE7C046FC10002063
:10423000001100200480010004C002005FC60000DD
:10424000F0B585B0039203220333DC17294D1440E7
:10425000E4182B68284F5A42534180225B42D20215
:10426000A4103B409B18A21C0291244E9100009187
:104270000190316800980A18934215D2FFF71AFE90
:104280002B685A42534180225B421F40D202BF1822
:104290003368009A9B189F4206D2194800F0FAFE34
:1042A0000025280005B0F0BD029B356819066B4655
:1042B0001A7BA423DB051343FF222F00090C1943AB
:1042C000019B12041B04134019432800FFF760FDF3
:1042D0000837281D21003760FFF75AFD002C04D055
:1042E0000A9A21003800FFF779FD009B083BFF1870
:1042F0003760D6E7FC10002000C0FEFF0011002050
:1043000003C6000010B5FFF7D5FD10BD70B59AB01B
:10431000FFF742FFFF221E4CD2000021200006F0D2
:1043200049FAFF25FFF7B2FD0026002814D102004C
:10433000C300E3580130591E8B41D218FF28F7D132
:10434000144901A806F07AFD01A800F0A3FE124866
:1043500000F0A0FE1AB070BD03681A142A400A2AA1
:104360000AD11A122A40FF2A03D0D200A1180B71D9
:10437000A050FFF761FDD8E7132AFAD11B122B409A
:10438000FF2BF6D0DB00E2181671E650F1E7C046CD
:1043900088250020CFC60000E3C600000021094B9D
:1043A000094A59600131516059680029FCD0002147
:1043B0001961012393600222044B8131FF315A506D
:1043C0001A607047FC1000400010004000E100E05F
:1043D0000222064B0121DA670022054B5A61054A89
:1043E00011615A69002AFCD07047C04604E100E020
:1043F000FC1000400010004010B5044C2378002B46
:1044000001D0FFF7E5FF0020207010BD051200204D
:10441000802301205B055B6E5B0018437047000042
:104420000120024B1B685B00184370478812002074
:104430000120024B1B685B001843704724000020DA
:104440000120024B1B685B00184370478C12002050
:1044500070B504000D001600FEF70AFB8023012151
:104460005B055A6E2670002653006170E17062721F
:10447000010A5A0A6071A171A272010C5A0C000E55
:104480005B0EA6702571E1712072E272237370BD1C
:1044900010B5044C200006F009FD01002000FEF7D5
:1044A00089FF10BD911200200E4B10B51B680E4CF9
:1044B0005A1C0FD00D4C002B0CD00D4C012B09D0E9
:1044C0000C4C022B06D0094C042B03D00A4C052BB4
:1044D00000D1074C200006F0E9FC01002000FEF7A7
:1044E00069FF10BD280000207BC7000074C70000D2
:1044F00086C700008BC7000080C7000070B5214C44
:104500002278002A3DD1204B01215A608022D20519
:1045100011605A68002AFCD0002207201B4B1C495E
:1045200001255A500439585008315A5019481A492F
:1045300058501A491A485A501A495A50A622D200BD
:104540009D50082218495A500431585002201749EA
:1045500058501749174858501748043958501820D0
:1045600016495850C12189005A500539FF39585809
:10457000921802435A501249124A9950FFF70EFFFF
:10458000257070BD05120020FC00004000100040A6
:104590000C050000746962751C050000240500000C
:1045A000200004022C050000140500003405000062
:1045B0003C050000FFFF0000211001005405000031
:1045C000061200200405000070B50E4B06001B7893
:1045D000002B01D1FFF792FF00200B4D2C78844275
:1045E0000ED00A4B202219780323091B1940084BCF
:1045F0004901C918300006F0C1F80120013C2C70B7
:1046000070BDC04605120020901200200412002048
:1046100006120020002370B588B0984235DD0D6881
:1046200001262C0034409C422FD12300042D2CD98C
:104630000F222B681A402300092A26D16A683F2AD4
:1046400023DD6846FFF7C0FF230000281DD06B461E
:1046500019783300A14203DB6B461B5D5B003343DB
:10466000A200AA1801349360202CF2D109216944D8
:104670004A780B7812021A438B781B041A43CB78C2
:104680001B061343024A13600423180008B070BDD0
:104690008C12002070B5454B8AB01B78002B01D1DD
:1046A000FFF72CFF02AC2000FFF78EFF002802D19D
:1046B00000200AB070BD23780B2BF9D96378012B49
:1046C000F6D1E378012BF3D100231120384E394D78
:1046D00033602B7068442379374A4178136002783D
:1046E00009021143827812041143C27812060A4368
:1046F00032490A60002B0ED1152169444A780B78A3
:1047000012021A438B781B041A43CB781B061343FF
:104710003360002318E0012B1AD1152169444A782F
:104720000B7812021A438B781B041A43CB781A2198
:104730001B06134333600E23627C6944934200DD01
:10474000130000229A422CD100220420EA54B0E740
:10475000022B03D1627B10331621EEE7042B0DD11F
:10476000152108226944684606F008F80098019966
:1047700002F088FA05F0B4FE3060CAE7052BC8D114
:10478000152108226944684605F0F8FF0098019950
:1047900002F078FA05F0A4FE3060627D0A231E2143
:1047A000CBE7885CA8540132CCE7C0460512002054
:1047B0008812002091120020280000208C12002076
:1047C00010B5134B04001B78002B01D1FFF796FEA8
:1047D000FFF7FEFD00200F4A0F49104B5450586060
:1047E0000130106058680028FCD0002018610130AA
:1047F000906018690028FCD0094B0A481B785B01BF
:104800001B185350FFF7E4FDFFF7C8FD10BDC0466D
:10481000051200200010004004050000FC100040BC
:10482000041200200612002010B588B000281DDDFB
:104830000A68012113000B4018D1042A16D90F2051
:1048400014682040092811D150683F280EDD9800D7
:10485000101880680024084201D04010C4B2684695
:10486000C4540133202BF2D1FFF7AAFF002008B077
:1048700010BD000010B5002813DD0C68E30710D54B
:104880006410532C0DD8084B1B78002B01D1FFF777
:1048900035FEFFF79DFDA123044ADB00D450FFF74E
:1048A0007DFD002010BDC046051200200010004014
:1048B00010B500280EDD0C68E3070BD56410FF2C43
:1048C00008D8054B1B78002B01D1FFF717FE034AD0
:1048D000034BD450002010BD0512002000100040F2
:1048E0002405000013B5002814DD0C68E30711D57A
:1048F000094B64100093094B0193072C0AD8084B0D
:104900001B78002B01D1FFF7F9FD6B46054A1957BB
:10491000054BD150002016BDE2ECF0F4F8FC000489
:1049200005120020001000400C05000070B588B092
:10493000002820DD0124086804401CD104281AD96D
:104940000F2302681340042B15D1FEF725FB060048
:1049500006F0ACFA0500122800D912252A0002211F
:104960000D326846FFF774FD6B465D73A54205DCAA
:104970006846FFF725FF002008B070BD2300325DB8
:104980006B449A730134F1E7F0B50D008BB0012848
:1049900032DD08680122040014402DD104282BD9EF
:1049A0000F2301680B40042B26D16B68134223D0E0
:1049B000FEF7F2FA6E6807007310019306F076FABC
:1049C00005000E2800D90E252A000121113202A867
:1049D000FFF73EFD6A46127902AB5A7302AA7312C0
:1049E0009373019B76141B0ED67313745574A542F2
:1049F00005DC02A8FFF7E4FE00200BB0F0BD3A5D35
:104A000002A963189A740134F1E730B589B000281F
:104A100014DD0C68E30711D5102268460021FFF76A
:104A200017FD6B466A4665105D73684663122D0E6E
:104A300064149373D4731574FFF7C2FE002009B099
:104A400030BD0000174B184A5968002903D00021D7
:104A5000596001319160196900291FD00020186147
:104A60008023DB00D3581149012B18D1A923DB0087
:104A7000D3585B420B600E490B78032B01D80133EE
:104A80000B7003200B490B78013303400B700A496C
:104A90005B015B180949535001239360704708601C
:104AA000FAE7C046FC10004000100040240000203F
:104AB00090120020041200200612002004050000BD
:104AC00010B5034A1021034800F0C6F810BDC046D7
:104AD000F4C60000EBC60000044A05491368C85438
:104AE00001339B059B0D13607047C046C016002024
:104AF000C012002070B5114C114A2368834202DCB9
:104B00000023236016E0155C411C2E00FA3E012EA6
:104B100005D899420FDA555C013D1F2D01D90800D7
:104B2000ECE70100151A565C6E5401318B42FADC39
:104B3000181A206070BD1570FAE7C046CC1A002024
:104B4000CC16002010B5FDF789FF064B1A6882428B
:104B500001D900221A601B68C31A03489842804199
:104B6000404210BDBC120020204E000010B5094C80
:104B7000094A23681268934200D110BD074AD05CED
:104B8000FEF78CF90028F8D0236801339B059B0DB4
:104B90002360ECE7C4160020C0160020C0120020DD
:104BA00010B50400064B074A1B6812689B1ADB43CA
:104BB0009B059B0DA34200DB10BDFFF7D7FFF1E77C
:104BC000C0160020C416002070B50020FFF734F98D
:104BD000FF260500002801D1280070BD03681C14C1
:104BE0003440FFF729F9DA2CF4D10500F2E7F7B5E4
:104BF000050056680191B000441C06301700FFF70D
:104C0000CFFFFB20FFF768FF1C20FFF765FFE8B22E
:104C1000FFF762FFE0B22412FFF75EFFE0B2FFF79A
:104C20005BFF6B461879FFF757FF0025AE4200DCAB
:104C3000F7BDAB00FB189C680135E0B2FFF74CFFF5
:104C40002012C0B2FFF748FF2014C0B2FFF744FFA4
:104C5000200EFFF741FFE9E770B5074E3368092BD7
:104C600008DC0C255D43054C013328516419616053
:104C7000A260336070BDC046C8160020202F0020FF
:104C8000F0B587B002900C00012803DC1B20FCF774
:104C90005BF945E0244B08680093C30709D4042856
:104CA00007D90F2302681340042B02D1FEF774F9D1
:104CB00000901D4B60680193C30709D4042807D9ED
:104CC0000F2302681340042B02D1FEF765F901900F
:104CD0000027164B1B680493049BBB42D6DD0C26B1
:104CE0007E43134B0099F618306806F0D5F8051E80
:104CF00005D17368B6680593059B9D4201DB0137BA
:104D0000EAE730680199039606F0C6F808360028ED
:104D100008D121000298039B083102385B6898474C
:104D200007B0F0BD0135E7E763C10000C8160020F9
:104D3000202F002010B5FCF753F8FEF7E1FFFEF737
:104D40004FF8FEF79DFBFEF7D3FBFFF7B9FE00F02F
:104D50007DFE01F061F810BD962210B51201002110
:104D6000034805F027FD0022024B1A6010BDC04623
:104D7000281C0020CC050020064B074A1B6812683F
:104D80009B1ADB439B059B0D0122834200DC002222
:104D900010007047C0160020C4160020F8B50500AA
:104DA0000C0016001F1E0ED10320FFF7E5FF0028A0
:104DB00008D0FA20FFF790FEE8B2FFF78DFEE0B2D0
:104DC000FFF78AFEF8BD501DFFF7D6FF0028F9D087
:104DD000FB20FFF781FEE8B2FFF77EFEE0B2FFF7AF
:104DE0007BFEF0B2FFF778FE3012C0B2FFF774FE20
:104DF0003C00E31B9E42E5DD2078FFF76DFE0134A9
:104E0000F7E7000070B50024F0250B4B1B68A342A8
:104E100002DCFFF7A1FF70BD2B006343074A9B181C
:104E20001A78002A05D05978002311201A00FFF7BC
:104E3000B5FF0134E9E7C046CC050020281C00205E
:104E4000F8B507000024F0252B0063430C4A013419
:104E50009E18B74211D0317800290BD00133D15CB4
:104E6000002311201A00FFF799FF2A0000213000CB
:104E700005F0A0FC0A2CE7D1F8BD024B1C60F9E755
:104E8000281C0020CC050020F0B5150001222F00C1
:104E90005E4C1740A54401900291002F11D005AB44
:104EA0001A706A105A70120E1A71052269129970DE
:104EB0006D140299DD70FFF771FFCF239B009D44B5
:104EC000F0BD042D1ED90F232A681340042B25D1D1
:104ED000023B04AA28001371FEF75EF8040005F0F7
:104EE000E5FF4B4B984200D91800B84204DC421C45
:104EF00005AB02990198DEE701377B1EE35C05AA4A
:104F0000D355F2E7042D7CD1032304AA043D137189
:104F10006B425D4105AB55710222EAE7092BCCD10A
:104F2000042205AB1A706A6851100091694652124A
:104F300009789A70009A59701F2A01DD2022009288
:104F40006A46127806ACDA70009BBB4202DC05AB05
:104F5000E21ACEE70126BB00EB189868064006D19E
:104F6000042837D90F2302681340022B0CD10123E8
:104F700023704310637042121B0E4014A270E07045
:104F8000237105340137DFE7042B21D1023B237065
:104F9000FEF702F8039005F089FFA31C0C2809D83E
:104FA0006070864201D19C19ECE7039A925D9A5594
:104FB0000136F6E70C226270039A925D9A5501362B
:104FC000092EF9D12E23E372237363730E34D9E7CC
:104FD000012B07D1032304382370434258416070EA
:104FE0000234CFE7092B09D1053B23704368E670F3
:104FF0005A105B126270A3700434C3E72670013448
:10500000C0E7002D00D058E77EE7C046C4FCFFFF94
:105010002303000070B502000024F0210D4E0800AB
:10502000604380194578954203D001340A2CF6D1AB
:1050300070BDF022002105F0BDFB074A1368013B5B
:10504000A34200D11460002329001A001120FFF7A9
:10505000A5FEEDE7281C0020CC05002010B5B2B05D
:1050600002236A460400137005F020FFC72800D908
:10507000C7200023984207DC421C6B46FE21142007
:10508000FFF78CFE32B010BD694601335A1EA25C98
:10509000CA54EFE730B5B3B002236A460500137077
:1050A00005F004FF0400C72800D9C72400239C4250
:1050B0000BDC20003230FFF773FD621C6B46FF21D2
:1050C0001420FFF76BFE33B030BD694601335A1E22
:1050D000AA5CCA54EBE70000F7B5234B06001B6837
:1050E000F02100930023009A9A4211DC0024F0235F
:1050F0001A006243019201991C4A55182F78002F1B
:1051000012D001340A2CF3D11948FFF7C3FF29E06C
:105110000A005A43154882185078B04202D11278DA
:10512000002A1FD10133DEE7F0223900280005F004
:1051300041FB02230D4A0199EB6053540D4AF100E3
:105140008A58009B6E70AE70AA602F616F61A34297
:1051500002DC054B01341C60002331001A001020D2
:10516000FFF71CFEF7BDC046CC050020281C002020
:105170008DCC00008825002010B5FFF743FEFF24EA
:10518000084AE3005B429B18074AD35C043B012BAF
:1051900003D8E043C0B2FFF79FFF013C002CEFD1E2
:1051A00010BDC046FC07000088250020F7B50F00A1
:1051B000FF247F2501901E4AE300D31A1D4A9A1846
:1051C0001278062A01D0032A20D1FF22D2009B1890
:1051D000186883682B401C2B18D1C3681A002A401A
:1051E000042A13D102692A40192A0FD11B0A01335C
:1051F0009B000C30C018FDF7CFFE03780600002B93
:1052000010D005F053FE0023B84209D0013C002C19
:10521000D1D1F7BD019AF15CD25C9142F6D1013354
:105220009F42F7DCE043C0B2FFF756FFEEE7C0460F
:1052300088250020FC07000070B50500FF24084AFF
:10524000E3005B429B18074AD35CAB4203D1E043C7
:10525000C0B2FFF741FF013C002CF0D170BDC04649
:10526000FC07000088250020F7B5FDF7F7FB514B40
:105270001A68824201D900221A601A684E49821ABD
:105280008A4200D883E01860FDF7F2FB071E00D1C8
:1052900001370020FDF7DEFC01900020FDF7EEFC59
:1052A000019B0090454C464D002B14D02368002BE9
:1052B00000D07AE02B682760002B00D171E0414BD1
:1052C00001261B78002B63D10920FFF7B5FF3E4B69
:1052D0001E703C4B1E70009B002B12D02B68002BC5
:1052E0000FD123682F60002B1ED0374B01261B786F
:1052F000002B52D10920FFF79FFF334B1E70314B1B
:105300001E702368002B0FD02F4E3278002A0BD14D
:105310009F4200D227602368FB1A312B04D9072053
:10532000FFF78AFF012333702B68002B0FD0254E27
:105330003278002A0BD1BB4200D92F602B68FF1AAC
:10534000312F04D90820FFF777FF0123337023683A
:10535000002B0CD0019B002B09D11B4E3378002B66
:1053600002D10720FFF768FF0023236033702B680A
:10537000002B0CD0009B002B09D1124C2378002B62
:1053800002D10820FFF758FF00232B602370F7BDE0
:105390000720FFF751FF0C4B9CE70820FFF74CFF5D
:1053A000ADE7009B002B9CD1ABE7009A002A95D17A
:1053B000AAE7C046B81200200F270000A81200205C
:1053C000B0120020B4120020AC12002037B5002427
:1053D0000500FFF717FD01A80194FDF729FC210046
:1053E0002000FEF7ADF9FEF739FBFDF7D5FCFDF720
:1053F000EFFCFEF77FFCFDF757FBA54204D0FDF75D
:1054000077FD0248FFF746FE37BDC0467ECC000060
:10541000002310B501001A001120FFF7BFFC10BDDA
:1054200007B56B46197069465A7013128B701314C6
:10543000120ECB700A716B46010005221320FFF794
:10544000ADFC07BD10B50A0001001220FFF71CFDDE
:1054500010BD70B5050008000C003230FFF7A0FB4E
:105460002B00220000211B20FFF798FC70BD10B517
:105470000C000300110014202200FFF78FFC10BD68
:10548000012370B5FF24084A41185B42884201D3CA
:10549000D84370BD06781D0A234073409B009B587B
:1054A00001306B40F2E7C04660C80000002313B52E
:1054B00001930B4BC2000400D058002805D043686C
:1054C00008309900FFF7DCFF01900920FFF768FB27
:1054D00001AB042221001720FFF760FC13BDC0467A
:1054E00088250020F7B50190FFF76EFB0125040029
:1054F000FF276D42002C01D12800FEBD2668331421
:105500003B40152B0DD121000198083105F0C4FC5A
:10551000002801D135123D402000FEF78DFC04002B
:10552000E8E71D2BF8D101256D42F5E7F0B580279E
:105530009DB0FFF71BFBA54CA54D2068FF00391A55
:105540004019FDF791FC23680600C3182360002B67
:105550000ED11DB0F0BD2068391A2818FDF784FC63
:10556000236806001B182360FDF778FA994B186032
:10557000002EF0DC2B78FA2B00D037E12368022BC9
:1055800007DCFFF7DFFA0028E3D00120FFF7B2FACB
:10559000DFE76878AC78023818282BD802F032FFA1
:1055A00019002C0030003400370040002A004A0067
:1055B0007C0086008A00A000F10002012A002A0077
:1055C0002A002A002A002A002A002A002A002A008B
:1055D0001001FF2C0ED02000FFF71CFD00227E4B97
:1055E000E100CA505B181A712100009213001320C9
:1055F000FEF726FE0320C9E72000FFF76DFDF9E75F
:105600002000FFF707FDF5E7FFF7B6FDF2E7FFF72C
:10561000F9FB0020FFF7DAFE7048FFF73BFDE9E7F2
:10562000632CE7D86E4BA200D25821001520FFF75B
:105630002BFCDFE7FFF7C8FAFF270400002CD9D0C6
:1056400025682B143B40152B04D02000FEF7F4FBFB
:105650000400F3E72000083005F028FC06000530C0
:10566000FFF79EFAFB20FFF737FA2D121D20FFF7F8
:1056700033FAE8B2FFF730FAF0B2FFF72DFA301242
:10568000C0B2FFF729FA25002B1B9E42DDDD287AE8
:10569000FFF722FA0135F7E700211D2000910B00EA
:1056A0000A00FEF7CDFDFDF723FCA3E72000FFF77E
:1056B000FDFE9FE7FDF7E4F903AC4A4A6421009040
:1056C000494B200005F088FB02232000237005F0E1
:1056D000EDFB2300020000211620FFF75FFB89E7A6
:1056E00000243D4AE300D558002D27D06B689E006A
:1056F000701DFFF755FA2B000025320008332100FA
:105700000120FFF74BFB2F00FFF75EFA2E00002869
:1057100018D1002F04D03A0001212000FFF767FACA
:10572000002D04D02A0002212000FFF760FA002E8D
:1057300004D0320000212000FFF759FA0134FF2C79
:10574000CFD157E7FF2103681A120A40A24209D1BC
:105750001A140A400B2A08D10B400CD0012B0CD094
:10576000022B0CD0FEF768FBD1E7132AFAD10025F3
:105770002F002E00F6E70600F4E70700F2E7050029
:10578000F0E70024FFF73EFB2200210000942300F5
:10579000DA20FEF755FDFF222100D2000E4805F069
:1057A00009F880E7012C02D1FEF768FC22E7022C01
:1057B00002D1FEF7A7FD1DE70120FFF707FE19E75D
:1057C000002321001A001A2087E7C046CC1A0020C7
:1057D000CC160020BC1200208825002060CC0000E0
:1057E000802D002077CC000072CC0000FB2B00D075
:1057F000CBE62268042A00DCC3E62E79E878574B12
:10580000360206439E4200DDBFE6331D9A4200DCAD
:10581000B7E6EB5CFE2B00D0B7E66B78AC78771E72
:105820001B2B61D019D8072B47D0082B1CD0012B7C
:1058300018D1FF2C16D02000FFF7ECFB6D79484AF9
:10584000B31E009221002A000A20FEF7F9FC454B06
:10585000E400E0501B191D7104E01D2B56D048D305
:105860001E2B6AD0701D91E6632CFBD86A79022A40
:1058700013D0032A1BD0012AF4D1E979AB790902AC
:1058800019432B7AA4001B0419436B7A1B060B43A4
:105890005B001343344AA350E4E7002FE2DDB11E5E
:1058A0002F48FDF787FD304BA400E050DAE7AB79D5
:1058B000A4005A1E93419B00ECE7632FD2DC03AD9A
:1058C0003A002A49280004F059FF00232800EB552C
:1058D000FFF708FE0028C5DB234B8000C2582100DB
:1058E0001520FFF7D1FABDE739002048FFF75EFC2D
:1058F000B8E7FF2CB6D06A79022AB3D818490B2032
:1059000000912100B31EFEF79BFCABE7632F00DD87
:105910006327002303A99F420ADCFB430022DB1715
:105920003B40CB181A70152000917B1C2100EAE740
:10593000EA185279CA540133EDE7012C92D1002FB5
:1059400090DD6B79002B03D01C00322B00DD32245C
:1059500064235C43064B1C6084E7C046F6030000EA
:10596000D216002088250020802D0020D11600208E
:10597000040000200122094B1A60094A1368002B19
:10598000FCD00322074B1B68D8171040C018012316
:1059900080100638400018437047C04600C00040E1
:1059A00000C1004008C500400120704710B5064CFA
:1059B000200000F0AFFA0549200000F0D3FA0122E0
:1059C000034B1A6010BDC046D81A0020801A06008A
:1059D000D01A002010B501210D20FDF757F8012144
:1059E0000E20FDF753F800210F20FDF74FF8044C6F
:1059F000200000F01BFC1021200000F033FC10BD43
:105A0000901B002010B504680D20E30703D5641037
:105A1000FF2C03D91720FBF797FA10BDFFF7DAFF29
:105A2000E1B2024800F040FC0020F6E7901B0020A5
:105A300010B5FFF7CFFF0021034800F035FC43000D
:105A40000120184310BDC046901B002010B5034A2A
:105A500008210348FFF700F910BDC046A4CC0000A0
:105A6000E4CC00000D4B70B51B6804000E0015005F
:105A7000002B01D1FFF79AFFE1B2094C200000F0A2
:105A800008FBF1B2200000F00BFAE9B2200000F0B0
:105A900007FA200000F068FB70BDC046D01A002055
:105AA000D81A002010B501240368234205D04168AC
:105AB000214202D08268224203D10D20FBF744FA32
:105AC00010BD5810802801D91520F7E74910FF298B
:105AD00001D91620F2E75210FF2A01D91720EDE76D
:105AE000FFF7C0FF0020EBE7F7B50122140090425A
:105AF00022DD0D682A421FD01D4B15411B684C68E2
:105B0000002B01D1FFF752FFE9B201272500194E02
:105B10003D40300000F0BDFA002D0FD03C41300078
:105B2000E1B200F0BDF9300000F01EFB0024A042FD
:105B300002D02320FBF708FA2000FEBD042CF2D986
:105B40000F2322681340092BEDD163685B1001938A
:105B5000019BAB42E7DDAB00E3189968394204D002
:105B60004910C9B2300000F09BF90135F0E7C0469A
:105B7000D01A0020D81A0020144B70B51B680500FD
:105B80000E00002B01D1FFF711FF114CEDB22900DF
:105B9000200000F07EFAF1B2200000F081F900212F
:105BA000200000F081FA002801D0404270BD01229F
:105BB0002900200000F068FA200000F062F90028B7
:105BC000FAD0200000F062F9F0E7C046D01A0020B9
:105BD000D81A002010B501240368234202D041687E
:105BE000214203D10D20FBF7AFF910BD58108028DA
:105BF00001D91520F7E74910FF2901D91620F2E74E
:105C0000FFF7BAFF40002043EFE70000002370B524
:105C1000344D0400EB5601330BD10D211D20FFF74D
:105C2000ABFF5A2814D101222A212A703D38FFF7F0
:105C300019FF0023EB56022B2AD0032B49D0012B4E
:105C40004CD121001D200124FFF796FF644225E07E
:105C50000F211920FFF790FF332805D102235F227F
:105C60002B7020211A38E2E70D211E20FFF784FF58
:105C7000C7280AD1032300222A21A9382B70FFF755
:105C8000F1FE1B222A211E20D1E700232B70D0E732
:105C9000012C13D129211920FFF76EFF7F2801DD88
:105CA0000138FF3803007F3301DA7F20404264234C
:105CB0007F21584302F03AFC604370BD032C0BD1A6
:105CC0002B211920FFF758FF043CE7E72D2119206D
:105CD000B9E721001E20B6E7052CF7D001240020EB
:105CE0006442E4E72C00002070B50120FFF78EFF2E
:105CF00004000320FFF78AFF05000520FFF786FF59
:105D00006D43644340436419201804F01FFC01F004
:105D1000E9F804F0E5FB43000120184370BD10B51D
:105D20000120FFF773FF43000120184310BD10B599
:105D30000320FFF76BFF43000120184310BD10B58F
:105D40000520FFF763FF43000120184310BD00004A
:105D5000F8B501231C00984229DD0F683B4226D08C
:105D60004E6835001D4022D1042E20D90F22316803
:105D70000A40092A1BD173685C10202C00DD202406
:105D8000134B1B68002B01D1FFF710FE7F10F9B2F7
:105D9000104F2200380000F077F9A54214DA3800DD
:105DA00000F06FF8002804D101246D002C4320007E
:105DB000F8BD380000F06AF80122AB004000F3188B
:105DC00010439860AD18E8E764000125EEE7C0468F
:105DD000D01A0020D81A00200020704701207047F8
:105DE0000020704700207047012070470020704756
:105DF0000020704700207047002070470020704747
:105E00000020704700207047002070470020704736
:105E1000704770477047000010B5034A0E210348D1
:105E2000FEF71AFF10BDC04634CD0000A4CD00001F
:105E300010B5FCF7E1FFFDF781F8FEF77BFF0448A2
:105E4000FFF728F9FEF762FAFFF796F910BDC04692
:105E50002DCE000010B5FCF7DDFC10BDF8B5050037
:105E60000E0017000024BC4208D02B68315D1B686F
:105E700028009847002801D00134F4E72000F8BD3D
:105E8000704710B51C3000F061FA10BD10B51C3021
:105E900000F04EFA10BD10B51C3000F05DFA10BDD8
:105EA00070B5437E0D00002B01D1002070BD643021
:105EB000040000F05AFA0028F7D12000290000F071
:105EC00028FA0120F2E70000F7B50193FA23002534
:105ED00004009B0083600D4B4560083303601C3059
:105EE0000F00160000F00AFA2000643000F006FAF5
:105EF000074A2761B600B35820006375019B9B00D9
:105F00009B586576A576A375FEBDC04648CE0000B9
:105F10000CCF00000123A022C375837D0E49C1333D
:105F2000FF33D2059B009950437DC133FF339B0063
:105F30009950CC220169094B5204CA5005220169CB
:105F4000243BCA50827D01690833CA500269417DF1
:105F5000034BD1507047C0460C06000024050000DA
:105F60000C050000A022002310B50469D200A35044
:105F70000A4CA1420FD90A4C8C425B4109495B4251
:105F80000B40CD21C9045B18046907496350052102
:105F90000369995010BDCC235B04F5E7A08601008E
:105FA00090D00300000098FD24050000F7B5040020
:105FB00000200D000193824265D01600402A00D9CE
:105FC000402627001C37380000F0AEF9B1232269C3
:105FD000DB00D55080220123216992008B50A27EE4
:105FE000002A03D122691362226913600025731EFF
:105FF000AB4207D1019B002B04D0802202212369F0
:1060000092009950012223691A622369FC33DA68ED
:10601000002A02D19A6A002AF9D09A6A002A0BD182
:10602000DA60A3232269DB00D1583800C9B20135F8
:1060300000F06FF9B542DAD3019B2269002B0FD132
:106040001300FC339B6A002B0AD10133A376D36182
:106050002369FC33DA6C002AFCD00022DA640AE0FF
:1060600000230121A37651611A002369FC3399684A
:106070000029FCD09A602369FC339A6A002A01D077
:1060800000229A62E8B2FEBD10B50123FFF78EFF31
:1060900010BD0300AC3310B504001970643000F07B
:1060A00043F90123637610BD0023020070B5AC32C2
:1060B00043760D001178B12204000069D2008150AE
:1060C0008022216992008B50226901331362226978
:1060D000936026006436300000F038F9002812D0B2
:1060E000300000F025F91E4B2269D0502369FC33A3
:1060F0001A6A002A02D19A6A002AF9D09A6A002AFA
:1061000001D11A62E5E723690122002D0DD11900A2
:10611000FC31896A002908D1DA612369FC33DA6C21
:10612000002AFCD00022DA6407E05A612369FC33BC
:106130009A68002AFCD000229A6000202369FC3370
:106140009A6A82420BD098622169064A8B588B501A
:106150001800022B03D0181F431E9841033070BD56
:106160001C050000C404000010B50121FFF79CFFCE
:1061700010BD000010B51323142202490248FFF796
:10618000A3FE10BD00400040D81A002070B50025C5
:1061900004AC24780573A94205D10A4B0A4A23218D
:1061A0000A4804F07DFA01600949920052589B00A8
:1061B00002715B58A40083716358856043710223A8
:1061C000C37170BD68CE0000CDCE000076CE000059
:1061D0000CCF0000037B002B04D143738373036156
:1061E00001330373704700001FB50191A021002403
:1061F0000068C900D2B24450012A10D0A24209D08E
:10620000032A0AD0074A8350074B019AC250012340
:1062100043501FBD02221343F4E70422FBE706228A
:10622000F9E7C046540500002405000010B504003D
:10623000FFF7D0FFA1222368A179D200995061799C
:10624000064A20009950217904329950044B19686C
:106250005A689B68FFF7C8FF10BDC0460C050000D8
:10626000A41B00204BB2002B0FDB80233F290FD84B
:106270001F290FD80F290FD807290FD803290FD8A6
:106280001B060168074A8B50704780239B04F8E780
:10629000DB04F6E71B05F4E75B05F2E79B05F0E797
:1062A000DB05EEE7240500000368074A99501A0051
:1062B000FC32D1680029FCD0A321C9005858002322
:1062C000C0B2D3607047C0461C05000007B58022ED
:1062D000074BD2051A6000229A6002321A710F230E
:1062E0000C3200930349023B0348FFF74FFF07BD01
:1062F000A41B002000300040901B002010B540225D
:106300000021040004F056FA002320002364636493
:1063100010BD10B53F24026C531C2340446C9C42BA
:1063200001D08154036410BD0023036443647047AB
:10633000436C026C934206D03F21C25C01330B4098
:1063400043641000704701204042FBE7036C406C3F
:10635000181A00D540307047436C026C934201D04C
:10636000C05C704701204042FBE73F22036C406C59
:1063700001331340181A43425841C0B2704700001D
:1063800003210A4802680A430260094802680A4376
:1063900002600849084A094B9B1A03DD043BC858B0
:1063A000D050FBDC00F012F8F9F7AEFE24050040F7
:1063B000540500405CD4000000000020640200206E
:1063C000FEE7FEE7FEE7FEE7FEE7FEE72D4B10B532
:1063D0001A68D2B2012A0FD12B4A126812070BD1C8
:1063E0002A4AE0241168F0220800104021422DD1F1
:1063F0002749096811422CD01A68D2B2012A12D159
:106400002149096809070ED1F02020490968014097
:10641000402908D11E490968014204D18020C121C8
:10642000C005C90042501B68DBB2012B0DD1164BD1
:106430001B681B0709D1154B1A68F0231A40A02AC4
:106440000FD1134A12681A420ED010BD3028CFD097
:10645000D2E7104A104911608021104A09021160E8
:10646000CAE7D02AF1D1ECE70D4B1A68012A04D013
:106470000C4A1A601A68012AFCD1C0220A4B1A6021
:10648000E3E7C046E00F00F0E40F00F0E80F00F093
:10649000EC0F00F004050040DFFF07C0186C00405F
:1064A00000EC06407593000014EC06400120704794
:1064B00010B503681322DB69984710BD70470000D0
:1064C000054B0269D1500369FC331A6A002AFCD0DB
:1064D000002201201A6270471C050000030010B55D
:1064E0005C331A781F231A401E3B19009140114A51
:1064F000D167C222042104699200A150026953604D
:106500000269D360A02300220169DB00CA50012385
:106510000169094A5B428B500169084A8B50016945
:106520000C3A8B50016908328B501430FFF7FCFE97
:1065300010BDC04604E100E00C0500001405000099
:1065400010B51430FFF702FF10BD10B51430FFF77F
:1065500003FF10BD10B51430FFF7EAFE10BD0000B8
:10656000030070B55E331A780469724BE250030081
:106570005D331A780469704BE250030061331C7874
:1065800002696E4B012C00D09EE005005F352E782D
:10659000A225ED005651020060321578A12206694D
:1065A000D200B5500269D4509623DB00994200D83E
:1065B0008CE096231B01994200D88AE096235B0168
:1065C000994200D888E096239B01994200D885E043
:1065D000E1239B01994200D882E09623DB01994296
:1065E00000D880E0E123DB01994200D87DE09623CA
:1065F0001B02994200D87AE0E1231B02994200D89D
:1066000077E096235B02994200D874E0E1235B02B5
:10661000994200D871E0E1239B02994200D86EE0D4
:10662000474B994200D86CE0E123DB02994200D845
:106630006AE0E122002312038A425B41414A5B4245
:106640001340802252059B1801693F4A8B50A023BA
:1066500004220169DB00CA5000210369FC33D960C0
:106660000369FC331962012301690B6001698B60C6
:10667000C1210469890062501F215C3002780A4000
:1066800093406231314AFF31535000214156002975
:106690003CDA0F230B40083B2D4C9B089B001B1939
:1066A00003242140A140FC348C40DD69A5432C002B
:1066B000C0258D4029002143D9611F23017819404D
:1066C0001E3B8B40136070BD00246CE79E23DB02F1
:1066D000BAE79D231B03B7E71E4BB5E71E4BB3E795
:1066E000EC239B03B0E71D4BAEE71D4BACE71D4B06
:1066F000AAE71D4BA8E71D4BA6E71D4BA4E71D4BC2
:10670000A2E78023DB049FE71B4B9DE78C080F4B20
:10671000A400E41803230B40FF21C025DB009940AF
:10672000AD0066598E433100C0269E4033000B43B6
:106730006351C2E70C050000140500006C05000061
:1067400090D0030000D0BEFE2405000000E100E070
:1067500000ED00E000B013000050270000A04E0044
:1067600000F0750000509D0000F0EB0000903A0131
:1067700000E0D70100B0AF0300705F07F7B50093EA
:1067800008AB1B7800250193FA2304009B0083606B
:106790000E4B45600833036014300F001600FFF7FE
:1067A000ADFD23005C3327611E70009B084A9B00EF
:1067B000995823005D331970019B20009B009A5863
:1067C00023005E33DD701A70FEBDC04690CF00001E
:1067D0000CCF0000036910B51A00FC32D268040027
:1067E000002A0AD0A322D20099581430C9B2FFF768
:1067F00090FD00222369FC33DA6010BD10B5024819
:10680000FFF7E8FF10BDC046B01B0020162307B5F8
:10681000022200930249013B0248FFF7AFFF07BD88
:1068200000200040B01B002010B5002801D004F06B
:106830007DFA10BD7047000010B500F011F8FFF7A9
:10684000F9FF012000F000FAFFF7F2FAFFF702FB70
:10685000024B002BFAD000E000BFF7E70000000079
:10686000C420114B80001A5810491140C022120256
:106870000A431A50C0218022490092025A501A60DD
:106880008023A3220021DB05D20099500122F93098
:106890009A60074BFF301950C12002318000195017
:1068A000403019501A60704700E100E0FF00FFFF20
:1068B00000100140014B18607047C046780000206E
:1068C000F7B5002320285AD8384B8000C258042A34
:1068D0005BD007D8022A54D055D80423012A09D006
:1068E00000234CE0062A54D051D31A2A53D0022355
:1068F0001B2AF5D12E4A116808294ED909294FD0F3
:106900000A240226A02001252A4AC00015502A4840
:106910002A4D07681C20BF000740294801970068DE
:106920005759009027481B0207401F43C023009877
:106930009B020340FF2057515759000207401F4355
:10694000019B1F43009B58016023184007433E43AF
:10695000565101251C4B156058680028FCD00020BA
:106960005860A1230125DB00D3585560A025ED0018
:1069700050511BB2A14202D015D2611ACB4018006F
:10698000FEBD0823B6E71023B4E72023B2E7402377
:10699000B0E78023AEE70123ACE708240026B1E787
:1069A0000C000126AEE7091B8B40E8E70CCF000086
:1069B000740000200070004030000020040500003A
:1069C00034000020FF00FFFFFC700040F0B52028DD
:1069D0005BD8364B8000C258354B1E68002E30D134
:1069E000C227344BBF00D859334C03250440C02084
:1069F00000022043D851C024802064008000185138
:106A00002E4F18602E4B803CD859FF3CA043D851E4
:106A10000437D859A8432043D8510837D8590C35E2
:106A2000A8438446072065462843D851A820C000C3
:106A30001E50C1208026800076021E501C601C4B18
:106A40001C60142500202B001E4C2E004643365996
:106A5000771C1BD14343E250A0230325C132FF32F0
:106A60009200DB05D550184B1A68082A14D114235C
:106A70004343E3189A6812485132FF32920059603A
:106A80001150DA68C1239B00C250F0BD9642E1D09C
:106A900001300328D9D1F8E7082A02D9083AD140B1
:106AA000E5E708239A1A9140E1E7C0460CCF0000C1
:106AB000141C002000E100E0FF00FFFF04050000BF
:106AC0000090004038000020780000202149F0B5F7
:106AD0004A6C2148002A14D0A025A12600230124B5
:106AE000ED05F600C258571C06D0C7187F68002F66
:106AF00002D027009740AF5114333C2BF2D1002332
:106B00004B64A0230121DB0500260F009C461423C3
:106B10004B43C3181A1F1268104C0E4D92001419E3
:106B20005219526C002A10D01A00143A1268551CDF
:106B300009D0103B1B68FF2B05D03B0093406546F6
:106B40001A00074BEA50FC34666401310429DED197
:106B5000F0BDC046FC90004038000020009000408E
:106B60000C05000000B5202810D80C4A800083587E
:106B700003290BD8A0220800C133FF33D2059B00A4
:106B800001F036FC020905070021D15000BD0C219F
:106B9000FBE70421F9E70321F7E7C0460CCF00002B
:106BA00020280AD8074B8000C25801239340A02216
:106BB000D205002902D1044953507047A121C900D0
:106BC000FAE7C0460CCF00000C05000003000020CF
:106BD000202B0AD8A021A222C905D2008858034A36
:106BE0009B009B58D8400123184070470CCF0000F1
:106BF000F7B506000D000C008B180193019B671B75
:106C00009C4207D0336821781B68300098470134D4
:106C10000028F3D13800FEBD0849094A094B10B5D8
:106C20001B688858FA22190A1B0618439200002391
:106C300001F0B4FD4904C00B084310BD0010014031
:106C400004050000181C002070B5041E09D0FFF7D1
:106C5000E3FF050000F014F8FFF7DEFF401BA04241
:106C6000F8D370BD0022044B9A60044A13680133C4
:106C7000DBB213607047C046FC100140181C0020B6
:106C800070470000F0B5C64600B5CB0F9846404AA5
:106C90004B005B0D9A1882B00D000400132A2FDC04
:106CA000002A49DB3B4F17413E000E40064323D0EC
:106CB0007F08390029400C430AD03749BD438C4630
:106CC00063445C425C418023DB021341E4071D43C3
:106CD0004146CE0031492B008E1922003468756878
:106CE0002000290001F000FF009001910098019917
:106CF00022002B0003F090F802B004BC9046F0BDD7
:106D0000332A08DD8023DB009A42F5D102000B0014
:106D100001F0EAFEF0E7224A94460122634452421F
:106D2000DA400242E8D052080242D1D09443802295
:106D3000D2051A411443CBE74B005B080343DBD079
:106D40000B031B0B1C436342234380244D0C240381
:106D50001B0B23406D042B4319004346DA000F4BF5
:106D60009B181C685D6802000B002000290001F0E0
:106D7000BBFE009001910098019922002B0003F0C6
:106D80004BF842464B005B08D60733431900B3E784
:106D900001FCFFFFFFFF0F00EEFBFFFFC0CF000075
:106DA000EDFBFFFFF8B5274A4B005B0D9A180C006E
:106DB0000700132A10DC002A36DB234B13410B4259
:106DC0003AD0802424031441002064189C43060018
:106DD000250030002900F8BD332A0EDD802306008F
:106DE000DB000D009A42F4D102000B0038002100B4
:106DF00001F07AFE06000D00EBE7144D0600AC46EC
:106E0000012563446D42DD40AC4663460D000342FC
:106E1000DFD033239A1A323B93401818874200D9A7
:106E20004C1C63469843D2E7C90FCC070020531C83
:106E3000CDD1074B1C43CAE706000D000028C0D186
:106E4000C7E7C04601FCFFFFFFFF0F00EDFBFFFFA0
:106E50000000F03F30B5214A4B0087B05B089342F9
:106E60001EDD1F4A934205DD02000B0002F0D4FF35
:106E700007B030BD02AA00F095F803231840049A29
:106E8000059B012813D002281DD0002814D0029899
:106E9000039900F06FFB80231B069C466144E7E7E3
:106EA000002300220093002301F0DEF8E0E70298BF
:106EB000039900F05FFBDBE701240298039900943B
:106EC00001F0D2F8D4E7012402980399009401F06C
:106ED000CBF880231B069C466144C9E7FB21E93FB0
:106EE000FFFFEF7FF0B54746CE4680B58DB004007A
:106EF0000D0000F067FA294B06001B780F005BB20B
:106F00009846013310D022002B002000290003F006
:106F1000CBFA8146002807D1002200232000290057
:106F200001F014FC002806D1300039000DB00CBC73
:106F300090469946F0BD01230293194B069407959C
:106F400003934B460A93434604940595002B15D0B2
:106F5000002300221900100002F0E2F843460890D6
:106F60000991022B0ED103F0B9FB212303600A9B88
:106F70000193002B0CD1089E099FD5E70023002424
:106F80000893099402A801F0C1F90028EFD1EAE7BB
:106F900003F0A4FB0A9B01930360ECE77C00002054
:106FA000D0CF0000F0B54E464546DE465746E0B528
:106FB000E14B4C008FB09046894664089C4200DC4F
:106FC00087E0DE4B9C4222DCDD4A002900DC92E0B7
:106FD000DC4B02F021FFDB4B06000F009C4200D18E
:106FE0007EE1D94AD94B02F017FF02000B0041465F
:106FF00030000A604B60390002F00EFFD34BD24ADA
:1070000002F00AFF434601259860D9606BE0D04B3F
:107010009C4200DC8FE0CF4B9C4200DD55E1CE4A24
:10702000231592469A4451460905631A19001D001A
:10703000040003F055FA03F089FA02000B00200067
:1070400029000892099302F0E7FE0022C34B02F0E8
:1070500071FC0F00060003F043FA03F077FA040016
:107060000D0002000B00300039000A940B9502F06D
:10707000D3FE0022B94B02F05DFC002200230C90ED
:107080000D9101F05DFB002800D192E10023002268
:107090002000290001F054FB434243410133B04A30
:1070A00041460192022208A80092524600F07CFB61
:1070B0004B460500002B16DA802243461206944602
:1070C00042465B68454263445360D3686344D3607F
:1070D00009E00B00020041460A604B6000220023D9
:1070E00000258A60CB6028000FB03CBC90469946D2
:1070F000A246AB46F0BD934B01F0F6FC914B060067
:107100000F009C4200D13DE18F4A904B01F0ECFC16
:1071100002000B00414630000A604B60390002F06B
:107120007BFE894A894B01F0DFFC012543466D4215
:107130009860D960D7E701F049F88A4A8A4B06007F
:107140000F0002F0F7FB0022884B01F0CDFC03F0AA
:10715000C7F9050003F0FAF9794A7A4B04900591D2
:1071600002F0E8FB02000B003000390002F054FE90
:10717000754A06000F0004980599744B02F0DAFB7B
:10718000029003911F2D00DCC7E0029A039B3000A0
:10719000390002F041FE83468A4653465B002415BF
:1071A0005B0DE31A102B6CDD04980599D322674B15
:1071B000520502F0BFFB02000B00300039000292C2
:1071C000039302F029FE0A000100130006910792C2
:1071D00002003900300002F01FFE029A039B02F009
:1071E0001BFE06000F0004980599614A614B02F0EE
:1071F000A1FB32003B0002F00FFE069E079F0B0032
:107200000200390030000292039302F005FE4B00A9
:107210005B0D83468A46E41A312C32DD04980599C9
:10722000B822544B920502F085FB03000C000200CB
:10723000029303940B000698079902F0EDFD0200FB
:107240000B0006000F000698079902F0E5FD029A70
:10725000039B02F0E1FD484A0290039104980599CE
:10726000464B02F067FB029A039B02F0D5FD020039
:107270000B00300039000292039302F0CDFD8346EB
:107280008A465A465346414630000A604B603900F0
:1072900002F0C2FD029A039B02F0BEFD44460B00C1
:1072A0000200A260E3604B46002B00DB1BE75B465D
:1072B000236080231B065344636080231B069C4687
:1072C0006144A060E1606D420DE70B00020002F036
:1072D000A3FD434600259860D9601860596002E715
:1072E000D3221A4B520502F097FD214A214B0D0083
:1072F000040002F091FD02000B00414620000A60EC
:107300004B60290002F088FD1A4B194A02F084FDF7
:10731000434601259860D960E5E602000B00300085
:10732000390002F079FD6B1E154A9B009B5883467D
:107330008A46A342A5D130E7FB21E93F7BD9024031
:1073400000004054FB21F93F3163621A61B4D03D23
:10735000FB213941FFFFEF7FEAFBFFFF0000704197
:1073600058D0000083C8C96D305FE43F0000E03FA3
:107370007370032E8A19A33BC14920259A837B3958
:10738000D8CF0000D3220C4B520501F0ADFB0B4AC5
:107390000B4B04000D0001F0A7FB02000B0041465F
:1073A00020000A604B60290002F036FD034A044BBE
:1073B000B9E6032373E6C04661B4D03D7370032E73
:1073C0008A19A33BF8B54746CE46674B80B50A00FD
:1073D0000F00190005003940994200D19BE00400DC
:1073E0000100002F69DD3F1500D1B4E05F4B1203AF
:1073F0009C468023120B5B0313435B00CA0F674458
:107400009B184A00F80703D5D20F5B009B188A002F
:1074100079108C46002180201624894680030D189F
:107420009D4202DC29185B1B8144D50F5B00013CA7
:107430005B1952004008002CF1D1002080468020CA
:1074400020250027000609E08B425CD0D40F5B00AA
:10745000013DE31852004008002D16D0C4198B429C
:10746000F2DD27180E00002C49DB5B1AA24289418D
:1074700049425B1A121BD40F5B00013D804431006E
:10748000E31852004008002DE8D113434ED1434683
:107490005B0837494A468846494652104244C90764
:1074A00002D5802109060B4361460F05BD1818005F
:1074B00029000CBC90469946F8BD7B005B0803434D
:1074C0003900002BF5D0002F3CD1E30A153A6405B2
:1074D000002BFAD08020400303423FD1002700E078
:1074E0000F005B00791C0342FAD0250020208D405C
:1074F000401A2900D71B2200C2401A4376E7FE43F8
:10750000F60F8E19B1E79442A0D82718002CF6DBAD
:107510001E000023AEE702003B002800390002F005
:1075200009FA2A003B0001F0DFFAC2E743460133C3
:1075300003D0434601335B08ABE7012398460023A1
:10754000C144A6E73B00020002F066FC02000B000B
:1075500001F0E6FDADE713000022BBE701272100A3
:1075600020207F42C6E7C0460000F07F01FCFFFFFD
:107570000000E03FF0B54746CE4680B587B00092A8
:107580000193754B4F00814688467F089F4263DC1C
:1075900002F0A6FF002800D1D4E04A464346484600
:1075A000414602F0C7F904000D006C4A6C4B02F032
:1075B000C1F96C4A6C4B01F097FA22002B0002F0E3
:1075C000B9F96A4A6A4B02F027FC22002B0002F04C
:1075D000B1F9684A684B01F087FA22002B0002F0EB
:1075E000A9F9664A664B02F017FC22002B0002F054
:1075F000A1F9644A644B01F077FA22002B0002F0F3
:1076000099F9029003910022604B2000290002F0BA
:1076100091F9029A039B06000F002000290002F056
:1076200089F9009A019B04000D004846414602F08A
:1076300081F902000B002000290002F0EDFB02009E
:107640000B003000390002F0E7FB02000B000020C5
:107650004F4902F0E1FB70E002000B0002F06AF912
:1076600004000D003D4A3E4B02F064F93D4A3E4B9A
:1076700001F03AFA22002B0002F05CF93B4A3C4B45
:1076800002F0CAFB22002B0002F054F9394A3A4BAF
:1076900001F02AFA22002B0002F04CF9374A384B4D
:1076A00002F0BAFB22002B0002F044F9354A364BB7
:1076B00001F01AFA2B00220002F03CF9354B02903F
:1076C00003919F429FDD344B00229F423DDC3349B2
:1076D00000207B182E4916001F0002F09DFB04902D
:1076E00005910022294B2000290002F023F93200E5
:1076F0003B0002F091FB029A039B06000F00200062
:10770000290002F017F9009A019B04000D00484679
:10771000414602F00FF902000B002000290002F0A0
:107720007BFB02000B003000390002F075FB020009
:107730000B000498059902F06FFB07B00CBC904653
:107740009946F0BD00201249F7E7154B0026049238
:107750000593144FC5E7C046FFFF3F3ED43888BEAF
:10776000E9FAA8BDC4B1B4BD9EEE213EAD529C80E5
:107770004F7E923E9015CB19A001FA3E7751C1166B
:107780006CC1563F4C5555555555A53F0000E03F3F
:107790000000F03F3233D33F0000E93F0000E0FF3C
:1077A0000000E73F0000D23FF0B5DE464E464546BA
:1077B0005746E0B5DC4CA5440D9114001900A49A7D
:1077C0000993DA4B9200D6584D1E03901821E01E03
:1077D0000696029500F0AAFEC3430100DB1719408C
:1077E0004B1C9A009B1ADB001B190B9105934C1B39
:1077F000771918D4A59BA5009C463F1922AE654475
:10780000013707E0286802F0A1FE013403C6043501
:10781000BC4208D0002CF5DA00200021013403C658
:107820000435BC42F6D1069B002B01DA00F0FDFBCB
:10783000069B03990133DB009A46099BDA009446C4
:1078400000920022914672AA0492B94A614493467A
:1078500088469AAB63449B44029B002B00DABCE150
:107860005D4600260027039C4D442A686B6803CCC4
:1078700002F060F802000B003000390001F034F92A
:10788000083D06000F004445EFD1049B4B441E60A9
:107890005F6008239C46E144D145DDD10EA8042158
:1078A0008446494261448C46069A93009C44614652
:1078B00084460A910399083B63448C460C93009BD1
:1078C000009263449B46009A0498D10003008C46C2
:1078D000634408911E685F68002A33DD954980463D
:1078E0008C466244D300984470AB9A460EAB9946DE
:1078F0000022914B3000390002F01CF802F0F0FD3C
:1079000002F024FE00228D4B04000D0002F012F85C
:1079100002000B003000390002F07EFA02F0E0FDB8
:107920004B4601C39946434620001A685B6829000C
:1079300001F0DAF808235B429C46E04406000F00A1
:10794000D045D5D1059B30001A003900984600F08B
:10795000DFFCFF2300229B0504000D0001F0EAFF7D
:1079600000F038FC0022764B01F0E4FF02000B002F
:107970002000290002F050FA0D00040002F0B0FDD2
:10798000814602F0E3FD02000B002000290002F016
:1079900043FA060040460F00002800DCEEE0009BA2
:1079A00018215A1E92000EAB9B58091A1D000D415A
:1079B000A9448D405D1B0EAB9D5017231B1A1D4122
:1079C000002D2DDD01239C46009BE144002B00DCB3
:1079D0001CE20E9C0123002C00D0B5E0009A012A85
:1079E00009D099000EAA54580133002C00D0ACE005
:1079F000009A9A42F5D1059B002B0EDD012B00D198
:107A0000A8E1022B09D1009B0EA95A1E92000EABD1
:107A10009B5807939B029B0A8B50022D00D1C1E01B
:107A2000002300223000390000F08AFE009B00286D
:107A300000D194E2069A591E8A4210DC414A0A9803
:107A400094460EAA6344944600229B0063441C683B
:107A5000043B22438342FAD1002A00D0C0E0069BB7
:107A60000EAA013B9B00D358002B00D0B3E00122AB
:107A70000C9B043B596801320029FAD0009B9C46BC
:107A80006244110007921A0001338B4246DC0B98C6
:107A900063468046A59C4344A046099C9B00A146A2
:107AA0004A449844D30022AA9146049A99449446A1
:107AB000089BA59A63448446614494469A468B0089
:107AC000634400934346586802F040FD4B461860FB
:107AD0005960029B002B24DB4D46039C00260027A7
:107AE00001E0286869680CCC01F024FF02000B005B
:107AF0003000390000F0F8FF083D06000F005C453B
:107B0000EFD153469E60DF6004239C460433E0447B
:107B10009C46009BE144E2449845D3D1079B0093E7
:107B2000D1E600260027ECE794FDFFFFA0D100007E
:107B300018FEFFFFFFFFFF1F0000703E00007041B6
:107B400000002040FFFFFF3F002180225204141B51
:107B50000EAA5450009999420EDD0EA884469B004F
:107B60000EAA8900D25861446344CF4800E01A68E5
:107B7000821A04C38B42FAD101243CE7059B002BF7
:107B800006D1009B0EAA013B9B00D558ED1517E7C7
:107B90000022C64B300000F0F7FD002800D024E1A1
:107BA00000253DE732003B000020C14902F034F9D6
:107BB00006000F00002C00D132E7059A0020BC49D6
:107BC00000F0A6FB02000B003000390002F024F99F
:107BD00006000F0024E7012250E70026002754E6A4
:107BE0004B46059A079388468B000EA9CB58183A46
:107BF00008950592002B0DD18C464146AD4B434470
:107C00009B006344043B58680139183A0028F9D0B6
:107C100088460592059A0020A54900F079FB434665
:107C200004000D00002B00DA05E29E000EAB9C461E
:107C30004346DB0066449C46059370AB9946049F1F
:107C400067440097306802F081FC22002B0001F0AD
:107C500071FE002238607960974B2000290001F006
:107C600069FE083F04000D00043EB945EAD14AAB65
:107C700003939B4600239A46069B424699464346F9
:107C80000132029204934B46002B00DAAAE08020D6
:107C90008A4B009D9846C00589490026002700248C
:107CA00008E008239C460835E044544511DC43466F
:107CB000186859682A686B6801F03CFE02000B00E6
:107CC0003000390000F010FF013406000F00A1451C
:107CD000E7DA5B46C0C39B4601239C46009BE24417
:107CE000083B0093029B9A45CDD1049B9846A49BE8
:107CF000022B00DD8EE0002B37DC1FD1059B002717
:107D00001D00039B00249C461E006544083E2A6813
:107D10006B683800210000F0E7FE083D07000C000A
:107D2000AE42F4D1089B002B03D080231B069C4657
:107D300064443A0023000D990A604B600720079BBA
:107D400018409B239B009D443CBC90469946A2460C
:107D5000AB46F0BD009B0EA95A1E92000EAB9B587D
:107D600007935B025B0A8B5057E64346002B00DA11
:107D700070E100200021DB004AAAD61848AF326823
:107D80007368083E00F0B0FEB742F8D1089B002BA4
:107D900000D025E10B0002004A984B990D9C22600F
:107DA000636002F039F8434607000C00002B13DD36
:107DB00001254CAEB14638002E0021004C4601365C
:107DC0000CCC00F091FEA146B045F7DA089B070005
:107DD0000C00002B00D015E13A0023000D998A60B9
:107DE000CB60ABE70026002773E701239C46009B8E
:107DF000E1440225002B00DDEBE532003B000020D2
:107E00002B4902F009F806000F0009E60024F2E50C
:107E10004AAB0393A49B032B00D08FE74346002B70
:107E200000DC14E1039ADB009B46130091465B449F
:107E30001E685F68234B43440293DB00994448ABC0
:107E40009A464B465C681B681800210032003B00D4
:107E50000090019100F048FE04000D0002000B00AC
:107E60000098019901F0D8FF3B00320000F03CFE81
:107E70004B469860D9601C605D6008235B429C465D
:107E8000E14426002F00CA45DBD14346012B00DC2C
:107E9000E3E0039A13005B441E685F68029BDB000B
:107EA00099464A44904610E0FFFFFF000000E03F83
:107EB0000000F03FFFFFFF3F0000703E60D1000078
:107EC000FB21F93FFFFFFF1F984643465C681B6894
:107ED0001800210032003B000090019100F004FEE8
:107EE00004000D0002000B000098019901F094FFBE
:107EF00032003B0000F0F8FD4346039A9860D960D9
:107F00001C605D60083B26002F009A42DCD14D4684
:107F10009446002600244746083565442A686B6865
:107F20003000210000F0E0FD083D06000C00AF42EB
:107F3000F4D1039B4A9F5D689968D868089B002B21
:107F400065D08022120694460D9B654460446444CB
:107F50001F605D609960D8601E615C61EEE69A46C4
:107F60004B460793059B30005A423900089500F0B4
:107F7000CFF900223A4B06000F0000F005FC002864
:107F800024D0384B00223000390001F0D3FC02F03D
:107F9000A7FA52460400950002F0D8FA0022304BAE
:107FA00001F0C8FC02000B003000390001F034FF82
:107FB00002F096FA0EAA50510122059B5244183342
:107FC0009046059393000EAAD45023E65346300002
:107FD00039009C0002F084FA0EAB1851D04619E625
:107FE00080230D9A1B06CB18106053600B00020013
:107FF0004A984B9901F010FF434607000C00002BF4
:1080000000DDD5E680231B069C466444E4E62B0095
:108010003A000D9D2A606B600A000300AA60EB60C5
:10802000320023002A616B6188E6099BDB00009324
:1080300072AB049332E4A49B022B00DDE8E6002B34
:1080400000DD92E600D079E6002700246AE60026EB
:1080500000246EE70020002198E60026340068E73F
:10806000000070410000703EF0B5CE46474680B536
:1080700087B000920193474A4B00814688465B08CF
:10808000934207DC4146484602F02AFA4146031E65
:10809000484666D04A4643464846414601F04AFCB7
:1080A00004000D0002000B004846414601F042FC6E
:1080B000394A3A4B06000F002000290001F03AFC33
:1080C000374A384B01F0A8FE22002B0001F032FCA9
:1080D000354A364B00F008FD22002B0001F02AFC47
:1080E000334A344B01F098FE22002B0001F022FCB1
:1080F000314B324A00F0F8FC0E9B02900391002BAA
:1081000034D00098019900222D4B01F013FC029A03
:10811000039B049005913000390001F00BFC020034
:108120000B000498059901F077FE22002B0001F066
:1081300001FC009A019B01F06FFE224A04000D0031
:10814000214B3000390001F0F5FB02000B0020004C
:10815000290000F0C9FC02000B004846414601F02E
:108160005BFE07B00CBC90469946F0BD02000B00C8
:108170002000290001F0DEFB124A134B01F04CFEF7
:1081800032003B0001F0D6FB4A46434600F0ACFC0F
:10819000E7E7C046FFFF3F3E7CD5CF5A3AD9E53DE1
:1081A000EB9C2B8AE6E55A3E7DFEB157E31DC73EA8
:1081B000D561C119A0012A3F1111813FA6F8101104
:1081C0000000E03F495555555555C53F49004B08FE
:1081D00019007047474AF0B54F4691464B005B0D7A
:1081E00099444646D6464A46C0B505000C000E00E6
:1081F00088460700132A27DC002A4BDB3E4B13413D
:108200009A460B0052461340034318D03B4A3C4B5E
:108210002800210000F068FC0022002300F0AAFAE8
:10822000002847D0002C04DA80234A465B03134120
:1082300098444646534600279E43380031001CBCF4
:1082400090469946A246F0BD332A08DD8023DB0024
:108250009945F4D102000B0000F046FCEFE7294AF3
:108260009446012263445242DA4092460242E6D0EA
:10827000224A234B2800210000F036FC0022002374
:1082800000F078FA002815D0002C1EDB5346464635
:108290009F430FE0194A1A4B2800210000F024FCEC
:1082A0000022002300F066FA002803D0002C04DB33
:1082B0000027002638003100C1E764006408254328
:1082C0000027002DF6D0104EF4E74B46142B0BD0B0
:1082D0003422D21A012393405D19BD4208D20123F2
:1082E0009C462F00E044D1E7133B9C46E044CDE799
:1082F0002F00CBE701FCFFFFFFFF0F009C750088FC
:108300003CE4377EEDFBFFFF0000F0BF002070472C
:108310004B0070B55B0D14000A00002B1AD14B0006
:108320005B08034315D0234B002201F003FB224BD3
:108330009C422DDB0A004B005B0D363B1F4DE318C2
:10834000AB422ADC002B0DDD1D4C1B0522401A43DD
:10835000110070BD1B4DAB42F0D102000B0000F0CC
:10836000C3FBF6E71D00353519DA174B02009C42B6
:1083700009DD0B001548164900F032F8134A144B7A
:1083800001F0D8FAE5E70B001248134900F028F88D
:10839000104A114B01F0CEFADBE70200E9E7084C86
:1083A000363322401B051343190000220B4B01F00A
:1083B000C1FACEE700005043B03CFFFFFE070000CB
:1083C000FFFF0F80FF07000050C300009C7500886E
:1083D0003CE4377E59F3F8C21F6EA5010000903CC3
:1083E00030B54A00DB0FDB0752081A43110030BDDD
:1083F00002B4714649084900095C49008E4402BC38
:108400007047C04603B47146490840004900095A04
:1084100049008E4403BC7047002243088B4274D34A
:1084200003098B425FD3030A8B4244D3030B8B4275
:1084300028D3030C8B420DD3FF22090212BA030C7E
:108440008B4202D31212090265D0030B8B4219D35F
:1084500000E0090AC30B8B4201D3CB03C01A52417F
:10846000830B8B4201D38B03C01A5241430B8B42C7
:1084700001D34B03C01A5241030B8B4201D30B03B0
:10848000C01A5241C30A8B4201D3CB02C01A5241D7
:10849000830A8B4201D38B02C01A5241430A8B429A
:1084A00001D34B02C01A5241030A8B4201D30B0283
:1084B000C01A5241CDD2C3098B4201D3CB01C01A9D
:1084C000524183098B4201D38B01C01A52414309A7
:1084D0008B4201D34B01C01A524103098B4201D395
:1084E0000B01C01A5241C3088B4201D3CB00C01A02
:1084F000524183088B4201D38B00C01A524143087A
:108500008B4201D34B00C01A5241411A00D201469E
:10851000524110467047FFE701B5002000F0F0F827
:1085200002BDC0460029F7D076E7704703460B43EB
:108530007FD4002243088B4274D303098B425FD35C
:10854000030A8B4244D3030B8B4228D3030C8B4288
:108550000DD3FF22090212BA030C8B4202D312126E
:10856000090265D0030B8B4219D300E0090AC30B43
:108570008B4201D3CB03C01A5241830B8B4201D3F0
:108580008B03C01A5241430B8B4201D34B03C01AD9
:108590005241030B8B4201D30B03C01A5241C30A51
:1085A0008B4201D3CB02C01A5241830A8B4201D3C2
:1085B0008B02C01A5241430A8B4201D34B02C01AAC
:1085C0005241030A8B4201D30B02C01A5241CDD251
:1085D000C3098B4201D3CB01C01A524183098B429C
:1085E00001D38B01C01A524143098B4201D34B0185
:1085F000C01A524103098B4201D30B01C01A5241E8
:10860000C3088B4201D3CB00C01A524183088B426E
:1086100001D38B00C01A524143088B4201D34B0057
:10862000C01A5241411A00D20146524110467047C9
:108630005DE0CA0F00D04942031000D340425340CE
:1086400000229C4603098B422DD3030A8B4212D38E
:10865000FC22890112BA030A8B420CD389019211C0
:108660008B4208D3890192118B4204D389013AD0FD
:10867000921100E08909C3098B4201D3CB01C01AD2
:10868000524183098B4201D38B01C01A52414309E5
:108690008B4201D34B01C01A524103098B4201D3D3
:1086A0000B01C01A5241C3088B4201D3CB00C01A40
:1086B000524183088B4201D38B00C01A5241D9D258
:1086C00043088B4201D34B00C01A5241411A00D2D9
:1086D0000146634652415B10104601D34042002BD5
:1086E00000D54942704763465B1000D3404201B554
:1086F000002000F005F802BD0029F8D016E7704709
:108700007047C046D0400B1C1141203A03D49C4610
:108710001341184363465242934018437047C04682
:108720008446101C62468C46191C634600E0C04615
:108730001FB501F097F8002801D40021C8421FBDE1
:1087400010B500F0EFFF4042013010BD10B501F050
:1087500089F8002801DB002010BD012010BDC046B3
:1087600010B501F07FF8002801DD002010BD0120C8
:1087700010BDC04610B501F011F8002801DC002042
:1087800010BD012010BDC04610B501F007F800284B
:1087900001DA002010BD012010BDC046F0B5CE4664
:1087A000474615042D0C2E0080B50704140C3F0C11
:1087B0009946030C7E435D43674363437F19340C42
:1087C000E4199C46A54203D980235B029846C44421
:1087D0004B4643435143250C36046544360C240470
:1087E000A4195B19591820000CBC90469946F0BD9D
:1087F000F0B54E4657464546DE46E0B543025B0AB5
:10880000450083B00F1C99462D0EC60F002D57D082
:10881000FF2D24D08020DB00C004184300238146B4
:108820009A469B467F3D7C027A00FB0F640A120E3B
:10883000984623D0FF2A4BD0E30080240020E40494
:108840007F3A1C43AD186B1C474601935346774053
:108850003A000F2B48D87D499B00CB589F46002BF0
:1088600000D085E008339A46063B9B467C027A009E
:10887000FB0FFF25640A120E9846DBD1002C00D0B6
:1088800090E0524601231A4392460120DBE74C4612
:1088900058461700022824D0032800D1CFE0002238
:1088A000002301284DD15802D205400AFF0710438A
:1088B000384303B03CBC90469946A246AB46F0BD57
:1088C000002B5BD104239A46033B00259B46AAE775
:1088D000FF35002C60D1524602231A4392460220F3
:1088E000B1E7FF220023DEE74B461B0C9C464B46BC
:1088F0002604360C180461463300220C6446000C32
:1089000043434E435043544380191A0C1218964265
:1089100003D9802149028C4664441B041B0C1004BB
:10892000C01883015E1EB341800E1843130C1B193F
:108930009B0103431C00230179D5012362081C40DD
:108940001443019A7F32002A4DDD630704D00F23C0
:108950002340042B00D00434230103D53C4B019A5F
:108960001C408032FE2ABCDCA3015B0AD2B29AE72B
:108970000C239A46093BFF259B4654E7180001F05B
:1089800071FE4A46431F76259A4000236D42914668
:108990002D1A9A469B4646E7524603231A439246AF
:1089A000032050E7200001F05DFE431F2D1A9C407C
:1089B000763D002047E780230027DB03FF2272E794
:1089C000424666E74C463200584662E780234A46F4
:1089D000DB031A4222D01C4220D123435B025B0AF4
:1089E0004746FF225FE701239A1A1B2A21DC230056
:1089F0000199D3409E318C401A0023005C1EA34194
:108A000013435A0704D00F221A40042A00D004331B
:108A10005A0111D49B015B0A002244E780234A4695
:108A2000DB0313435B025B0A3700FF223BE7019540
:108A300087E70022002336E70122002333E7802363
:108A4000DB0323435B025B0AFF222CE7B0D100006B
:108A5000FFFFFFF770B500283DD0C317C5185D4074
:108A6000C40F280001F0FEFD9E22121A962A07DC90
:108A7000D2B2082833DD083885406802400A23E076
:108A8000992A0BDD052329001B1AD94003001B334B
:108A90009D402B005D1EAB4119430D00052801DDF3
:108AA000431F9D402B000F490B406E0709D00F2636
:108AB0003540042D05D004335D0102D59F220B40C3
:108AC000121A9B01580AD2B24002D205400AE407AA
:108AD0001043204370BD002400220020F4E7680208
:108AE000400AF1E7FFFFFFFBF0B54F464646D6468A
:108AF0000C000903C0B5490A470F5E0039431F0344
:108B0000DB0F9C4665007B0A570F1F436D0DE40F7A
:108B1000760DA146C000B846D200AB1B64457BD0A1
:108B2000002B5FDD002E00D0A4E03E00164300D1F4
:108B300012E15E1E002E00D09EE1871A4346B84225
:108B400080410125C91A4042091A0B0200D431E1C3
:108B500049024E0A002E00D16EE1300001F082FD84
:108B60000300083B1F2B00DD61E120223900D21AEF
:108B70009E40D1409F400E439D4200DD51E15D1B70
:108B80006B1C1F2B00DD7CE12021C91A3D00300049
:108B90008F408840DD40791E8F41310007222843F5
:108BA000D940002507433A40002A09D00F233B4013
:108BB000042B05D03B1DBB42BF417F42C9191F009A
:108BC0000B0200D426E26A1CC64B55056D0D9A4275
:108BD00000D106E1C44AFF080A40530752023B4352
:108BE000120B8EE0002B00D0B8E06B1C5B055B0D18
:108BF000012B00DC30E1871A4346B842B641CB1A5C
:108C000076429E1B330200D54CE13B003343A1D199
:108C100000220024002570E0002B00DCE5E0002E9F
:108C200000D183E0AF4EB54260D080263604374392
:108C3000B846382B00DC3EE1434613431F007A1E42
:108C400097413F1887428041404209180B0200D4E7
:108C5000B0E0A44B01359D4200D1C3E0A24A7B089D
:108C60000A4001210F401F435108D30707221F4329
:108C70003A4099E79B4EB54238D0802636043743B8
:108C8000B846382B00DDDCE01F2B00DC30E11E0095
:108C90004746203EF740BC46202B04D04026F31A1E
:108CA00046469E403243170063467A1E97411F4353
:108CB000CCE0002B00D104E24346134300D159E13C
:108CC0004B07C00818438023C9081B03194208D06A
:108CD0004546ED081D4204D14346D00859070843D4
:108CE0002900420FC9007F4D1143C0004B07CA083D
:108CF0007C49C00803438D4268D012036D05120BF6
:108D00006D0D002112031800130B0A0D12051A43F2
:108D1000764B2D0513402B435B00E4075B08234390
:108D200019001CBC90469946A246F0BD3E00164371
:108D300012D05E1E002E00D000E1871887428041CD
:108D400041444042091801250B0233D5022585E72D
:108D500064463300414610001D00C7E7002D00D0D7
:108D6000DAE00C000443F3D05C1C00D19FE15D4CC1
:108D7000A64200D12FE1DB43382B00DD66E11F2B3B
:108D800000DD83E120240500E41A0F00DD40D94016
:108D9000A0404346A7405B1A441EA04198462F437B
:108DA0003843171ABA42924143465242991A6446CE
:108DB0003500CAE607223A40002A00D0F6E64B0703
:108DC000CA084849FF083B438D4296D11900114318
:108DD00000D19EE1802109030A431203120B414D89
:108DE0008FE71500002200238BE7002B00D0C7E09F
:108DF0006B1C5F057F0D012F00DCF1E0394DAB42AC
:108E000000D1B9E085180A008542894142444942AF
:108E100051180722CF076D082F4349083A401D001B
:108E2000C2E607223049ED1A31403A40BCE63E0026
:108E30002838864000279FE6380001F013FC2030D8
:108E40008EE6434613431F007A1E9741C71BB84264
:108E500080414042091A78E60E003B000643134366
:108E6000002D61D1002E00D0F4E0002B00D11BE1D9
:108E700064463900100039E71A4FBB427AD03300FC
:108E8000FFE630001F3DE840202B03D04021CB1AE5
:108E90009E4037437B1E9F41072207433A400021F3
:108EA000002589E7171A4346BA42B641591A764255
:108EB0008E1B64464EE61F2B00DDADE020264746A4
:108EC000F61AB740B9461700B246DF404E463E4359
:108ED00037005646B240561EB24117434246DA406A
:108EE0008918AEE6FF070000FFFF7FFFFFFF0F803E
:108EF00020264746F61AB740B9461700B246DF406B
:108F00004E463E4337005646B240561EB2411743C6
:108F10004246DA40891A99E77F4CA6425BD080240A
:108F200024045B42214327E7002E0CD1002B00D103
:108F3000CBE0644639001000774DD7E6764FBB4250
:108F400018D0330075E6002B14D04B07C008184327
:108F50008023C9081B03194207D0FC081C4204D116
:108F60007907D0080843E14621004C46420FC9006A
:108F70001143C000684DB9E61D0000220023C0E681
:108F8000002D5BD10D00054300D1E2E65D1C00D150
:108F9000B0E0614DAE421FD0DB43382B71DC1F2B9C
:108FA00000DD96E020250F00ED1AAF40B94607001E
:108FB000AA46DF404D463D432F005546A840D940C4
:108FC000451EA84188440743BF1897429241514229
:108FD000414435003AE6644635004146100085E6D6
:108FE0000B000343002D00D063E6002BF5D0434671
:108FF000134300D17AE68718874280410722414413
:10900000404209183A400B0200D4D5E6434B0135E3
:109010001940C9E5380069E61E004746203EF74082
:10902000BC46202B04D04026F31A46469E403243CD
:10903000170063467A1E97411F4302E6364DAE4243
:10904000CAD080252D045B422943A6E70843411E70
:109050008841A6E6002B00D148E6871A4346B8426D
:10906000B641CB1A76429E1B33024BD5171A4346A4
:10907000BA429241591A5242891A072264463A402A
:1090800092E501430F00791E8F419DE71C000F0000
:10909000203CE740202B03D04024E31A99400843AA
:1090A000411E884138437CE60022002425E6171A39
:1090B0004346BA429241591A5242891A64463500CF
:1090C00043E541461000144D10E6802200241203AF
:1090D00080E61D000F00203DEF40BC46202B03D052
:1090E0004025EB1A9940084307006346781E8741E4
:1090F0001F4369E7871897429B4141445B42C91867
:109100003500A3E53B003343CED0072231003A407F
:1091100052E600231A00F4E5FF070000FFFF7FFF7F
:10912000F0B55746DE464E464546E0B58346070055
:109130000E03480085B092461C00360B400DCD0F43
:10914000002800D19DE0954B984239D08023F6004D
:109150001B041E43924A7B0F3343994694460300F7
:109160006344009300230026FF00029323031B0B9C
:1091700098466300E40F52465B0D019400D1B3E0C2
:1091800086498B4200D19EE04246D10080221204E3
:109190000A435146490F11438B46814952468C463A
:1091A00000996344CB1A0021D20000932B00634046
:1091B0009A460F2E00D905E17A4BB6009B599F467F
:1091C0005B463343994600D0B8E0022308260027C7
:1091D00000900293CAE7CB463A0002990195019BA1
:1091E0009A46022927D0032900D180E2012944D0E0
:1091F0006D49009B8C4663441C00002C38DD5307EE
:1092000000D013E2D2085B46DB0109D55946674B13
:1092100019408B468021C9008C46009B63441C008A
:10922000634B9C4207DC5B4664055F075B021743A8
:109230001B0B620D02E000230027584A00211B038C
:109240001C0B0B0D1B05234314055A4A3800134011
:109250001C4353466400DB0764081C43210005B02F
:109260003CBC90469946A246AB46F0BD0122524214
:1092700001231B1B382B00DCADE10022002300275B
:10928000DCE75B46334399465ED0002E00D18AE18D
:10929000300001F0E7F903000B3B1C2B00DD7BE104
:1092A0001D22D31A5A460100DA4008398E401300B5
:1092B0005F46334399468F403F4B00261B1A00936D
:1092C0000023029352E7414653460B433B499B46DA
:1092D0008C46009B634400935B46002B3BD10223EA
:1092E00000221E43022161E7434613439B4637D0C9
:1092F0004346002B00D162E1404601F0B3F9030080
:109300000B3B1C2B00DD53E102004146083A914023
:1093100088461D21CB1A5146D9400B0041460B43CC
:109320009B46534693401A00009B25499C46604447
:1093300003008C4663440093002137E70323B146C2
:1093400000900C26029311E70023009301330426BA
:10935000002702930AE70323C3461E43032125E7A0
:1093600001331E430022012120E700239A46802377
:1093700000271B03094A61E7802349461B03194262
:1093800000D1E2E05946194200D0DEE00B431B0356
:1093900017001B0BA246014A50E7C046FF0700001A
:1093A00001FCFFFFF0D10000FF030000FFFFFFFE04
:1093B000FE070000FFFF0F800DFCFFFF01F8FFFF1D
:1093C000F3030000D94500D9CBE000D1C6E03C0052
:1093D00048460027009B013B00935B46160E1B028C
:1093E0001E431302984633041B0C9946310C01911D
:1093F000FFF798F84A4642430B04210C0500194335
:109400008A4207D98919013D8E4203D88A4201D97F
:10941000851E8919881A0199FFF784F809048C467A
:109420004A46210464464243090C030021438A4210
:1094300004D98919013B8E4200D8F1E02D041D4367
:10944000AB464346891A4246280C12041D0C5B4663
:10945000140C22001B041B0C5A4303946B4344431B
:10946000029568431B19150CEB189C4203D9802404
:109470006402A44660441C0C15041B042D0C201827
:109480005D19814277D373D00C1AA24A7D1BAF427B
:10949000BF419446009B7F426344E01B1C00864210
:1094A00000D1DBE00199FFF73DF84A4642430B0447
:1094B000290C070019438A4207D98919013F8E42B6
:1094C00003D88A4201D9871E8919881A0199FFF7A2
:1094D00029F809044A46894629044D464243090CA5
:1094E000030029438A4207D98919013B8E4203D8D8
:1094F0008A4201D9831E89193F04891A3A00039FC1
:109500001A43380013041B0C584381460298150C6B
:109510006F43434345434846000C8446DB1963448C
:109520009F4203D9802040028446654448461F0C70
:1095300000041B04000C7D191818A94200D284E015
:1095400000D17FE001231A4357E680234A461B03DC
:1095500013431B031B0BAA466F4A6FE6BA4200D99E
:1095600035E74B46DC0758087B081C43FF0734E708
:109570000024AF4289D247444745A4415B46644238
:10958000A4196418013BA6421ED2A0426DD800D196
:10959000B6E0241A9B4678E703005A46283B9A40D7
:1095A0000027914688E6584601F05CF8203072E6C4
:1095B00003005246283B9A4093460022B4E65046A8
:1095C00001F050F820309AE6A642E2D1B845DCD945
:1095D000341A9B4659E71F2B65DC504C0099A44672
:1095E0005C46614408008C4011008240D940501E06
:1095F00082410C4314435A46DA401300620709D0F3
:109600000F222240042A05D02200141D94428941D1
:1096100049425B181A0262D50122002300270DE699
:109620008A4200D80AE7831E891907E70F231340EF
:10963000042B00D1E6E5171D9742924153429B440B
:10964000FA08E0E5002800D1D7E57118531EB142B1
:1096500027D3A94215D358D01A0073E7002B00DC9A
:1096600004E6012300229B44CDE5022347444745FD
:1096700089415B429C46494289190C19E344241AEA
:1096800003E743465F0047459B41B8465B429E194E
:10969000023A8919A94200D054E7404500D051E769
:1096A000ABE51A00F6E71F215F4649420C1BE74075
:1096B000202B07D01A49009B8C46634418005B4658
:1096C00083401A43501E82413A4307270023174024
:1096D00009D00F21002311401400042995D1220044
:1096E0005F075B021B0BD20817430022A6E580230D
:1096F00059461B030B431B0317001B0B064A9DE532
:10970000BD42B2D89B460024BFE68045B9D31A00BB
:10971000C3E7C046FF030000FF0700001E0400006F
:109720003E040000F0B54F464646D6468446C0B5D6
:109730008046194E18030F034D00000B5C00824653
:109740003F0B6D0DC90F9146640DDB0F0120B54233
:109750000AD0B44203D0A54201D157450CD01CBC5D
:1097600090469946A246F0BD66463E43F7D1AC42CC
:10977000F5D154461443F2D10120C845EFD19942A6
:1097800007D0002DEBD163461F433800471EB84178
:10979000E5E70020E3E7C046FF070000F0B54F46CD
:1097A0004646D6464D00C0B50E03C90F8A462C4921
:1097B0001F035C008046360B6D0D91463F0B640D18
:1097C000DB0F8D421ED08C4216D0002D1ED13043AF
:1097D0008446002C01D13A4323D06246002A1AD095
:1097E0009A4529D0514602200139084001381CBC55
:1097F00090469946A246F0BD39001143E5D00220BB
:109800004042F4E73043FAD1AC420FD0002C0FD1E4
:109810003A43E7D00CE00122013B934318000130AA
:10982000E5E763460020002BE1D0DBE73A43E6D1D1
:109830009A45D7D1A542D5DCA54205DBBE42D1D899
:1098400008D00020BE42D2D25046012301389843AE
:109850000130CCE7C845C5D80020C845F4D3C6E7D9
:10986000FF070000F0B54F464646D6464D00C0B54E
:109870000E03C90F8A462E491F035C008046360B33
:109880006D0D91463F0B640DDB0F8D4218D08C425D
:1098900011D0002D18D130438446002C1ED13A43FC
:1098A0001CD163460020002B30D0514602200139E4
:1098B000084001382AE039001143EAD0022025E0AF
:1098C0003043FBD1AC4226D0002C26D13A4324D1E0
:1098D0005146022001390840013817E06246002A4B
:1098E0000FD09A45E1D1A54205DBBE42DDD819D0A3
:1098F0000020BE420AD2504601230138984301306D
:1099000004E00122013B9343180001301CBC904647
:109910009946A246F0BD3A43D0D19A45C5D1A54259
:10992000C3DCE0E7C845C0D80020C845E3D3EDE775
:10993000FF070000F0B55746DE464E464546E0B507
:10994000834606000F03480087B092461D003F0B78
:10995000400DCC0F002800D16FE0DE4B984238D08C
:109960008023FF001B041F43730F3B430193DA4B1B
:109970000027994600239B46F60081442B0369008B
:109980001B0B52469846490DED0F002900D185E08A
:10999000D04B994200D173E04346DA0080231B0488
:1099A00013435246CC48520F84461343524600207C
:1099B0006144D20089442100694000918C46012114
:1099C00049448A460F2F00D990E0C449BF00CF59BF
:1099D000BF465B463B43019300D06AE10223082760
:1099E000002681469B46C9E732005846019B6146E6
:1099F0000091022800D175E0032800D1FEE1012882
:109A000000D02CE100230027002600253F032A0D6B
:109A10003F0BB34812053A4302401B051343009A1B
:109A20005B00D1075B080B433000190007B03CBC5A
:109A300090469946A246AB46F0BD5B463B43019338
:109A400000D12FE1002F00D1A5E1380000F00AFE7F
:109A500003000B3B1C2B00DD96E11D22D31A5A4656
:109A60000100DA405E4608398F4013008E403B43C8
:109A700001939C4B00271B1A994600239B467DE7C8
:109A8000414653460B4393498C46E144002B00D09A
:109A90001AE102220220174300228CE7134300D16F
:109AA0000DE14346002B00D181E1404600F0DAFD94
:109AB00002000B3A1C2A00DD72E10100434608391E
:109AC0008B4098461D239A1A5346D3401A004346AA
:109AD000134352468A404946081A824989468144BE
:109AE000002068E77B4B002700268EE7140C120449
:109AF000120C1100370C3604350C794328008C46C3
:109B00002E0060436044834656432100300C80465B
:109B10005846794340440291844506D988468021BD
:109B200049028C46E044414602913604010C360C51
:109B300000048B4681191E0C1B041B0C0391190099
:109B400079438C46280075436544A8465843050C64
:109B500045447743A94203D9802149028C46674492
:109B6000290C8C4639000004000C2D042D1861448A
:109B7000AB4405915946049101990F043F0C080C20
:109B8000390051434243904602008C46090C8B46F3
:109B900062437C4344445C44A04503D9802149028C
:109BA00088464244210C884661460904090C8C46CB
:109BB00039005943434370437E430F0CF618240485
:109BC000BE19644442448C46B34203D980235B02ED
:109BD00098464044029B61469846049B37044344A0
:109BE0009B46AB45AD416B420D0405992D0C8C464F
:109BF0007F196744FD18A8465D462D19A542A4416A
:109C000093466442A446C344DC448F42BF41984516
:109C10009B4193459241A445A4415B427F421F432F
:109C2000360C52426442BF192243BF1862463818AC
:109C30004302D20D039913436A020A43501E824124
:109C40006146ED0D2A434E023243D90100D4B3E000
:109C50000126500832400243DE0732435B08224CA3
:109C60005444002C62DD510709D00F201040042815
:109C700005D0101D9042924152429B180200D9011A
:109C800004D580241948E400034054441848844211
:109C900000DD27E75E075B02D2081F0B6305164352
:109CA0005B0DB2E6002399460133042700269B464C
:109CB00064E60323019781460C279B465EE601225A
:109CC00001201743002276E6032303201F43434667
:109CD00071E6C046FF07000001FCFFFF30D2000024
:109CE000FFFF0F800DFCFFFFFF030000FFFFFFFEE3
:109CF000FE0700000023802700933F030026434B0C
:109D000083E6019B3200A446584670E6AC466EE6F8
:109D1000802701993F0339422DD03B422BD11F436D
:109D20003F033F0B00951600384B6EE601252D1BB7
:109D3000382D00DD66E61F2D40DC35481C00504400
:109D4000160082408440EE40501E8241344314434A
:109D5000EB40620709D00F222240042A05D02200DE
:109D6000141D9442804140421B181A023ED5012323
:109D70000027002649E68027019B3F031F433F033E
:109D80003F0B0094214B40E603005A46283B9A4083
:109D9000002601926DE6584600F064FC203057E63C
:109DA00003005246283B9A401300002293E6504697
:109DB00000F058FC20307BE6CA4650E71F201E000A
:109DC0004042041BE640202D03D0124C5444A340D3
:109DD0001A43501E8241324307260027164009D0FD
:109DE0000F200023104014000428B9D122005E0780
:109DF0005B021F0BD2081643002306E680273F03B1
:109E00001F433F033F0B1600004BFEE5FF0700001A
:109E10001E0400003E040000F8B557464E46454675
:109E2000DE460C000903E0B5490A460F5F003143E6
:109E30001E03DB0F760A9B46530F3343C84E650063
:109E4000C000E40FD2006D0DA24681467F0D9C46F6
:109E50009046B74200D1B9E05B46012673409B466D
:109E6000EE1BA34500D183E0002E63DD002F00D060
:109E7000B1E06346134300D123E1731E002B00D0F1
:109E8000BAE1861A6346B04280410125C91A4042B0
:109E9000091A0B0200D447E149024B0A984643468F
:109EA000002B00D189E1404600F0DCFB0300083BB9
:109EB0001F2B00DD7CE120223000D21A4146D04029
:109EC000994002009E400A439D4200DD6AE15D1B0D
:109ED0006B1C1F2B00DD94E1202110003500C91AF6
:109EE0008E40DA408840DD40711E8E41110007220D
:109EF0002843002506433240002A09D00F2333406F
:109F0000042B05D0331DB342B641764289191E0099
:109F10000B0200D43DE26A1C914B55056D0D9A422F
:109F200000D119E18F4AF6080A4057075202374319
:109F3000120B9BE0002E00D0C5E06E1C7605760D5E
:109F4000012E00DC48E16746861ACB1BB042BF41B8
:109F50007F42B8461F004346FF1A3B00B8461B022B
:109F600000D55FE137439AD100220024002579E033
:109F7000002E00DCFAE0002F00D18DE0784B9D42EE
:109F800067D0802367461B041F43BC46382E00DC85
:109F900052E1634613435A1E93411E188642804184
:109FA000404209180B0200D4BEE06D4B01359D42C2
:109FB00000D1D2E06B4A73080A4001210E401E43D3
:109FC0005108D30707221E43324095E71E0016436F
:109FD00000D045E740E7624B9D423AD08023674678
:109FE0001B041F43BC46382E00DDEBE01F2E00DCB7
:109FF0003AE133006746203BDF403B00202E05D08E
:10A000004027BF1B6646BE40324390464646721EFE
:10A0100096413343DAE0002B00D114E26346134348
:10A0200000D168E180234E07C008C9081B0306431E
:10A03000194208D06046C008184204D163460100A6
:10A04000D2085E071643F3009946C900720F444DCB
:10A0500011434B46DE08424B4F073743CA089D4227
:10A0600000D16EE012036D05120B6D0D002112037D
:10A07000130B0A0D12051A433B4B2D0513402B43BE
:10A080005B00E4075B082343380019003CBC9046A2
:10A090009946A246AB46F8BD6346134311D0731EE2
:10A0A000002B00D007E1861886428041614440427F
:10A0B000091801250B0237D502257BE73E006146D2
:10A0C00091463500C5E75C46002D00D0E1E00B006D
:10A0D0000343F3D0731C00D1ACE1214B9F4200D16C
:10A0E0003AE1F343382B00DD6FE11F2B00DD8CE1FB
:10A0F00020250E00ED1AAE40B0460600AA46DE400E
:10A10000454635432E005546D940A8406346451E76
:10A11000A8415B1A9C463043161AB24292416346EC
:10A120005242991A3D00B4E607223240002A00D07C
:10A13000E4E60B4BF6084F073743CA089D4200D0B0
:10A1400090E73B00134300D1A6E180231B031A4391
:10A150001203120B024D89E715000022002785E744
:10A16000FF070000FFFF7FFFFFFF0F80002E00D0E2
:10A17000C7E06B1C5E05760D012E00DCF0E0C84DDB
:10A18000AB4200D1B9E085180A008542894162449A
:10A19000494251180722CE076D082E434908324024
:10A1A0001D00A9E6BF49ED1A114007223240A3E67F
:10A1B000320028388240002686E6300000F052FA4D
:10A1C000203073E6634613435A1E9341C61AB042C9
:10A1D00080414042091A5CE60E0067460643174379
:10A1E000002D5ED1002E00D0F3E0002F00D11EE143
:10A1F0005C46614691462CE7A94FBE427BD01E00CB
:10A20000F1E610001F3DE840202B03D04021CB1A7F
:10A210009A401643731E9E41072206433240002196
:10A22000002583E7161A6346B2428041591A40421C
:10A230000B1A98465C4632E61F2E00DDABE0202765
:10A24000BB1B9A4663465746BB40994613004F4690
:10A25000F3401F433B005746BA40571EBA411343D1
:10A260006246F240891898E62027BB1B9A4663464F
:10A270005746BB40994613004F46F3401F433B00EF
:10A280005746BA40571EBA4113436246F240891AF4
:10A290009CE7834B9F425FD080252D047342294366
:10A2A00020E7002E0CD1002F00D1D0E05C466146A3
:10A2B00091467B4DCDE67A4FBE421CD01E0065E62E
:10A2C000002F18D0C0084E0706438020C90800039D
:10A2D000014208D06346DC08044204D12100DA467A
:10A2E000D2085E071643F300994601245346C9007D
:10A2F000720F11431C406A4DABE61D00002200277F
:10A30000B4E6002D59D10B00034300D1D6E6731CEF
:10A3100000D1B2E0624B9F421ED0F343382B6FDC7A
:10A320001F2B00DD97E020250E00ED1AAE40B04651
:10A330000600AA46DE40454635432E005546A84055
:10A34000D940451EA8418C440643B6189642924116
:10A35000514261443D0025E63D006146914678E664
:10A360000B000343002D00D055E6002BF5D06346CB
:10A37000134300D16DE68618864280416144404215
:10A38000091800220B0200D4D0E6464B01351940D3
:10A39000B2E5B1465DE633006746203BDF403B0057
:10A3A000202E05D04027BF1B6646BE403243904654
:10A3B0004646721E96413343EFE5394B9F42CBD060
:10A3C00080252D0473422943A8E70843411E884194
:10A3D000A2E6002F00D13CE66346861ACF1AB042AF
:10A3E0009B415B42FB1A98461B024ED5161A6346E8
:10A3F000B2429241591A5242891A5C4600227BE5C8
:10A4000001430E00711E8E419FE71D000E00203D8E
:10A41000EE40B046202B04D04025EB1A994008436B
:10A42000814648464346411E8841184374E600224F
:10A43000002417E6161A6346B2429241591A524254
:10A44000891A3D0025E561469146154D01E68022B9
:10A450000024120379E61D000E00203DEE40B046B8
:10A46000202B04D04025EB1A9940084381464E46E4
:10A470004346711E8E411E4367E7861896429B41F4
:10A4800061445B42C9183D008CE547463743CED056
:10A4900007224146324049E600273A00E6E5C04639
:10A4A000FF070000FFFF7FFF70B50C4E0D031C037C
:10A4B00049005B002D0B490D240B5B0DB14208D008
:10A4C000064900208B4203D114432000441EA041C2
:10A4D00070BD05430120002DFAD1F1E7FF07000010
:10A4E00030B5144D0A034B00120B5B0DC90F00244D
:10A4F000AB4211DD104CA34210DC802464032243E4
:10A500000E4CE41A1F2C0CDD0D48C31ADA40130060
:10A510005C42002900D11C00200030BD094BCC1842
:10A52000FAE7094DE040AC4663449A401300034308
:10A53000EEE7C046FE0300001D04000033040000E7
:10A5400013040000FFFFFF7FEDFBFFFF70B5002845
:10A550002DD0C317C5185D40C40F280000F082F845
:10A56000154B1B1A5B055B0D0A2815DD0B38854062
:10A5700000222D032D0B002110002D030A0D2D0BA1
:10A5800012052A430D4D1B052A4013435B00E407C7
:10A590005B082343190070BD020029001532914069
:10A5A0000A000B21081AC5402D032D0BE3E70024F8
:10A5B000002300250022DEE71E040000FFFF0F80BD
:10A5C0004100090E4B1C70B5DBB24602750AC40F80
:10A5D000012B14DDE0239B006D07360BCB18002107
:10A5E0000A0D280012051C4D32435B052A405B080A
:10A5F00013435B00E4075B082343190070BD002987
:10A6000014D1002D1ED0280000F02CF80A281CDCE4
:10A610000B232A001B1ADA40030015339D400F4B11
:10A6200012031B1A5B05160B5B0DD8E7002D06D035
:10A63000320B802636036D071643094BCFE7084BD4
:10A640000026CCE700230026C9E703002A000B3BC5
:10A650009A400025E3E7C046FFFF0F808903000012
:10A66000FF0700001C2101231B04984201D3000CAA
:10A6700010391B0A984201D3000A08391B09984275
:10A6800001D30009043902A2105C40187047C0468B
:10A6900004030202010101010000000000000000AB
:10A6A00030B51C00094B05001B6885B0D868084B05
:10A6B000002A01D1074B1A000292019300912B004E
:10A6C0002200054900F026F800F086FD80000020F9
:10A6D00070D2000063C100007DD20000014B1868F9
:10A6E0007047C04680000020084B10B50400002BC6
:10A6F00002D0002100E000BF054B1868836A002BE0
:10A7000000D09847200001F03DFBC046000000004B
:10A71000ACD200000EB403B5010003AB044804CB77
:10A720000068019300F076F802B008BC03B0184747
:10A730008000002070B500260C4D0D4C641BA41049
:10A74000A64209D1002601F01FFB0A4D0A4C641BEA
:10A75000A410A64205D170BDB300EB58984701364E
:10A76000EEE7B300EB5898470136F2E750020020BD
:10A77000500200205002002060020020002310B58B
:10A780009A4200D110BDCC5CC4540133F8E710B537
:10A79000884202D98B18984203D3002307E08B5CD0
:10A7A0008354013AFBD210BDCC5CC45401339A42AD
:10A7B000FAD1F8E703001218934200D170471970DC
:10A7C0000133F9E7936810B5013B9360002B04DA7D
:10A7D0009469A34207DB0A2905D01368581C10604E
:10A7E0001970080010BD00F02BFC0100F9E7F8B566
:10A7F00006000F001400D518AC4201D1002007E07C
:10A8000021783A003000FFF7DDFF0134431CF3D11B
:10A81000F8BD0000F0B59FB002900F001600059340
:10A82000002805D083690493002B01D100F0D4FDEA
:10A830007B4B9F425BD1029B5F68BB891B0762D544
:10A840003B69002B5FD0002306AC63612033637645
:10A850001033A37635002B78002B01D0252B5CD14B
:10A86000AB1B04930CD0320039000298FFF7BFFFF6
:10A87000431C00D1C4E06269049B94466344636155
:10A880002B78002B00D1BBE00122002352426260F2
:10A8900002A9543252186E1C2360E360A360137047
:10A8A000A365317805225F4800F0B4FE751C0028CE
:10A8B00035D12268D30604D5532302A95B18202181
:10A8C0001970130704D5532302A95B182B211970A3
:10A8D00033782A2B2CD0350000210A20E3682A780F
:10A8E0006E1C303A092A64D900292ED026E04E4B3E
:10A8F0009F4202D1029B9F689FE74C4B9F429CD195
:10A90000029BDF6899E73900029800F0EFFB00280E
:10A9100099D0012040421FB0F0BD01359BE7414B6B
:10A920002268C01A01238340134323602E00B8E736
:10A93000059B191D1B680591002B01DB099304E0A1
:10A940005B42E3600223134323602B782E2B0AD152
:10A950006B782A2B35D1059B02351A1D1B68059291
:10A96000002B2BDB0793324E29780322300000F0B6
:10A9700051FE002806D04023801B83402268013509
:10A9800013432360297806222A486E1C217600F0A2
:10A9900041FE00283AD0284B002B25D10722059BE9
:10A9A00007339343083305936369039A9B186361E4
:10A9B00050E7434301219B18350090E701235B4298
:10A9C000D0E700230A201A000135636029786E1C45
:10A9D0003039092903D9002BC5D00792C3E7424378
:10A9E000012352183500F1E705AB00933A00134BF1
:10A9F0002100029800E000BF0390039B0133D3D1F4
:10AA0000BB895B0600D584E70B9884E705AB009310
:10AA10003A000A4B2100029800F080F8ECE7C046AB
:10AA200004D30000B0D2000024D30000E4D2000020
:10AA3000B6D20000BAD2000000000000EFA700006C
:10AA4000F7B5150001938A680B6900900C009342DA
:10AA500000DA130022002B6043321278002A01D062
:10AA600001332B6023689B0602D52B6802332B60D1
:10AA7000062723681F4027D0230043331B785A1E24
:10AA800093412268920630D4220001994332009803
:10AA9000089EB047431C25D0062320682A68E16839
:10AAA00003400025042B03D18D1AEB43DB171D4017
:10AAB000A3682269934201DD9B1AED180027BD426D
:10AAC00020D1002010E00137E3682A689B1ABB42BE
:10AAD000D2DD22000123193201990098089EB04767
:10AAE000431CF0D101204042FEBD3020E11843312B
:10AAF000087021005A1C45310978A21843320233EC
:10AB00001170C1E7220001231A3201990098089EB2
:10AB1000B047431CE6D00137D1E70000F0B589B05B
:10AB200004920A0043320593039002920A7E0C00BD
:10AB30000E9B6E2A00D186E01FD8632A33D008D836
:10AB4000002A00D18CE0582A4DD0250042352A70C9
:10AB500030E0642A01D0692AF7D1196825680A1DF6
:10AB6000280629D508681A60002803DA2D23029ADE
:10AB7000404213706B4E0A274FE0732A74D008D8F6
:10AB80006F2A1FD0702AE0D1202209680A43226070
:10AB900003E0752A16D0782AD7D1220078214532D1
:10ABA0001170614E22E025001A684235111D1960AE
:10ABB00013682B70012365E008681A606906D3D515
:10ABC00000B2D1E719682568081D186008682E06CC
:10ABD00005D5544E08276F2A1BD00A2719E06D06A9
:10ABE000F7D580B2F5E745314E4E0A7018682268F5
:10ABF000011D00681960150621D5D30702D5202351
:10AC00001A4322601027002803D1202322689A4388
:10AC100022602300002243331A706368A360002B74
:10AC200058DB0422216891432160002854D1029D01
:10AC3000002B5AD02500337842352B7055E055064D
:10AC4000DBD580B2D9E71A680D68101D4969186014
:10AC500013682E0601D5196002E06D06FBD5198038
:10AC60000023029D23614FE01A68111D19601568C9
:10AC700000216268280000F0CDFC002801D0401BB4
:10AC80006060636823610023029A13703CE02369CB
:10AC90002A0004990398059DA847431C3ED02368C9
:10ACA0009B0715D4079BE068984239DA180037E013
:10ACB00022000123193204990398059EB047431CD2
:10ACC0002CD00135E368079A9B1AAB42F0DCE9E728
:10ACD0000025F7E70028ADD0029D3900FDF722FCE2
:10ACE000735C013D2B700028F7D1082F09D1236830
:10ACF000DB0706D563682269934202DC3023013DFD
:10AD00002B70029B5B1B2361059B07AA009321000C
:10AD1000049B0398FFF794FE431CB8D101204042E6
:10AD200009B0F0BDC1D20000D2D200000D4B70B509
:10AD30001C680500A36B002B0FD1182000F04EFCFF
:10AD4000094BA0630360094B01224360084B8360F9
:10AD50000B2383810023026143610022A36B1D61E9
:10AD60005A6170BD800000200E33CDAB34126DE609
:10AD7000ECDE0500124B10B51C68A36B002B0FD145
:10AD8000182000F02BFC0F4BA06303600E4B012238
:10AD900043600E4B83600B23838100230261436178
:10ADA000A46B0B4A206961690A4BFDF7F7FC01228D
:10ADB000002380185941206161614800400810BD9E
:10ADC000800000200E33CDAB34126DE6ECDE0500C2
:10ADD0002D7F954C2DF451580CB430B5164B9DB0C9
:10ADE0000C1E1D6808DA8B2301202B6040421DB029
:10ADF00030BC08BC02B01847822302A99B008B819B
:10AE00000023029008619C4200D0631E8B604B615E
:10AE100001235B42CB81209A21AB2800019300F0F3
:10AE200035FD431C01DA8B232B60002CDFD000237F
:10AE3000029A1370DBE7C046800000200EB400B514
:10AE40000B499CB01DAB02900690079104910948F4
:10AE5000094904CB0591006802A9019300F016FD91
:10AE60000023029A13701CB008BC03B01847C046F8
:10AE7000FFFFFF7F800000200802FFFF020010B5E7
:10AE80001378541C002B05D1CC5CD4540133002C16
:10AE9000FAD110BD2200F3E702780B78002A03D024
:10AEA000013001319A42F7D0D01A70470023C25CBA
:10AEB0000133002AFBD1581E704730B50500002A27
:10AEC00000D130BD0C78013A6B1C2C700131002C84
:10AED00005D19A189A42F4D01C700133FAE71D008C
:10AEE000EDE710B50378002B0FD10B785A42534190
:10AEF0005B42184010BD0023CA5C002AFAD0C45C33
:10AF0000944201D10133F7E701300378002BF2D1ED
:10AF10001800EFE7F0B51F000E0087B00590019113
:10AF200002920C98347800F0EAFA0822001943786B
:10AF3000751C134036D12D2C36D1B51C74780126E2
:10AF4000002F62D0102F09D1302C07D120222B786E
:10AF50009343582B54D110276C7802352D4B390070
:10AF6000F31818000393FDF7DDFA04910121002383
:10AF7000494202008C4618002100303909291AD8AC
:10AF80000C00A74223DD591C09D06346824206D338
:10AF900002D10499A14202DB0123784320182C78C6
:10AFA0000135E9E72E00BCE72B2C01D01E00C7E7D6
:10AFB000B51C7478FAE721004139192901D8373CCA
:10AFC000DFE721006139192901D8573CD9E75A1C1C
:10AFD00008D1059A23331360029B0398002B09D1F3
:10AFE00007B0F0BD002E00D04042029A002AF7D0F0
:10AFF000002B01D06B1E0193029B019A1A60EFE7B0
:10B000003024002FAAD10827A8E7302C9ED00A2789
:10B01000A4E7C046FFFFFF7F37B51300064A0500CF
:10B020001068046A002C00D1044C0A000094290026
:10B03000FFF770FF3EBDC04680000020E400002006
:10B04000F8B505000E001400002804D08369002B19
:10B0500001D100F0C1F9224B9C422DD16C68A3694B
:10B06000A360A3891B0731D52369002B2ED0236849
:10B070002269F7B2981A6369F6B2834205DC2100AF
:10B08000280000F03BF9002826D1A3680130013BDD
:10B09000A36023685A1C22601F706369834204D036
:10B0A000A389DB071AD50A2E18D12100280000F049
:10B0B00025F9002812D00FE00A4B9C4201D1AC6860
:10B0C000CDE7094B9C42CAD1EC68C8E721002800B3
:10B0D00000F00CF80028CAD0012676423000F8BDF6
:10B0E00004D3000024D30000E4D20000364B70B536
:10B0F0001D6806000C00002D05D0AB69002B02D1A5
:10B10000280000F069F9314B9C420FD16C680C2388
:10B11000E25E93B219072DD4D90611D40923012078
:10B12000336037331343A381404270BD284B9C42A8
:10B1300001D1AC68EBE7274B9C42E8D1EC68E6E72D
:10B140005B0713D5616B002908D023004433994273
:10B1500002D0300000F06AFA002363632422A3893E
:10B160009343A38100236360236923600823A2899A
:10B170001343A3812369002B0BD1A0218022A38933
:10B18000890092000B40934203D02100300000F070
:10B19000E1F90123A289134011D00023A360636960
:10B1A0005B42A361002023698342BED10C23E25E8F
:10B1B0001306BAD540231343A3810138B5E792079C
:10B1C00000D46369A360EDE78000002004D3000091
:10B1D00024D30000E4D2000010B5062000F090FC5B
:10B1E000012000F0CFFD0000F7B58A8905000C00B2
:10B1F000130760D44B68002B04DC0B6C002B01DCC4
:10B200000020FEBDE76A002FFAD000232E682B60D5
:10B2100080235B01216A1A4034D0606DA3895B07EB
:10B2200006D56368C01A636B002B01D0236CC01A6B
:10B230000200216A00232800E76AB847A189431C5D
:10B2400006D12B681D2B30D82B4ADA40D3072CD5DA
:10B250000023636023692360CB0405D5431C02D11E
:10B260002B68002B00D16065616B2E600029C7D070
:10B2700023004433994202D0280000F0D7F900207F
:10B280006063BEE701232800B847431CC6D12B6882
:10B29000002BC3D01D2B01D0162B01D12E60AFE7A0
:10B2A0004023A2891343A381ABE740230B43012032
:10B2B000A3814042A5E70F69002FA1D00B680F6062
:10B2C000DB1B01930023920700D14B69A360019B14
:10B2D000002B00DC94E7019B3A00216A2800A66A53
:10B2E000B047002803DC4023A2891343DFE7019B1A
:10B2F0003F181B1A0193EAE7010040200B6970B563
:10B3000005000C00002B01D1002070BD002804D0E6
:10B310008369002B01D100F05FF80B4B9C4209D1EF
:10B320006C680C22A35E002BEED021002800FFF7F2
:10B330005BFFEAE7054B9C4201D1AC68F1E7044BA7
:10B340009C42EED1EC68ECE704D3000024D300006B
:10B35000E4D20000002310B5040003604360836062
:10B3600081814366C28103614361836119000822C0
:10B370005C30FFF71FFA054B24626362044BA36243
:10B38000044BE362044B236310BDC04641BB000085
:10B3900069BB0000A1BB0000CDBB000010B5024995
:10B3A00000F08CF810BDC046FDB2000070B56825F5
:10B3B0004A1E55430E002900743100F081F9041E25
:10B3C00008D000212A00016046600C30A06068327D
:10B3D000FFF7F0F9200070BD836913B50400002B5E
:10B3E00028D18364C3640365134B144A1B688262CB
:10B3F0000193984201D101238361200000F020F8DD
:10B400006060200000F01CF8A060200000F018F838
:10B410000022E06004216068FFF79CFF01220921FF
:10B42000A068FFF797FF02221221E068FFF792FF62
:10B430000123A36113BDC046ACD200009DB3000040
:10B44000F8B51C4B07001E68B369002B02D1300011
:10B45000FFF7C2FF4836B4687368013B04D5336810
:10B46000002B07D03668F6E70C22A55E002D0DD024
:10B470006834F2E704213800FFF798FF30600028B5
:10B48000F0D10C2304003B602000F8BD20000A4BE3
:10B49000656625606560A560E36025616561A561FD
:10B4A000082229005C30FFF785F96563A563A56470
:10B4B000E564E9E7ACD200000100FFFFF7B5040046
:10B4C0000700002601914834002C01D13000FEBD58
:10B4D0006368A5680093009B013B009301D5246835
:10B4E000F2E7AB89012B08D90E22AB5E013304D001
:10B4F00029003800019B984706436835EBE7EC309C
:10B500000068704770B50E001D000E23C95E96B02E
:10B510001400002907DA00232B60B3891B0611D41D
:10B520008023DB000FE06A4600F088FB0028F2DB96
:10B53000F022019B12021340054A9B185A425341C4
:10B540002B60EDE740230020236016B070BDC0469D
:10B5500000E0FFFFF7B502268B8905000C0033429F
:10B5600006D0230047332360236101236361F7BDC5
:10B5700001AB6A46FFF7C6FF00990700280000F0FC
:10B580009FF8002808D10C22A35E9A05EFD403226D
:10B5900093431E43A681E4E70F4BAB628023A2894D
:10B5A00020601343A381009B20616361019B002BFA
:10B5B0000DD00E23E15E280000F052FB002806D0DB
:10B5C0000322A38993431A0001231343A381A08973
:10B5D0003843A081CBE7C0469DB3000010B5034BB4
:10B5E0000100186800F06CF810BDC0468000002013
:10B5F00082B0002900D101A9101E06D0002B06D070
:10B6000013780B601078431E984102B070470220F7
:10B610004042FAE7C9B28218904201D10020704737
:10B6200003788B42FBD00130F6E7000070B50500CF
:10B63000002910D00C1F2368002B00DAE418280022
:10B6400000F034FB1D4A1368002B05D163601460C1
:10B65000280000F02CFB70BDA34209D921686018B6
:10B660008342F3D118685B6841182160EEE713004C
:10B670005A68002A01D0A242F9D919685818A04284
:10B680000BD120680918581819608242E0D110685F
:10B690005268411819605A60DAE7A04202D90C23B7
:10B6A0002B60D5E721686018824203D11068526888
:10B6B0004118216062605C60CAE7C0461C1C002023
:10B6C000032370B5CD1C9D43083506000C2D1ED2FA
:10B6D0000C25A9421DD8300000F0E8FA254A14686C
:10B6E0002100002919D1244C2368002B03D13000FC
:10B6F00000F0CAF920602900300000F0C5F9431CB1
:10B700002BD10C233000336000F0D1FA03E0002D80
:10B71000DFDA0C233360002070BD0B685B1B19D48B
:10B720000B2B03D90B60CC18256003E04B688C42CF
:10B730000DD11360300000F0BAFA200007220B3060
:10B74000231D9043C31AE7D05A42E250E4E76360F6
:10B750000C00EFE70C004968C3E70323C41C9C43BB
:10B76000A042E1D0211A300000F08EF9431CDBD159
:10B77000C7E7C0461C1C0020201C0020F8B50700AD
:10B780000D001600002905D11100FFF799FF0400F4
:10B790002000F8BD002A03D1FFF748FF3400F7E787
:10B7A00000F086FA2C00B042F2D231003800FFF7E8
:10B7B00087FF041EECD029003200FEF7DFFF2900CE
:10B7C0003800FFF733FFE3E7F0B58E6885B0070078
:10B7D0000C00039201939E423CD890238A89DB009F
:10B7E0001A4234D00325096923685B1A02936369FE
:10B7F00002985D43EB0F5D19019B6D1001331B181F
:10B80000AB4200D91D00530532D529003800FFF79F
:10B8100057FF061E09D10C233B6040230120A2895B
:10B8200040421343A38105B0F0BD029A2169FEF79F
:10B83000A5FFA389144A1A4080231343A381029BC6
:10B840002661F61826606561019EED1AA560019BD0
:10B850009E4200D9019E320003992068FEF797FFAF
:10B86000A36800209B1BA36023689E192660DAE76B
:10B870002A003800FFF782FF061EE0D12169380058
:10B88000FFF7D4FEC7E7C0467FFBFFFFF0B59FB0D0
:10B89000029005938B890F0016001B0611D50B69CA
:10B8A000002B0ED14021FFF70BFF386038610028D4
:10B8B00005D10C23029A013813601FB0F0BD40235C
:10B8C0007B61002306AC6361203363761033A3767B
:10B8D00035002B78002B01D0252B46D1AB1B0493D0
:10B8E0000CD0320039000298FFF76EFF431C00D1E4
:10B8F000AEE06269049B9446634463612B78002B3D
:10B9000000D1A5E0012200235242626002A9543214
:10B9100052186E1C2360E360A3601370A365317836
:10B9200005225448FFF776FE751C00281FD12268B7
:10B93000D30604D5532302A95B18202119701307DD
:10B9400004D5532302A95B182B21197033782A2BB5
:10B9500016D0350000210A20E3682A786E1C303AA0
:10B96000092A4ED9002918D010E00135B1E7414B22
:10B970002268C01A01238340134323602E00CEE7C0
:10B98000059B191D1B680591002B01DB099304E041
:10B990005B42E3600223134323602B782E2B0AD1F2
:10B9A0006B782A2B35D1059B02351A1D1B68059231
:10B9B000002B2BDB0793304E297803223000FFF752
:10B9C00029FE002806D04023801B834022680135D1
:10B9D000134323602978062228486E1C2176FFF73E
:10B9E00019FE00283CD0264B002B25D10722059BB1
:10B9F00007339343083305936369039A9B18636184
:10BA000066E7434301219B183500A6E701235B420B
:10BA1000D0E700230A201A000135636029786E1CE4
:10BA20003039092903D9002BC5D00792C3E7424317
:10BA3000012352183500F1E705AB00933A00114B92
:10BA40002100029800E000BF0390039B0133D3D193
:10BA5000BB890B985B0600D42FE7012040422CE7FE
:10BA600005AB00933A00074B21000298FFF756F808
:10BA7000EAE7C046B0D20000B6D20000BAD2000059
:10BA800000000000C9B70000002370B5064C050097
:10BA90000800236000F060F9431C03D12368002BE9
:10BAA00000D02B6070BDC046982F002070B50400F8
:10BAB0000D001F2904D9162303600120404270BDE8
:10BAC000436C002B04D08A009B181A68002A08D106
:10BAD000200000F031F82A000100200000F01AF8E0
:10BAE000EDE70020012AEAD0511C03D116230130D2
:10BAF0002360E4E7002428001C6090472000DEE774
:10BB000010B5034B01001868FFF7D0FF10BDC04609
:10BB100080000020002370B5064C050008001100CD
:10BB2000236000F001F9431C03D12368002B00D0EF
:10BB30002B6070BD982F002010B500F0E5F810BD07
:10BB400070B50C000E25495F00F0BAF8002803DB41
:10BB5000636D1B18636570BDA389024A1340A381FE
:10BB6000F9E7C046FFEFFFFFF8B51F008B8905001E
:10BB70000C001600DB0505D50E23C95E002202234A
:10BB800000F080F8A389054A28001340A381320001
:10BB90000E23E15E3B0000F02BF8F8BDFFEFFFFF46
:10BBA00070B50C000E25495F00F06CF8A389421CAB
:10BBB00003D1054A1340A38170BD80225201134373
:10BBC000A3816065F8E7C046FFEFFFFF10B50E23C5
:10BBD000C95E00F021F810BD0B1E04D0FF2A04D965
:10BBE0008A2303608B3B180070470A700123FAE731
:10BBF00070B50500080011000022064C22601A00F2
:10BC000000F0B8F8431C03D12368002B00D02B6050
:10BC100070BDC046982F0020002370B5064C05006B
:10BC20000800236000F060F8431C03D12368002B58
:10BC300000D02B6070BDC046982F0020002370B547
:10BC4000064C050008001100236000F055F8431C65
:10BC500003D12368002B00D02B6070BD982F0020EB
:10BC6000002370B5064C05000800236000F054F86E
:10BC7000431C03D12368002B00D02B6070BDC0464D
:10BC8000982F002070B50500080011000022064C16
:10BC900022601A0000F050F8431C03D12368002BE7
:10BCA00000D02B6070BDC046982F002070477047B1
:10BCB0000B1F1B68181F002B01DA0B58C0187047A8
:10BCC00070B50500080011000022064C22601A0021
:10BCD00000F03AF8431C03D12368002B00D02B60FE
:10BCE00070BDC046982F002058220120014B4042D1
:10BCF0001A607047982F002058220120014B4042C3
:10BD00001A607047982F002058220120014B4042B2
:10BD10001A607047982F00205822024B00201A60AA
:10BD20007047C046982F002058220120014B404206
:10BD30001A607047982F002058220120014B404282
:10BD40001A607047982F002058220120014B404272
:10BD50001A607047982F0020044A1368002B00D106
:10BD6000034B1818106018007047C046241C0020B0
:10BD7000A02F002058220120014B40421A6070473A
:10BD8000982F0020FEE7C046F8B5C046F8BC08BCB6
:10BD90009E467047F8B5C046F8BC08BC9E46704742
:10BDA00064617461000000001CBE0000EB01000033
:10BDB00025BE0000170400002DBE0000290700006A
:10BDC00034BE00003908000039BE0000DF02000068
:10BDD00044BE00008304000049BE0000B109000019
:10BDE00055BE00001B0200005FBE000031060000CF
:10BDF0006DBE00009F05000072616E646F6D006192
:10BE00006C6C006C6173740066616C7365007472B5
:10BE1000756500252E3135732E2E2E006D616B65F4
:10BE20004C697374006164644C6173740064656C84
:10BE3000657465006A6F696E00636F707946726F32
:10BE40006D546F0066696E64006A6F696E53747238
:10BE5000696E677300756E69636F64654174007520
:10BE60006E69636F6465537472696E6700667265AC
:10BE7000654D656D6F727900C80F0000D80F000026
:10BE8000F20F000070100000A8100000DE1000008B
:10BE9000161100003C11000078110000BA110000DA
:10BEA0001012000054120000C0120000081300001D
:10BEB0002E13000066130000AC130000D213000024
:10BEC00000140000321400006A140000EE14000098
:10BED000B61500002C16000098160000EC160000A5
:10BEE0000C1700002E170000E017000026180000B5
:10BEF0009E180000C80F0000C80F0000CC180000FA
:10BF000034190000B8190000FE190000461A00009C
:10BF1000B81A00002A1B0000721B0000B81B0000AA
:10BF2000EE1B0000341C00007A1C0000C21C000044
:10BF3000161D0000741D0000B21D00001C1E000034
:10BF4000521E00009A1E0000E21E00002A1F000080
:10BF5000641F0000AC1F0000F41F0000C80F0000A9
:10BF6000C80F0000C80F00005C200000C80F0000D0
:10BF700092200000BE200000F420000020210000DC
:10BF8000C80F0000C80F0000C80F0000C80F000055
:10BF900056210000A2210000C80F0000C80F0000B9
:10BFA000E8210000382200005E220000C80F0000D7
:10BFB000C80F0000C80F00008C220000BC22000047
:10BFC000EC220000222300004C230000822300000A
:10BFD000AC230000D4230000FC2300002C2400002C
:10BFE0005C24000086240000B0240000E02400004F
:10BFF0000A250000C80F0000C80F0000C80F00008D
:10C00000C80F0000C80F00003A250000802500007E
:10C01000AC250000D8250000042600003A260000C8
:10C0200070260000A6260000DC260000082700007D
:10C03000342700006A270000C80F0000C80F000066
:10C04000C80F0000C80F0000C80F0000C80F000094
:10C05000C80F0000C80F0000C80F0000C80F000084
:10C06000C80F0000C80F0000C80F0000C80F000074
:10C0700096270000CC270000282564206974656D90
:10C08000206C6973742900286F626A656374207478
:10C090007970653A2025642900537461636B2075BB
:10C0A0006E646572666C6F77000000000700000028
:10C0B00003000000F6C00000ED280000FEC00000F4
:10C0C0009D29000007C10000352A000010C10000B2
:10C0D000F128000000000000010000000200000044
:10C0E00003000000040000000A0000006D69637294
:10C0F0006F3A62697400686173546F6E6500706CAA
:10C100006179546F6E6500686173536572766F0074
:10C11000736574536572766F00474320746F6F6B5D
:10C120002025642075736563733B20667265652006
:10C13000256420776F726473003C496E746567658F
:10C14000723E003C4F626A6563743E003C4C69730A
:10C15000743E000D0A564D2050616E69633A2025E9
:10C16000730D0A006D697363000000007CC100005C
:10C170002D34000085C10000E53300006865785467
:10C180006F496E740073696E00000000D8C1000032
:10C1900099340000E0C100009D340000EAC10000B5
:10C1A000BB340000F3C10000C5340000FEC1000034
:10C1B000CF3400000AC20000D93400001BC20000C6
:10C1C000E334000031C20000A73400004AC200007E
:10C1D000B13400006E657400686173576946690088
:10C1E0007374617274576946690073746F7057692C
:10C1F00046690077696669537461747573006D7977
:10C20000495041646472657373007468696E674471
:10C2100065736372697074696F6E00636C656172D7
:10C220005468696E674465736372697074696F6E90
:10C2300000617070656E64546F5468696E67446520
:10C24000736372697074696F6E00617070656E649B
:10C25000546F5468696E6750726F706572747900BC
:10C260001A1B1C03040607090A171819000000000E
:10C270000008080800080A4A4000000A5FEA5FEA6E
:10C280000ED92ED36E19324489330C924C924D083C
:10C290000800000004880808040804848488000A50
:10C2A000448A4000048EC480000000048800000E10
:10C2B000C000000000080001224488100C92525275
:10C2C0004C048C84848E1C824C901E1EC244924C62
:10C2D00006CA525FE21FF01EC13E02448ED12E1FDD
:10C2E000E24488100ED12ED12E0ED12EC488000823
:10C2F00000080000048004880244880482000EC004
:10C300000EC008048244880ED126C0040ED135B375
:10C310006C0C925ED2521C925C925C0ED010100E8D
:10C320001C9252525C1ED01C901E1ED01C90100EEF
:10C33000D013712E12525ED2521C8808081C1FE2C4
:10C3400042524C1254981492101010101E113B754A
:10C35000B131113935B3710C9252524C1C925C9030
:10C36000100C92524C861C925C92510ED00C825C46
:10C370001FE4848484125252524C1131312A4411E8
:10C380003135BB7112524C9252112A4484841EC41E
:10C3900088101E0EC808080E10080482410EC24202
:10C3A000424E048A400000000000001F0804800084
:10C3B00000000ED2524F10101C925C000ED0100ED6
:10C3C00002424ED24E0C925C900E06C81C88080E9B
:10C3D000D24EC24C10101C925208000808080240AD
:10C3E00002424C10149814920808080806001B75A5
:10C3F000B131001C925252000C92524C001C925CC3
:10C4000090000ED24EC2000ED010100006C8049844
:10C4100008080EC807001252524F0011312A44007A
:10C42000113135BB00124C8C9200112A4498001E29
:10C43000C4881E06C48C8486080808080818080CDE
:10C44000881800000C83600000000000010000005C
:10C4500002000000030000000400000005000000CE
:10C4600006000000070000000800000009000000AE
:10C470000A0000000B0000000C0000000D0000008E
:10C480000E0000000F00000010000000120000006D
:10C490001400000016000000180000001A00000040
:10C4A0001C0000001E00000020000000230000000F
:10C4B00026000000290000002C0000002F000000D2
:10C4C00032000000360000003A0000003E0000008C
:10C4D00042000000460000004B0000005000000039
:10C4E000550000005A0000006100000068000000D4
:10C4F0006F000000760000007D0000008400000056
:10C500008B0000009200000099000000A0000000D5
:10C51000A7000000AE000000B5000000BC00000055
:10C52000C3000000CA000000D1000000D8000000D5
:10C53000DF000000E6000000ED000000F400000055
:10C54000FB000000FF00000098C500000935000056
:10C55000A3C50000313A0000ADC50000413700001E
:10C56000BAC5000061370000C1C50000B137000046
:10C57000CAC5000001380000D6C50000DD36000045
:10C58000E7C5000041390000F4C50000FD39000096
:10C59000646973706C6179006C696768744C657666
:10C5A000656C006D62446973706C6179006D624402
:10C5B0006973706C61794F6666006D62506C6F7460
:10C5C000006D62556E706C6F74006D6244726177BD
:10C5D0005368617065006D625368617065466F7283
:10C5E0004C6574746572006E656F506978656C5344
:10C5F000656E64006E656F506978656C5365745044
:10C60000696E004E6F7420656E6F75676820726F7B
:10C610006F6D206576656E20616674657220636F4C
:10C620006D70616374696F6E00436F6D70616374E8
:10C63000656420466C61736820636F646520737461
:10C640006F72650A2564206279746573207573655D
:10C650006420282564252529206F66202564004252
:10C660006164207265636F726420666F756E64200A
:10C67000647572696E6720696E697469616C697A44
:10C680006174696F6E00256420256420256420286C
:10C69000256420776F7264732900256420726563B6
:10C6A0006F7264732C20256420776F7264732C2062
:10C6B0006D617849442025642C20636F6D7061633F
:10C6C00074696F6E206379636C6573202564005212
:10C6D0006573746F7265642025642073637269707A
:10C6E0007473005374617274656400726164696F7D
:10C6F0000000000092C70000F94300009FC700003F
:10C7000095460000AFC7000015460000BDC70000F9
:10C7100029480000C8C7000021440000D8C7000015
:10C72000A9440000ECC7000091440000FBC70000D2
:10C730000B4A000007C800008949000010C800002B
:10C740002D4900001BC800007548000026C80000E5
:10C75000B14800002FC80000E548000038C80000BC
:10C760003144000047C800001144000050C80000D8
:10C77000414400006E756D626572006E6F6E6500FB
:10C780006F74686572007061697200737472696EAB
:10C79000670064697361626C65526164696F006D02
:10C7A000657373616765526563656976656400707A
:10C7B00061636B657452656365697665007061637A
:10C7C0006B657453656E6400726563656976656454
:10C7D000496E746567657200726563656976656444
:10C7E0004D65737361676554797065007265636543
:10C7F00069766564537472696E670073656E644927
:10C800006E74656765720073656E6450616972006D
:10C8100073656E64537472696E6700736574436800
:10C82000616E6E656C0073657447726F757000732E
:10C830006574506F776572007369676E616C5374CD
:10C8400072656E6774680064657669636549440063
:10C850006C6173744D6573736167654944000000D2
:10C8600000000000963007772C610EEEBA5109994E
:10C8700019C46D078FF46A7035A563E9A395649EAA
:10C880003288DB0EA4B8DC791EE9D5E088D9D297CE
:10C890002B4CB609BD7CB17E072DB8E7911DBF902A
:10C8A0006410B71DF220B06A4871B9F3DE41BE844E
:10C8B0007DD4DA1AEBE4DD6D51B5D4F4C785D383AA
:10C8C00056986C13C0A86B647AF962FDECC9658A4E
:10C8D0004F5C0114D96C0663633D0FFAF50D088DAA
:10C8E000C8206E3B5E10694CE44160D5727167A24E
:10C8F000D1E4033C47D4044BFD850DD26BB50AA5AA
:10C90000FAA8B5356C98B242D6C9BBDB40F9BCACCD
:10C91000E36CD832755CDF45CF0DD6DC593DD1AB29
:10C92000AC30D9263A00DE518051D7C81661D0BF4D
:10C93000B5F4B42123C4B3569995BACF0FA5BDB8A9
:10C940009EB802280888055FB2D90CC624E90BB14D
:10C95000877C6F2F114C6858AB1D61C13D2D66B6A9
:10C960009041DC760671DB01BC20D2982A10D5EF0D
:10C970008985B1711FB5B606A5E4BF9F33D4B8E869
:10C98000A2C9077834F9000F8EA8099618980EE10D
:10C99000BB0D6A7F2D3D6D08976C6491015C63E669
:10C9A000F4516B6B62616C1CD83065854E0062F28D
:10C9B000ED95066C7BA5011BC1F4088257C40FF5E9
:10C9C000C6D9B06550E9B712EAB8BE8B7C88B9FC0D
:10C9D000DF1DDD62492DDA15F37CD38C654CD4FB69
:10C9E0005861B24DCE51B53A7400BCA3E230BBD40D
:10C9F00041A5DF4AD795D83D6DC4D1A4FBF4D6D369
:10CA00006AE96943FCD96E34468867ADD0B860DA0C
:10CA1000732D0444E51D03335F4C0AAAC97C0DDD68
:10CA20003C710550AA41022710100BBE86200CC98C
:10CA300025B56857B3856F2009D466B99FE461CEE8
:10CA40000EF9DE5E98C9D9292298D0B0B4A8D7C70C
:10CA5000173DB359810DB42E3B5CBDB7AD6CBAC068
:10CA60002083B8EDB6B3BF9A0CE2B6039AD2B17484
:10CA70003947D5EAAF77D29D1526DB048316DC73E0
:10CA8000120B63E3843B64943E6A6D0DA85A6A7A84
:10CA90000BCF0EE49DFF099327AE000AB19E077DE0
:10CAA00044930FF0D2A3088768F2011EFEC2066904
:10CAB0005D5762F7CB67658071366C19E7066B6E60
:10CAC000761BD4FEE02BD3895A7ADA10CC4ADD6784
:10CAD0006FDFB9F9F9EFBE8E43BEB717D58EB060E0
:10CAE000E8A3D6D67E93D1A1C4C2D83852F2DF4F84
:10CAF000F167BBD16757BCA6DD06B53F4B36B248E0
:10CB0000DA2B0DD84C1B0AAFF64A0336607A044183
:10CB1000C3EF60DF55DF67A8EF8E6E3179BE6946DF
:10CB20008CB361CB1A8366BCA0D26F2536E2685203
:10CB300095770CCC03470BBBB91602222F2605555F
:10CB4000BE3BBAC5280BBDB2925AB42B046AB35C83
:10CB5000A7FFD7C231CFD0B58B9ED92C1DAEDE5BDF
:10CB6000B0C2649B26F263EC9CA36A750A936D02C3
:10CB7000A906099C3F360EEB85670772135700051F
:10CB8000824ABF95147AB8E2AE2BB17B381BB60C43
:10CB90009B8ED2920DBED5E5B7EFDC7C21DFDB0B9F
:10CBA000D4D2D38642E2D4F1F8B3DD686E83DA1FC3
:10CBB000CD16BE815B26B9F6E177B06F7747B7181F
:10CBC000E65A0888706A0FFFCA3B06665C0B0111C3
:10CBD000FF9E658F69AE62F8D3FF6B6145CF6C161F
:10CBE00078E20AA0EED20DD75483044EC2B30339C3
:10CBF000612667A7F71660D04D476949DB776E3E1F
:10CC00004A6AD1AEDC5AD6D9660BDF40F03BD83742
:10CC100053AEBCA9C59EBBDE7FCFB247E9FFB5309E
:10CC20001CF2BDBD8AC2BACA3093B353A6A3B424C2
:10CC30000536D0BA9306D7CD2957DE54BF67D9231E
:10CC40002E7A66B3B84A61C4021B685D942B6F2AC2
:10CC500037BE0BB4A18E0CC31BDF055A8DEF022D1E
:10CC6000416C6C207461736B732073746F707065AA
:10CC700064007630373600202573202573004D651B
:10CC80006D6F727920636C6561726564004E6F2010
:10CC900066726565207461736B20656E7472696578
:10CCA00073000000ECCC0000E95C0000F9CC00004F
:10CCB0007559000005CD00001F5D00000BCD000080
:10CCC0002F5D000011CD00003F5D000017CD00007A
:10CCD000A959000021CD0000515D000029CD0000C0
:10CCE000E95A000073656E736F7273006163636568
:10CCF0006C65726174696F6E0074656D70657261E8
:10CD0000747572650074696C74580074696C745938
:10CD10000074696C745A00746F756368526561645D
:10CD200000693263526561640069326357726974E5
:10CD300065000000A8CD0000D95D0000B6CD000060
:10CD4000DD5D0000BFCD0000E95D0000C9CD000041
:10CD5000ED5D0000D2CD0000F15D0000D7CD0000F8
:10CD6000F55D0000DCCD0000F95D0000E8CD0000BD
:10CD7000FD5D0000EFCD0000015E0000F8CD000079
:10CD8000055E0000FDCD0000095E000008CE000039
:10CD90000D5E000012CE0000E15D00001CCE000020
:10CDA000E55D000074667400656E61626C654469DF
:10CDB00073706C61790067657457696474680067A3
:10CDC000657448656967687400736574506978654F
:10CDD0006C006C696E65007265637400726F756ECD
:10CDE0006465645265637400636972636C650074A2
:10CDF0007269616E676C650074657874007466743E
:10CE0000546F756368656400746674546F75636805
:10CE10005800746674546F7563685900746674546E
:10CE20006F75636850726573737572650057656CD2
:10CE3000636F6D6520746F204D6963726F426C6F14
:10CE4000636B732100000000000000000000000080
:10CE5000A15E00005D5E0000835E00008D5E00004C
:10CE6000975E0000815E0000705F73706920213D55
:10CE7000204E554C4C002F686F6D652F62726F6DA0
:10CE800061676F73612F2E706C6174666F726D696C
:10CE90006F2F7061636B616765732F6672616D657B
:10CEA000776F726B2D61726475696E6F6E6F7264ED
:10CEB00069636E7266352F6C69627261726965733F
:10CEC0002F5350492F5350492E63707000535049CF
:10CED000436C6173733A3A535049436C61737328DE
:10CEE0004E52465F5350495F547970652A2C207525
:10CEF000696E74385F742C2075696E74385F742C99
:10CF00002075696E74385F7429000000030000000A
:10CF10000200000001000000040000000500000005
:10CF2000110000000C0000000B00000012000000C7
:10CF30000A000000060000001A00000014000000B3
:10CF4000170000001600000015000000100000008F
:10CF5000FFFFFFFFFFFFFFFF000000001E000000BB
:10CF60001900000018000000070000000800000081
:10CF7000090000000D0000000E0000000F0000007E
:10CF80001C0000001B0000001D000000130000003A
:10CF90000000000000000000C1640000F16B000010
:10CFA00041650000556500004B650000BD64000050
:10CFB000B164000061650000DD640000AD64000044
:10CFC000000000000000304300000000000030C3FB
:10CFD0007371727400000000FB21F93FFB210940CE
:10CFE0007CD91240FB2119407A6A1F407CD922402B
:10CFF000BBFD2540FB2129403A462C407A6A2F4050
:10D000005C4731407CD932409C6B3440BBFD35409D
:10D01000DB8F3740FB2139401BB43A403A463C4055
:10D020005AD83D407A6A3F404C7E40405C47414080
:10D030006C1042407CD942408CA243409C6B4440DF
:10D04000AC344540BBFD4540CBC64640DB8F474036
:10D05000EB584840FB21494083F9A200444E6E0042
:10D06000FC291500D1572700DD34F50062DBC00034
:10D070003C999500419043006351FE00BBDEAB003C
:10D08000B761C5003A6E2400D24D42004906E00067
:10D0900009EA2E001C92D100EB1DFE0029B11C00F4
:10D0A000E83EA700F535820044BB2E009CE98400D1
:10D0B000B4267000417E5F00D69139005383390059
:10D0C0009CF439008B5F840028F9BD00F81F3B00F9
:10D0D000DEFF97000F980500112FEF000A5A8B0012
:10D0E0006D1F6D00CF7E360009CB2700464FB7007D
:10D0F0009E663F002DEA5F00BA277500E5EBC7008A
:10D100003D7BF100F739070092528A00FB6BEA0081
:10D110001FB15F00085D8D00300356007BFC4600A8
:10D12000F0AB6B0020BCCF0036F49A00E3A91D00E1
:10D130005E619100081BE60085996500A0145F0000
:10D140008D40680080D8FF0027734D00060631002F
:10D15000CA561500C9A873007BE260006B8CC00042
:10D1600000000040FB21F93F000000002D44743E08
:10D17000000000809846F83C0000006051CC783BED
:10D1800000000080831BF0390000004020257A3821
:10D19000000000802282E336000000001DF36935A4
:10D1A0000200000003000000040000000600000070
:10D1B000E88800009288000092880000C089000082
:10D1C0008E8800008E880000B6890000C0890000AB
:10D1D0008E880000B68900008E880000C08900009B
:10D1E000C4890000C4890000C4890000CC89000003
:10D1F000C4930000369200007A920000DE91000095
:10D200007A9200006A9300007A920000DE9100009A
:10D2100036920000369200006A930000DE91000012
:10D22000D6910000D6910000D691000078930000BE
:10D23000EC9A0000EE990000EE9900000C9D0000B1
:10D24000E8990000E8990000F49C00000C9D0000A3
:10D25000E8990000F49C0000E89900000C9D000093
:10D26000029D0000029D0000029D0000109D000034
:10D270002C2066756E6374696F6E3A20006173735B
:10D28000657274696F6E2022257322206661696C55
:10D2900065643A2066696C6520222573222C206C17
:10D2A000696E65202564257325730A0084000020BB
:10D2B000232D302B2000686C4C006566674546477F
:10D2C0000030313233343536373839414243444502
:10D2D0004600303132333435363738396162636471
:10D2E0006566000000000000000000000000000073
:10D2F000000000000000000000000000000000002E
:10D30000000000000000000000000000000000001D
:10D31000000000000000000000000000000000000D
:10D3200000000000000000000000000000000000FD
:10D3300000000000000000000000000000000000ED
:10D34000000000004300504F5349580000202020A7
:10D3500020202020202028282828282020202020A5
:10D360002020202020202020202020202088101075
:10D3700010101010101010101010101010040404D1
:10D38000040404040404041010101010101041418F
:10D39000414141410101010101010101010101017D
:10D3A0000101010101010101101010101010424291
:10D3B000424242420202020202020202020202024D
:10D3C00002020202020202021010101020000000ED
:10D3D000000000000000000000000000000000004D
:10D3E000000000000000000000000000000000003D
:10D3F000000000000000000000000000000000002D
:10D40000000000000000000000000000000000001C
:10D41000000000000000000000000000000000000C
:10D4200000000000000000000000000000000000FC
:10D4300000000000000000000000000000000000EC
:10D4400000000000000000000000000000000000DC
:04D4500000000000D8
:08D45400B42CFF7F0100000071
:10D45C00FFFFFFFF4006000001000000E803DC05B1
:10D46C00DC05DC05DC050000FFFFFFFFFFFFFFFF15
:10D47C001800000019FCFFFFFFFFFFFFFF0000007A
:10D48C000200000003000000FFFFFFFF000000008F
:10D49C00010000000000020001000000FFFFFFFF80
:10D4AC000000000002000000000004000200000068
:10D4BC00FFFFFFFF00000000030000000000080059
:10D4CC00030000000A00000008000000010000003A
:10D4DC00840000200000000004D3000024D30000CE
:10D4EC00E4D200000000000000000000000000007A
:10D4FC000000000000000000000000000000000020
:10D50C00000000000000000000000000000000000F
:10D51C0000000000000000000000000000000000FF
:10D52C0000000000000000000000000000000000EF
:10D53C00000000004300000000000000000000009C
:10D54C0000000000000000000000000000000000CF
:10D55C00000000004300000000000000000000007C
:10D56C0000000000000000000000000000000000AF
:10D57C00000000004300000000000000000000005C
:10D58C00000000000000000000000000000000008F
:10D59C00000000004300000000000000000000003C
:10D5AC00000000000000000000000000000000006F
:10D5BC00000000004300000000000000000000001C
:10D5CC00000000000000000000000000000000004F
:10D5DC0000000000430000000000000000000000FC
:10D5EC00000000000000000000000000000000002F
:10D5FC0000000000430000000000000000000000DC
:10D60C00000000000000000000000000000000000E
:10D61C0000000000D9BB0000F1B5000000000000C4
:10D62C004CD300001ABE000063C1000063C10000AF
:10D63C0063C1000063C1000063C1000063C100004E
:10D64C0063C1000063C1000063C10000FFFFFFFF66
:10D65C00FFFFFFFFFFFFFFFFFFFF00000100415333
:10D66C0043494900000000000000000000000000D9
:10D67C00000000000000000000000000000041530A
:10D68C0043494900000000000000000000000000B9
:10D69C00000000000000000000000000000000007E
:10D6AC00E900000075610000CD6200000D6800000B
:04D6BC00C1000000A9
:040000030000638115
:00000001FF
